:020000040800F2
:1000000000000220A1BF00089DBD0008A5BD00089A
:10001000ADBD0008B5BD0008BDBD00080000000072
:10002000000000000000000000000000C5BD000846
:10003000D3BD000800000000E1BD0008EFBD0008CE
:10004000F1BF0008F1BF0008F1BF0008F1BF0008D0
:10005000F1BF0008F1BF0008F1BF0008F1BF0008C0
:10006000F1BF0008F1BF0008F1BF0008F1BF0008B0
:10007000F1BF0008F1BF0008F1BF0008F1BF0008A0
:10008000F1BF0008F1BF0008F1BF0008F1BF000890
:10009000FDBD000811BE000825BE0008F1BF000824
:1000A000F1BF0008F1BF0008F1BF0008F1BF000870
:1000B000F1BF0008F1BF0008F1BF0008F1BF000860
:1000C000F1BF0008F1BF0008F1BF0008F1BF000850
:1000D000F1BF0008F1BF0008F1BF0008F1BF000840
:1000E00039BE0008F1BF0008F1BF0008F1BF0008E9
:1000F000F1BF0008F1BF0008F1BF0008F1BF000820
:10010000F1BF0008F1BF0008F1BF0008F1BF00080F
:10011000F1BF0008F1BF0008F1BF0008F1BF0008FF
:10012000F1BF0008F1BF0008F1BF0008F1BF0008EF
:10013000F1BF0008F1BF0008F1BF0008F1BF0008DF
:10014000F1BF0008F1BF0008F1BF0008F1BF0008CF
:10015000F1BF0008F1BF0008F1BF0008F1BF0008BF
:10016000F1BF0008F1BF0008F1BF0008F1BF0008AF
:10017000F1BF0008F1BF0008F1BF0008F1BF00089F
:10018000F1BF0008F1BF0008F1BF0008F1BF00088F
:10019000F1BF000800000000F1BF0008F1BF000837
:1001A000F1BF0008F1BF0008F1BF0008F1BF00086F
:1001B000F1BF0008F1BF0008F1BF0008F1BF00085F
:1001C000F1BF0008F1BF0008F1BF0008F1BF00084F
:0801D000F1BF0008F1BF0008B7
:1001E00081F0004102E000BF83F0004330B54FEAE8
:1001F00041044FEA430594EA050F08BF90EA020F55
:100200001FBF54EA000C55EA020C7FEA645C7FEAE7
:10021000655C00F0E2804FEA5454D4EB5555B8BF0A
:100220006D420CDD2C4480EA020281EA030382EA7B
:10023000000083EA010180EA020281EA0303362D0D
:1002400088BF30BD11F0004F4FEA01314FF4801CE0
:100250004CEA113102D0404261EB410113F0004FF2
:100260004FEA03334CEA133302D0524263EB4303A9
:1002700094EA050F00F0A780A4F10104D5F1200E47
:100280000DDB02FA0EFC22FA05F2801841F10001A2
:1002900003FA0EF2801843FA05F359410EE0A5F176
:1002A00020050EF1200E012A03FA0EFC28BF4CF0A7
:1002B000020C43FA05F3C01851EBE37101F000455D
:1002C00007D54FF0000EDCF1000C7EEB00006EEB6A
:1002D0000101B1F5801F1BD3B1F5001F0CD34908F4
:1002E0005FEA30004FEA3C0C04F101044FEA44524B
:1002F00012F5800F80F09A80BCF1004F08BF5FEAD2
:10030000500C50F1000041EB045141EA050130BDB1
:100310005FEA4C0C404141EB0101013C28BFB1F5C3
:10032000801FE9D291F0000F04BF01460020B1FA0E
:1003300081F308BF2033A3F10B03B3F120020CDAE1
:100340000C3208DD02F1140CC2F10C0201FA0CF0BF
:1003500021FA02F10CE002F11402D8BFC2F1200C24
:1003600001FA02F120FA0CFCDCBF41EA0C019040DA
:10037000E41AA2BF01EB0451294330BD6FEA040423
:100380001F3C1CDA0C340EDC04F11404C4F120020E
:1003900020FA04F001FA02F340EA030021FA04F320
:1003A00045EA030130BDC4F10C04C4F1200220FA77
:1003B00002F001FA04F340EA0300294630BD21FAB5
:1003C00004F0294630BD94F0000F83F4801306BF7B
:1003D00081F480110134013D4EE77FEA645C18BF6F
:1003E0007FEA655C29D094EA050F08BF90EA020F06
:1003F00005D054EA000C04BF1946104630BD91EAFE
:10040000030F1EBF0021002030BD5FEA545C05D100
:100410004000494128BF41F0004130BD14F580043F
:100420003CBF01F5801130BD01F0004545F0FE41B3
:1004300041F470014FF0000030BD7FEA645C1ABFE8
:10044000194610467FEA655C1CBF0B46024650EA1F
:10045000013406BF52EA033591EA030F41F400214B
:1004600030BD00BF90F0000F04BF0021704730B5D1
:100470004FF4806404F132044FF000054FF00001A6
:1004800050E700BF90F0000F04BF0021704730B567
:100490004FF4806404F1320410F0004548BF40423C
:1004A0004FF000013EE700BF42004FEAE2014FEA91
:1004B00031014FEA02701FBF12F07F4393F07F4F6C
:1004C00081F06051704732F07F4208BF704793F06F
:1004D0007F4F04BF41F40021704730B54FF4607482
:1004E00001F0004521F000411CE700BF50EA010285
:1004F00008BF704730B54FF000050AE050EA01022E
:1005000008BF704730B511F0004502D5404261EB9D
:1005100041014FF4806404F132045FEA915C3FF4DE
:10052000D8AE4FF003025FEADC0C18BF03325FEA7B
:10053000DC0C18BF033202EBDC02C2F1200300FA2C
:1005400003FC20FA02F001FA03FE40EA0E0021FA51
:1005500002F11444BDE600BF70B54FF0FF0C4CF43F
:10056000E06C1CEA11541DBF1CEA135594EA0C0FF1
:1005700095EA0C0F00F0DEF82C4481EA030621EA2C
:100580004C5123EA4C5350EA013518BF52EA033567
:1005900041F4801143F4801338D0A0FB02CE4FF019
:1005A0000005E1FB02E506F00042E0FB03E54FF049
:1005B0000006E1FB03569CF0000F18BF4EF0010E41
:1005C000A4F1FF04B6F5007F64F5407404D25FEA3D
:1005D0004E0E6D4146EB060642EAC62141EA5551F0
:1005E0004FEAC52040EA5E504FEACE2EB4F1FD0C32
:1005F00088BFBCF5E06F1ED8BEF1004F08BF5FEAB0
:10060000500E50F1000041EB045170BD06F0004661
:1006100046EA010140EA020081EA0301B4EB5C040E
:10062000C2BFD4EB0C0541EA045170BD41F4801106
:100630004FF0000E013C00F3AB8014F1360FDEBF2B
:10064000002001F0004170BDC4F10004203C35DA07
:100650000C341BDC04F11404C4F1200500FA05F38A
:1006600020FA04F001FA05F240EA020001F000422B
:1006700021F0004110EBD37021FA04F642EB0601A1
:100680005EEA430E08BF20EAD37070BDC4F10C04CB
:10069000C4F1200500FA04F320FA05F001FA04F28F
:1006A00040EA020001F0004110EBD37041F100017B
:1006B0005EEA430E08BF20EAD37070BDC4F1200586
:1006C00000FA05F24EEA020E20FA04F301FA05F2EE
:1006D00043EA020321FA04F001F0004121FA04F296
:1006E00020EA020000EBD3705EEA430E08BF20EA66
:1006F000D37070BD94F0000F0FD101F000464000A0
:1007000041EB010111F4801F08BF013CF7D041EA21
:10071000060195F0000F18BF704703F00046520025
:1007200043EB030313F4801F08BF013DF7D043EAF6
:100730000603704794EA0C0F0CEA135518BF95EAAC
:100740000C0F0CD050EA410618BF52EA4306D1D133
:1007500081EA030101F000414FF0000070BD50EA52
:10076000410606BF1046194652EA430619D094EADC
:100770000C0F02D150EA013613D195EA0C0F05D1C6
:1007800052EA03361CBF104619460AD181EA03011A
:1007900001F0004141F0FE4141F470014FF00000D2
:1007A00070BD41F0FE4141F4780170BD70B54FF06D
:1007B000FF0C4CF4E06C1CEA11541DBF1CEA1355ED
:1007C00094EA0C0F95EA0C0F00F0A7F8A4EB0504CF
:1007D00081EA030E52EA03354FEA013100F08880C6
:1007E0004FEA03334FF0805545EA131343EA12638F
:1007F0004FEA022245EA111545EA10654FEA002644
:100800000EF000419D4208BF964244F1FD0404F5FC
:10081000407402D25B084FEA3202B61A65EB030558
:100820005B084FEA32024FF480104FF4002CB6EB15
:10083000020E75EB030E22BFB61A754640EA0C0095
:100840005B084FEA3202B6EB020E75EB030E22BFD5
:10085000B61A754640EA5C005B084FEA3202B6EB16
:10086000020E75EB030E22BFB61A754640EA9C00D5
:100870005B084FEA3202B6EB020E75EB030E22BFA5
:10088000B61A754640EADC0055EA060E18D04FEA63
:10089000051545EA16754FEA06164FEAC30343EA03
:1008A00052734FEAC2025FEA1C1CC0D111F4801FD0
:1008B0000BD141EA00014FF000004FF0004CB6E7C9
:1008C00011F4801F04BF01430020B4F1FD0C88BF68
:1008D000BCF5E06F3FF6AFAEB5EB030C04BFB6EB73
:1008E000020C5FEA500C50F1000041EB045170BD66
:1008F0000EF0004E4EEA113114EB5C04C2BFD4EB93
:100900000C0541EA045170BD41F480114FF0000E16
:10091000013C90E645EA060E8DE60CEA135594EA92
:100920000C0F08BF95EA0C0F3FF43BAF94EA0C0F95
:100930000AD150EA01347FF434AF95EA0C0F7FF40A
:1009400025AF104619462CE795EA0C0F06D152EA5E
:1009500003353FF4FDAE1046194622E750EA410642
:1009600018BF52EA43067FF4C5AE50EA41047FF453
:100970000DAF52EA43057FF4EBAE12E74A0011D205
:1009800012F5001211D20DD56FF47873B3EB6252E9
:100990000ED44FEAC12343F0004343EA505323FAF5
:1009A00002F070474FF00000704750EA013002D16A
:1009B0004FF0FF3070474FF00000704710F8012BE8
:1009C00011F8013B012A28BF9A42F7D0D01A70478C
:1009D00001F0FF01102A2BDB10F0070F08D010F8F0
:1009E000013B013A8B422DD010F0070F42B3F6D1F4
:1009F000F0B441EA012141EA014122F007047FF00D
:100A000000070023F0E80256083C85EA010586EA63
:100A1000010685FA47F5A3FA87F586FA47F6A5FA9F
:100A200087F68EB9EED1F0BC01F0FF0102F00702AB
:100A300032B110F8013B013A83EA010313B1F8D156
:100A40000020704701387047002D06BF3546033837
:100A5000073815F0010F07D1013015F4807F02BF70
:100A6000013015F4C03F0130F0BC0138704700BFC1
:100A700053B94AB9002908BF00281CBF4FF0FF3105
:100A80004FF0FF3000F00CB8ADF1080C6DE904CE6A
:100A900012F0F2FBDDF804E0DDE9022304B0704758
:100AA000704700BF0348044B834202D0034B03B19D
:100AB000184770475802002058020020000000002C
:100AC0000548064B1B1AD90F01EBA301491002D0B0
:100AD000034B03B11847704758020020580200200A
:100AE0000000000010B5064C237843B9FFF7DAFF89
:100AF000044B13B10448AFF300800123237010BDF1
:100B000058020020000000007035010808B5054BB0
:100B10001BB105490548AFF30080BDE80840FFF769
:100B2000CFBF00BF000000005C020020703501084C
:100B300080B400AF064BD3F88830054A43F4700305
:100B4000C2F8883000BFBD465DF8047B704700BF27
:100B500000ED00E080B584B000AF78607B68002BCA
:100B600001D10123C0E07B6893F89132DBB2002B06
:100B700006D17B68002283F8902278680AF0BAF8E0
:100B80007B68032283F891227B681B68184601F07A
:100B90003EFD0023FB733EE0FA7B796813469B0021
:100BA0001344DB000B44113301221A70FA7B79687D
:100BB00013469B001344DB000B441033FA7B1A707E
:100BC000FA7B796813469B001344DB000B44133314
:100BD00000221A70FA7B796813469B001344DB00ED
:100BE0000B44203300221A60FA7B796813469B007D
:100BF0001344DB000B44243300221A60FB7B79682A
:100C00005A1C13469B001344DB000B4400221A605D
:100C1000FB7B0133FB737B681B79FA7B9A42BBD366
:100C20000023FB7344E0FA7B796813469B0013446E
:100C3000DB000B4403F2511300221A70FA7B79682F
:100C400013469B001344DB000B4403F5A873FA7BA7
:100C50001A70FA7B796813469B001344DB000B443F
:100C600003F2531300221A70FA7B796813469B0033
:100C70001344DB000B4403F5B07300221A60FA7BC7
:100C8000796813469B001344DB000B4403F5B273F1
:100C900000221A60FA7B796813469B001344DB003C
:100CA0000B4403F5B47300221A60FB7B0133FB7322
:100CB0007B681B79FA7B9A42B5D37B6818687B689E
:100CC000043393E8060001F0BDFC7B6800221A7330
:100CD0007B68012283F891227B689B7A012B02D1E9
:100CE000786801F053FC002318461037BD4680BDDC
:100CF00080B582B000AF78607B68002B01D1012302
:100D000015E07B68032283F891227B681B681846F4
:100D100003F034FA0346002B01D0012307E0786882
:100D20000AF024F87B68002283F8912200231846F9
:100D30000837BD4680BD80B582B000AF78607B6863
:100D400093F89032012B01D1022312E07B6801223B
:100D500083F890227B681B68184601F041FC7B6891
:100D60001B68184603F035FA7B68002283F890224E
:100D7000002318460837BD4680BD80B582B000AF5D
:100D800078607B6893F89032012B01D1022312E046
:100D90007B68012283F890227B681B68184601F06B
:100DA00036FC7B681B68184603F02AFA7B68002231
:100DB00083F89022002318460837BD4680BD80B5D1
:100DC00084B000AF78607B681B68184603F02DFA8A
:100DD000F860FB6803F40043002B03D0786800F050
:100DE00006FB10E1FB6803F48063002B13D07B68E3
:100DF0001B68B3F844309AB27B681B6822F48062A7
:100E000092B2A3F8442078680AF01FF800217868AD
:100E100000F0FCF8F7E0FB6803F48043002B0CD0F3
:100E20007B681B68B3F844309AB27B681B6822F475
:100E3000804292B2A3F84420E5E0FB6803F400533B
:100E4000002B0CD07B681B68B3F844309AB27B68E7
:100E50001B6822F4005292B2A3F84420D3E0FB684E
:100E600003F48053002B34D07B681B68B3F8403008
:100E70009AB27B681B6822F0040292B2A3F8402069
:100E80007B681B68B3F840309AB27B681B6822F01D
:100E9000080292B2A3F840207B6893F8C832012B75
:100EA00007D17B68002283F8C822002178680AF005
:100EB000F5F978680AF002F87B681B68B3F84430EB
:100EC0009AB27B681B6822F4805292B2A3F8442045
:100ED00099E0FB6803F40063002B27D07B681B6854
:100EE000B3F840309AB27B681B6842F0080292B2B5
:100EF000A3F840207B681B68B3F844309AB27B6843
:100F00001B6822F4006292B2A3F844207B681B683D
:100F1000B3F840309AB27B681B6842F0040292B288
:100F2000A3F84020786809F0AFFF6CE0FB6803F09D
:100F30008003002B40D07B681B68B3F844309AB222
:100F40007B681B6822F0800292B2A3F844207B6881
:100F500093F8C832002B2BD17B681B68B3F8403064
:100F60009AB27B681B6842F0040292B2A3F8402058
:100F70007B681B68B3F840309AB27B681B6842F00C
:100F8000080292B2A3F840207B68012283F8C822AD
:100F90007B681B68B3F854309BB29B0803F03C029B
:100FA0007B68C3F8CC22012178680AF077F92AE03F
:100FB000786809F069FF26E0FB6803F40073002BF2
:100FC0000FD07B681B68B3F844309AB27B681B680B
:100FD00022F4007292B2A3F84420786809F027FF47
:100FE00011E0FB6803F48073002B0CD07B681B6856
:100FF000B3F844309AB27B681B6822F4807292B2D4
:10100000A3F8442000BF1037BD4680BD80B582B034
:1010100000AF78600B46FB707B6893F89032012B31
:1010200001D1022312E07B68012283F890227B68C1
:10103000FA781A737B681B68FA781146184603F031
:10104000B4F87B68002283F8902200231846083702
:10105000BD4680BD80B584B000AF786008461146BB
:101060001A460346FB700B463B801346BB700023B9
:10107000FB7297F90330002B0EDAFB7803F00702BE
:1010800013469B001344DB0010337A681344FB6063
:10109000FB6801225A700EE0FB7803F0070213464A
:1010A0009B001344DB0003F5A8737A681344FB60CC
:1010B000FB6800225A70FB7803F00703DAB2FB6882
:1010C0001A703B88C3F30A02FB681A61FB68BA789E
:1010D000DA70BB78022B02D1FB6800221A717B68A0
:1010E00093F89032012B01D102230EE07B6801229C
:1010F00083F890227B681B68F968184601F0C0FAF3
:101100007B68002283F89022FB7A18461037BD4690
:1011100080BD80B584B000AF78600B46FB7097F956
:101120000330002B0EDAFB7803F0070213469B0016
:101130001344DB0010337A681344FB60FB68012220
:101140005A700EE0FB7803F0070213469B0013442D
:10115000DB0003F5A8737A681344FB60FB68002288
:101160005A70FB7803F00703DAB2FB681A707B68E9
:1011700093F89032012B01D102230EE07B6801220B
:1011800083F890227B681B68F968184601F060FFBD
:101190007B68002283F89022002318461037BD4652
:1011A00080BD80B586B000AFF8607A603B600B46CA
:1011B000FB72FB7A03F0070213469B001344DB002B
:1011C00003F5A873FA6813447B617B697A685A61F6
:1011D0007B693A689A617B690022DA617B69002247
:1011E0005A70FB7A03F00703DAB27B691A70FB6866
:1011F0001B687969184602F018F900231846183759
:10120000BD4680BD80B483B000AF78600B46FB70F4
:10121000FB7803F00702796813469B001344DB0058
:101220000B4403F5B6731B6818460C37BD465DF8D2
:10123000047B704780B586B000AFF8607A603B6091
:101240000B46FB72FB7A03F0070213469B00134424
:10125000DB001033FA6813447B617B697A685A615A
:101260007B693A689A617B69012283F824207B6953
:101270003A681A627B690022DA617B6901225A703E
:10128000FB7A03F00703DAB27B691A70FB681B680C
:101290007969184602F0C9F8002318461837BD4688
:1012A00080BD80B584B000AF78600B46FB70FB78E2
:1012B00003F007037A681279934201D901233EE0D3
:1012C00097F90330002B0EDAFB7803F00702134680
:1012D0009B001344DB0010337A681344FB60FB6807
:1012E00001225A700CE0FA7813469B001344DB008D
:1012F00003F5A8737A681344FB60FB6800225A70F8
:10130000FB6801229A70FB7803F00703DAB2FB68EE
:101310001A707B6893F89032012B01D102230EE002
:101320007B68012283F890227B681B68F968184665
:1013300002F02AFE7B68002283F8902200231846E0
:101340001037BD4680BD80B584B000AF78600B46D5
:10135000FB70FB7803F00F037A681279934201D98E
:10136000012340E097F90330002B0EDAFB7803F0FD
:10137000070213469B001344DB0010337A681344C2
:10138000FB60FB6801225A700EE0FB7803F0070255
:1013900013469B001344DB0003F5A8737A681344DB
:1013A000FB60FB6800225A70FB6800229A70FB7891
:1013B00003F00703DAB2FB681A707B6893F8903287
:1013C000012B01D102230EE07B68012283F89022D9
:1013D0007B681B68F968184602F027FE7B680022CC
:1013E00083F89022002318461037BD4680BD80B593
:1013F00092B000AF786033E37B681B68B3F8443089
:101400007B877B8FDBB203F00F0387F8393097F8C7
:101410003930002B40F008817B8F03F01003002B44
:101420004CD17B681B681B889BB223F4E14323F0FB
:1014300070033B817B681A683B896FEA43436FEA1C
:1014400053439BB213807B6810333B647B681B68FB
:10145000B3F850309BB21A463B6C1B78DB00134448
:101460007A681268134403F202431B88C3F309022B
:101470003B6CDA613B6C5A693B6CDB691A443B6C30
:101480005A610021786809F0B8FC7B681B7BDBB2ED
:10149000002B00F0E5823B6C9B69002B40F0E08262
:1014A0007B681B7BDBB263F07F03DAB27B681B686F
:1014B000A3F84C207B6800221A73D1E27B6803F505
:1014C000A8733B647B681B681B88FB86FB8E03F458
:1014D0000063002B32D07B681B68B3F850309BB29E
:1014E0001A463B6C1B78DB0013447A68126813447D
:1014F00003F206431B88C3F309023B6CDA617B6885
:1015000018687B6803F526713B6CDA883B6CDB69F5
:101510009BB202F0DDFE7B681B681B889AB240F626
:101520008F7313407B817B681B687A8942F080024D
:1015300092B21A80786809F033FC91E2B7F936303C
:10154000002B80F28D827B681B681B889AB240F664
:101550008F731340FB817B681B68FA8942F080021D
:1015600092B21A807B681B68B3F850309BB21A465F
:101570003B6C1B78DB0013447A681268134403F257
:1015800006431B88C3F309023B6CDA613B6CDB69E1
:10159000002B19D03B6C5B69002B15D07B68186859
:1015A0003B6C59693B6CDA883B6CDB699BB202F09F
:1015B0008FFE3B6C5A693B6CDB691A443B6C5A6189
:1015C0000021786809F0FEFB7B681B681B88FB869E
:1015D000FB8E03F40063002B40F04282FB8E03F489
:1015E0004053B3F5405F00F03B827B681B681B886B
:1015F0009BB223F4804323F07003BB81BB8983F447
:101600008053BB81BB8983F40053BB817B681A681C
:10161000BB8943F07F4343F47F0343F4004343F02B
:1016200080039BB213801BE27B681B681A4697F805
:1016300039309B0013441B88FB86B7F93630002BEA
:1016400080F2F1807B681B681A4697F839309B005E
:1016500013441B889AB240F68F731340BB867B6895
:101660001B681A4697F839309B001344BA8E42F033
:10167000800292B21A8097F8392013469B001344D7
:10168000DB0003F5A8737A6813443B643B6C1B7B57
:10169000002B23D17B681B68B3F850309BB21A46ED
:1016A0003B6C1B78DB0013447A681268134403F226
:1016B00006431B88C3F30903A7F84630B7F8463042
:1016C000002B00F08B807B6818683B6C59693B6C81
:1016D000DA88B7F8463002F0FBFD7FE03B6CDB7840
:1016E000022B09D1FB8E1A46396C786800F0C6F9D6
:1016F0000346A7F8463071E07B681B681A463B6CCE
:101700001B789B0013441B889BB223F4E04323F017
:101710007003BB877B681B681A463B6C1B789B0079
:101720001A44BB8F43F07F4343F47F0343F40043E9
:1017300043F0C0039BB213807B681B681A463B6C66
:101740001B789B0013441B889BB203F48043002B3F
:1017500022D07B681B68B3F850309BB21A463B6CB2
:101760001B78DB0013447A681268134403F20243C7
:101770001B88C3F30903A7F84630B7F84630002B9F
:101780002CD07B6818683B6C59693B6C1A89B7F898
:10179000463002F09DFD21E07B681B68B3F85030B5
:1017A0009BB21A463B6C1B78DB0013447A681268C4
:1017B000134403F206431B88C3F30903A7F846301A
:1017C000B7F84630002B09D07B6818683B6C596924
:1017D0003B6C5A89B7F8463002F07AFD3B6CDA6907
:1017E000B7F846301A443B6CDA613B6C5A69B7F87B
:1017F00046301A443B6C5A613B6C9B69002B05D008
:10180000B7F846203B6C1B699A4206D23B6C1B78AA
:101810001946786809F0D6FA05E07B681B68396CD0
:10182000184601F002FEFB8E03F08003002B00F04F
:10183000178197F8392013469B001344DB001033BF
:101840007A6813443B647B681B681A4697F8393002
:101850009B0013441B889BB223F4E14323F07003E5
:10186000FB877B681B681A4697F839309B001A443F
:10187000FB8F6FEA43436FEA53439BB213803B6C89
:10188000DB78012B40F0A1803B6C00229A613B6C1D
:101890001B7B002B00F09280FB8E03F04003002B9B
:1018A00046D03B6C5B78002B26D17B681B687B6144
:1018B0007B681B68B3F850309BB21A467B691344AF
:1018C0007B613B6C1B78DA007B69134403F20243B3
:1018D0003B613B691B889BB2C3F309039AB23B6926
:1018E0001A803B691B889BB26FEA43436FEA5343FC
:1018F0009AB23B691A8061E03B6C5B78012B5DD149
:101900007B681B68FB617B681B68B3F850309BB237
:101910001A46FB691344FB613B6C1B78DA00FB69D8
:10192000134403F20243BB61BB6900221A8045E005
:101930007B681B68FB623B6C5B78002B26D17B6865
:101940001B687B627B681B68B3F850309BB21A46F9
:101950007B6A13447B623B6C1B78DA007B6A13441E
:1019600003F206433B623B6A1B889BB2C3F3090345
:101970009AB23B6A1A803B6A1B889BB26FEA434368
:101980006FEA53439AB23B6A1A8017E03B6C5B786C
:10199000012B13D17B681B68B3F850309BB21A46F9
:1019A000FB6A1344FB623B6C1B78DA00FB6A13444E
:1019B00003F20643BB62BB6A00221A803B6C1B78B1
:1019C0001946786809F019FA4AE0FB8E03F480732F
:1019D000002B3FD17B681B68B3F850309BB21A468E
:1019E0003B6C1B78DB0013447A681268134403F2E3
:1019F00002431B88C3F309037B863B6C9A697B8E89
:101A00009A4206D93B6C9A697B8ED21A3B6C9A61DA
:101A100002E03B6C00229A613B6C9B69002B06D173
:101A20003B6C1B781946786809F0E7F918E03B6CC5
:101A30005A697B8E1A443B6C5A613B6CDA697B8E27
:101A40001A443B6CDA617B681B68396C184601F0FC
:101A5000ECFC05E0FB8E1A46396C786800F017F94B
:101A60007B681B68B3F844309BB21BB2002BFFF6B7
:101A7000C3AC002318464837BD4680BD80B588B04A
:101A800000AFF860B9601346FB80FB8803F4804325
:101A9000002B7CD0FB681B68B3F850309BB21A4611
:101AA000BB681B78DB001344FA681268134403F226
:101AB00002431B88C3F309037B83BB689A697B8B52
:101AC0009A4206D3BB689A697B8BD21ABB689A612B
:101AD00002E0BB6800229A61BB689B69002B23D19E
:101AE000FB681B681A46BB681B789B0013441B8865
:101AF0009BB223F4804323F070033B833B8B83F43E
:101B000000533B83FB681B681A46BB681B789B002D
:101B10001A443B8B43F07F4343F47F0343F4004379
:101B200043F080039BB21380FB8803F04003002B3B
:101B30001FD0FB681B681A46BB681B789B001344C8
:101B40001B889BB223F4E04323F07003FB82FB6805
:101B50001B681A46BB681B789B001A44FB8A43F03B
:101B60007F4343F47F0343F4004343F0C0039BB23D
:101B700013807B8B002B00F08580FB681868BB68A6
:101B80005969BB681A897B8B02F0A2FB7AE0FB687B
:101B90001B68B3F850309BB21A46BB681B78DB0059
:101BA0001344FA681268134403F206431B88C3F314
:101BB00009037B83BB689A697B8B9A4206D3BB6817
:101BC0009A697B8BD21ABB689A6102E0BB680022DB
:101BD0009A61BB689B69002B23D1FB681B681A467E
:101BE000BB681B789B0013441B889BB223F4804383
:101BF00023F07003FB83FB8B83F40053FB83FB68B0
:101C00001B681A46BB681B789B001A44FB8B43F089
:101C10007F4343F47F0343F4004343F080039BB2CC
:101C20001380FB8803F04003002B1FD1FB681B6867
:101C30001A46BB681B789B0013441B889BB223F495
:101C4000E04323F07003BB83FB681B681A46BB6844
:101C50001B789B001A44BB8B43F07F4343F47F0304
:101C600043F4004343F0C0039BB213807B8B002BF3
:101C700008D0FB681868BB685969BB685A897B8BB8
:101C800002F026FB7B8B18462037BD4680BD80B511
:101C9000A6B000AFF860B9601346FB80FB8803F084
:101CA0004003002B00F0F781FB681B68B3F850304D
:101CB0009BB21A46BB681B78DB001344FA681268B3
:101CC000134403F202431B88C3F30903A7F89630B9
:101CD000BB689A69B7F896309A4207D9BB689A6987
:101CE000B7F89630D21ABB689A6102E0BB6800224E
:101CF0009A61BB689B69002B40F0E180BB685B7810
:101D0000002B26D1FB681B683B63FB681B68B3F89C
:101D100050309BB21A463B6B13443B63BB681B7845
:101D2000DA003B6B134403F20243FB62FB6A1B883D
:101D30009BB2C3F309039AB2FB6A1A80FB6A1B8841
:101D40009BB26FEA43436FEA53439AB2FB6A1A802D
:101D50001AE0BB685B78012B16D1FB681B68BB637C
:101D6000FB681B68B3F850309BB21A46BB6B134438
:101D7000BB63BB681B78DA00BB6B134403F20243FE
:101D80007B637B6B00221A80FB681B68BB62BB68AD
:101D90005B78002B26D1FB681B683B62FB681B68E5
:101DA000B3F850309BB21A463B6A13443B62BB689F
:101DB0001B78DA003B6A134403F20643FB61FB69BC
:101DC0001B889BB2C3F309039AB2FB691A80FB69B3
:101DD0001B889BB26FEA43436FEA53439AB2FB6995
:101DE0001A8017E0BB685B78012B13D1FB681B6876
:101DF000B3F850309BB21A46BB6A1344BB62BB684F
:101E00001B78DA00BB6A134403F206437B627B6AE9
:101E100000221A80BB68DB78022B23D1FB681B6889
:101E20001A46BB681B789B0013441B889BB223F4A3
:101E3000E04323F040037B837B8B83F020037B8391
:101E4000FB681B681A46BB681B789B001A447B8B97
:101E500043F07F4343F47F0343F4004343F08003A4
:101E60009BB21380BB681B781946F86808F0C5FF61
:101E7000FB8803F48043002B1FD0FB681B681A46C5
:101E8000BB681B789B0013441B889BB223F4E04380
:101E900023F070033B83FB681B681A46BB681B7802
:101EA0009B001A443B8B43F07F4343F47F0343F48E
:101EB000404343F080039BB2138000231FE3FB8861
:101EC00003F48043002B21D0FB681B681A46BB68D3
:101ED0001B789B0013441B889BB223F4E04323F040
:101EE0007003A7F84E30FB681B681A46BB681B7866
:101EF0009B001A44B7F84E3043F07F4343F47F030E
:101F000043F4404343F080039BB21380BB6893F8D3
:101F10002430012B40F0CA82BB685A69B7F896306A
:101F20001A44BB685A61BB68DA69B7F896301A443C
:101F3000BB68DA61BB681A6ABB681B699A4209D33D
:101F4000BB681B69BB65BB681A6ABB6DD21ABB68EC
:101F50001A6215E0BB681B6A002B07D1B7F89630F0
:101F6000BB65BB68002283F8242009E0BB6800221F
:101F700083F82420BB681B6ABB65BB6800221A6219
:101F8000BB685B78002B5FD1FB681B683B64FB6818
:101F90001B68B3F850309BB21A463B6C13443B6449
:101FA000BB681B78DA003B6C134403F20243FB630B
:101FB000FB6B1B889BB2C3F309039AB2FB6B1A80BD
:101FC000BB6D002B0AD1FB6B1B889BB26FEA4343AE
:101FD0006FEA53439AB2FB6B1A8051E0BB6D3E2B04
:101FE00016D8BB6D5B083B65BB6D03F00103002B8E
:101FF00002D03B6D01333B65FB6B1B889AB23B6D96
:102000009BB29B029BB213439AB2FB6B1A8037E0E0
:10201000BB6D5B093B65BB6D03F01F03002B02D159
:102020003B6D013B3B65FB6B1B889AB23B6D9BB2E2
:102030009B029BB213439BB26FEA43436FEA534345
:102040009AB2FB6B1A801BE0BB685B78012B17D13F
:10205000FB681B68BB64FB681B68B3F850309BB21D
:102060001A46BB6C1344BB64BB681B78DA00BB6CBC
:10207000134403F202437B64BB6D9AB27B6C1A80FB
:10208000FB681868BB685969BB681A89BB6D9BB24D
:1020900002F0DBF80AE2FB681B68B3F850309BB231
:1020A0001A46BB681B78DB001344FA6812681344B5
:1020B00003F206431B88C3F30903A7F89630BB68F5
:1020C0009A69B7F896309A4207D3BB689A69B7F80D
:1020D0009630D21ABB689A6102E0BB6800229A610E
:1020E000BB689B69002B40F0F680BB685B78002BD7
:1020F00026D1FB681B687B67FB681B68B3F8503010
:102100009BB21A467B6F13447B67BB681B78DA006F
:102110007B6F134403F202433B673B6F1B889BB208
:10212000C3F309039AB23B6F1A803B6F1B889BB2C3
:102130006FEA43436FEA53439AB23B6F1A801AE047
:10214000BB685B78012B16D1FB681B68FB67FB68DB
:102150001B68B3F850309BB21A46FB6F1344FB6701
:10216000BB681B78DA00FB6F134403F20243BB67C2
:10217000BB6F00221A80FB681B68C7F88430BB68FD
:102180005B78002B2FD1FB681B68C7F88C30FB688D
:102190001B68B3F850309BB21A46D7F88C30134402
:1021A000C7F88C30BB681B78DA00D7F88C30134442
:1021B00003F20643C7F88830D7F888301B889BB2F3
:1021C000C3F309039AB2D7F888301A80D7F8883059
:1021D0001B889BB26FEA43436FEA53439AB2D7F826
:1021E00088301A801CE0BB685B78012B18D1FB6833
:1021F0001B68B3F850309BB21A46D7F884301344AA
:10220000C7F88430BB681B78DA00D7F884301344F1
:1022100003F20643C7F88030D7F8803000221A80D6
:10222000BB68DB78022B27D1FB681B681A46BB68AA
:102230001B789B0013441B889BB223F4E04323F0DC
:102240004003A7F89430B7F8943083F02003A7F840
:102250009430FB681B681A46BB681B789B001A44C5
:10226000B7F8943043F07F4343F47F0343F40043D3
:1022700043F080039BB21380BB681B781946F86853
:1022800008F0BBFDFB8803F48043002B21D1FB68E1
:102290001B681A46BB681B789B0013441B889BB2C3
:1022A00023F4E04323F07003A7F89230FB681B6827
:1022B0001A46BB681B789B001A44B7F8923043F06B
:1022C0007F4343F47F0343F4404343F080039BB2D6
:1022D0001380002313E1FB8803F48043002B21D1FA
:1022E000FB681B681A46BB681B789B0013441B885D
:1022F0009BB223F4E04323F07003A7F85630FB6849
:102300001B681A46BB681B789B001A44B7F8563006
:1023100043F07F4343F47F0343F4404343F080039F
:102320009BB21380BB6893F82430012B40F0BE8031
:10233000BB685A69B7F896301A44BB685A61BB68E3
:10234000DA69B7F896301A44BB68DA61BB681A6A72
:10235000BB681B699A4209D3BB681B69BB65BB6834
:102360001A6ABB6DD21ABB681A6215E0BB681B6A99
:10237000002B07D1B7F89630BB65BB68002283F805
:10238000242009E0BB681B6ABB65BB6800221A6297
:10239000BB68002283F82420FB681B68FB65BB68D0
:1023A0005B78002B5FD1FB681B68BB66FB681B6812
:1023B000B3F850309BB21A46BB6E1344BB66BB6881
:1023C0001B78DA00BB6E134403F206437B667B6E18
:1023D0001B889BB2C3F309039AB27B6E1A80BB6D54
:1023E000002B0AD17B6E1B889BB26FEA43436FEAD6
:1023F00053439AB27B6E1A804EE0BB6D3E2B16D8CB
:10240000BB6D5B083B66BB6D03F00103002B02D084
:102410003B6E01333B667B6E1B889AB23B6E9BB270
:102420009B029BB213439AB27B6E1A8034E0BB6D61
:102430005B093B66BB6D03F01F03002B02D13B6EB3
:10244000013B3B667B6E1B889AB23B6E9BB29B0244
:102450009BB213439BB26FEA43436FEA53439AB272
:102460007B6E1A8018E0BB685B78012B14D1FB6887
:102470001B68B3F850309BB21A46FB6D1344FB65E2
:10248000BB681B78DA00FB6D134403F20643FB665E
:10249000BB6D9AB2FB6E1A80FB681868BB685969FD
:1024A000BB685A89BB6D9BB201F0CFFEFB681B680D
:1024B0001A46BB681B789B0013441B889BB223F40D
:1024C000E04323F04003FB82FB8A83F01003FB828E
:1024D000FB8A83F02003FB82FB681B681A46BB68FB
:1024E0001B789B001A44FB8A43F07F4343F47F032D
:1024F00043F4004343F080039BB21380002318464B
:102500009837BD4680BD80B487B000AFF8607B606F
:102510000B467B8113463B817B8903F080039BB292
:10252000002B0BD07B8903F0070213469B0013445A
:10253000DB001033FA6813447B6109E07A891346A3
:102540009B001344DB0003F5A873FA6813447B6116
:102550003B89002B07D17B6900221A737B689AB2F2
:102560007B69DA800BE07B6901221A737B689AB27F
:102570007B691A817B681B0C9AB27B695A810023A4
:1025800018461C37BD465DF8047B704780B485B0A3
:1025900000AF78607B681B68FB607B680122C3F832
:1025A000D0227B68002283F8C822FB68B3F854303D
:1025B0009BB243F001039AB2FB68A3F85420FB6876
:1025C000B3F854309BB243F002039AB2FB68A3F80D
:1025D0005420002318461437BD465DF8047B70472D
:1025E00080B485B000AF78607B680022A3F84420F7
:1025F0004BF68073FB60FB689AB27B68A3F84020BF
:10260000002318461437BD465DF8047B704780B43C
:1026100085B000AF78604BF68073FB607B68B3F8E1
:1026200040309AB2FB689BB2DB439BB213409AB234
:102630007B68A3F84020002318461437BD465DF898
:10264000047B704780B485B000AFF8603B1D83E821
:102650000600FB680122A3F84020FB680022A3F8D3
:102660004020FB680022A3F84420FB680022A3F866
:102670005020002318461437BD465DF8047B704790
:1026800080B4A7B000AF78603960002387F8973036
:102690007A683B681B789B0013441B889BB223F429
:1026A000EC4323F07003A7F894303B68DB78032BEE
:1026B0001FD801A252F823F0C9260008E526000819
:1026C000FB260008D7260008B7F8943043F40073BF
:1026D000A7F8943012E0B7F8943043F4C063A7F839
:1026E00094300BE0B7F8943043F48063A7F894304B
:1026F00004E0012387F8973000E000BF7A683B6868
:102700001B789B001A44B7F8943043F07F4343F49E
:102710007F0343F4004343F080039BB213807A6845
:102720003B681B789B0013441B889BB21BB223F4AD
:10273000E04323F070031AB23B681B781BB21343CB
:102740001BB2A7F886307A683B681B789B001A4456
:10275000B7F8863043F07F4343F47F0343F40043EC
:1027600043F080039BB213803B681B7B002B40F03F
:1027700080813B685B78002B00F084807B68BB61C4
:102780007B68B3F850309BB21A46BB691344BB61F7
:102790003B681B78DA00BB69134403F580637B61F7
:1027A0003B68DB885B089BB25B009AB27B691A804E
:1027B0007A683B681B789B0013441B887B827B8A6A
:1027C00003F04003002B1BD07A683B681B789B000A
:1027D00013441B889BB223F4E04323F070033B8235
:1027E0007A683B681B789B001A443B8A43F07F431E
:1027F00043F47F0343F4004343F0C0039BB21380D0
:102800003B68DB78012B20D07A683B681B789B0003
:1028100013441B889BB223F4E04323F04003BB81A5
:10282000BB8983F02003BB817A683B681B789B00DF
:102830001A44BB8943F07F4343F47F0343F40043CE
:1028400043F080039BB21380F9E37A683B681B78FE
:102850009B0013441B889BB223F4E04323F0400306
:10286000FB817A683B681B789B001A44FB8943F024
:102870007F4343F47F0343F4004343F080039BB260
:102880001380DCE37B683B637B68B3F850309BB21A
:102890001A463B6B13443B633B681B78DA003B6B87
:1028A000134403F20443FB623B68DB885B089BB282
:1028B0005B009AB2FB6A1A807B68BB627B68B3F8E4
:1028C00050309BB21A46BB6A1344BB623B681B780C
:1028D000DA00BB6A134403F206437B627B6A1B88FF
:1028E0009BB2C3F309039AB27B6A1A803B681B69E7
:1028F000002B0AD17B6A1B889BB26FEA43436FEAC5
:1029000053439AB27B6A1A8041E03B681B693E2BB5
:102910001CD83B681B695B08C7F890303B681B6993
:1029200003F00103002B04D0D7F890300133C7F82F
:1029300090307B6A1B889AB2D7F890309BB29B028A
:102940009BB213439AB27B6A1A8020E03B681B69F2
:102950005B09C7F890303B681B6903F01F03002B2D
:1029600004D1D7F89030013BC7F890307B6A1B88C0
:102970009AB2D7F890309BB29B029BB213439BB2A2
:102980006FEA43436FEA53439AB27B6A1A807A68CC
:102990003B681B789B0013441B887B847B8C03F46F
:1029A0008043002B1BD07A683B681B789B00134444
:1029B0001B889BB223F4E04323F070033B847A68C6
:1029C0003B681B789B001A443B8C43F07F4343F4E5
:1029D0007F0343F4404343F080039BB213803B6882
:1029E0001B78002B24D17A683B681B789B0013442A
:1029F0001B889BB223F4804323F07003BB83BB8B03
:102A000083F48053BB83BB8B83F40053BB837A680E
:102A10003B681B789B001A44BB8B43F07F4343F415
:102A20007F0343F4004343F080039BB2138006E32B
:102A30007A683B681B789B0013441B889BB223F485
:102A4000804323F07003FB83FB8B83F40053FB83F1
:102A50007A683B681B789B001A44FB8B43F07F43EA
:102A600043F47F0343F4004343F080039BB213809D
:102A7000E5E23B68DB78022B1ED17A683B681B7865
:102A80009B0013441B889BB223F4E04323F07003A4
:102A9000A7F882307A683B681B789B001A44B7F825
:102AA000823043F07F4343F47F0343F4014343F018
:102AB00080039BB213801DE07A683B681B789B0003
:102AC00013441B889BB223F4E24323F07003A7F85E
:102AD00084307A683B681B789B001A44B7F88430CE
:102AE00043F07F4343F47F0343F4004343F0800308
:102AF0009BB213807B68FB677B68B3F850309BB256
:102B00001A46FB6F1344FB673B681B78DA00FB6FC8
:102B1000134403F58063BB673B681B895B089BB26A
:102B20005B009AB2BB6F1A807B687B677B68B3F8E7
:102B300050309BB21A467B6F13447B673B681B780F
:102B4000DA007B6F134403F204433B673B685B8905
:102B50005B089BB25B009AB23B6F1A803B685B7864
:102B6000002B40F0AF817A683B681B789B001344D0
:102B70001B88A7F86030B7F8603003F48043002B5F
:102B80001DD07A683B681B789B0013441B889BB25E
:102B900023F4E04323F07003A7F85E307A683B68C3
:102BA0001B789B001A44B7F85E3043F07F4343F430
:102BB0007F0343F4404343F080039BB213807A6861
:102BC0003B681B789B0013441B88A7F85C30B7F860
:102BD0005C3003F04003002B1DD07A683B681B7803
:102BE0009B0013441B889BB223F4E04323F0700343
:102BF000A7F85A307A683B681B789B001A44B7F8EC
:102C00005A3043F07F4343F47F0343F4004343F0DF
:102C1000C0039BB213803B685B78002B6BD17B6851
:102C2000FB647B68B3F850309BB21A46FB6C1344CC
:102C3000FB643B681B78DA00FB6C134403F202432D
:102C4000BB64BB6C1B889BB2C3F309039AB2BB6C19
:102C50001A803B681B69002B0AD1BB6C1B889BB296
:102C60006FEA43436FEA53439AB2BB6C1A805DE04C
:102C70003B681B693E2B1CD83B681B695B08C7F887
:102C80008C303B681B6903F00103002B04D0D7F89C
:102C90008C300133C7F88C30BB6C1B889AB2D7F8E4
:102CA0008C309BB29B029BB213439AB2BB6C1A80CE
:102CB0003CE03B681B695B09C7F88C303B681B69CB
:102CC00003F01F03002B04D1D7F88C30013BC7F869
:102CD0008C30BB6C1B889AB2D7F88C309BB29B02AD
:102CE0009BB213439BB26FEA43436FEA53439AB2DA
:102CF000BB6C1A801AE03B685B78012B16D17B68AD
:102D00007B657B68B3F850309BB21A467B6D1344E9
:102D10007B653B681B78DA007B6D134403F202434A
:102D20003B653B681B699AB23B6D1A807B687B648C
:102D30003B685B78002B6BD17B68FB637B68B3F8E7
:102D400050309BB21A46FB6B1344FB633B681B7805
:102D5000DA00FB6B134403F20643BB63BB6B1B88B7
:102D60009BB2C3F309039AB2BB6B1A803B681B6921
:102D7000002B0AD1BB6B1B889BB26FEA43436FEAFF
:102D800053439AB2BB6B1A805BE03B681B693E2BD6
:102D90001CD83B681B695B08C7F888303B681B6917
:102DA00003F00103002B04D0D7F888300133C7F8B3
:102DB0008830BB6B1B889AB2D7F888309BB29B02D5
:102DC0009BB213439AB2BB6B1A803AE03B681B6913
:102DD0005B09C7F888303B681B6903F01F03002BB1
:102DE00004D1D7F88830013BC7F88830BB6B1B880B
:102DF0009AB2D7F888309BB29B029BB213439BB226
:102E00006FEA43436FEA53439AB2BB6B1A8018E0F0
:102E10003B685B78012B14D17B68B3F850309BB2D0
:102E20001A467B6C13447B643B681B78DA007B6C2E
:102E3000134403F206433B643B681B699AB23B6C44
:102E40001A807A683B681B789B0013441B889BB2EE
:102E500023F4804323F07003FB86FB8E83F48053BE
:102E6000FB86FB8E83F40053FB867A683B681B78F5
:102E70009B001A44FB8E43F07F4343F47F0343F4EB
:102E8000004343F080039BB213807A683B681B7851
:102E90009B0013441B889BB223F4E04323F04003C0
:102EA000BB867A683B681B789B001A44BB8E43F054
:102EB0007F4343F47F0343F4004343F080039BB21A
:102EC0001380BCE07A683B681B789B0013441B8826
:102ED000A7F86E30B7F86E3003F48043002B1DD096
:102EE0007A683B681B789B0013441B889BB223F4D1
:102EF000E04323F07003A7F86C307A683B681B78D6
:102F00009B001A44B7F86C3043F07F4343F47F03CF
:102F100043F4404343F080039BB213807A683B68DC
:102F20001B789B0013441B88A7F86A30B7F86A30F7
:102F300003F04003002B1DD07A683B681B789B0090
:102F400013441B889BB223F4E04323F07003A7F8DB
:102F500068307A683B681B789B001A44B7F8683081
:102F600043F07F4343F47F0343F4004343F0C00343
:102F70009BB213803B68DB78012B24D07A683B68D6
:102F80001B789B0013441B889BB223F4E04323F07F
:102F90004003A7F86430B7F8643083F02003A7F843
:102FA00064307A683B681B789B001A44B7F8643039
:102FB00043F07F4343F47F0343F4004343F0800333
:102FC0009BB213801DE07A683B681B789B0013441A
:102FD0001B889BB223F4E04323F04003A7F866303C
:102FE0007A683B681B789B001A44B7F8663043F058
:102FF0007F4343F47F0343F4004343F080039BB2D9
:1030000013807A683B681B789B0013441B889BB233
:1030100023F4804323F07003A7F862307A683B689A
:103020001B789B001A44B7F8623043F07F4343F4A7
:103030007F0343F4004343F080039BB2138097F86F
:10304000973018469C37BD465DF8047B704700BF3B
:1030500080B48DB000AF786039603B681B7B002B7B
:1030600040F08E803B685B78002B44D07A683B68E8
:103070001B789B0013441B88BB81BB8903F0400372
:10308000002B1BD07A683B681B789B0013441B887D
:103090009BB223F4E04323F070037B817A683B68A2
:1030A0001B789B001A447B8943F07F4343F47F03E2
:1030B00043F4004343F0C0039BB213807A683B683B
:1030C0001B789B0013441B889BB223F4E04323F03E
:1030D00040033B817A683B681B789B001A443B891C
:1030E00043F07F4343F47F0343F4004343F0800302
:1030F0009BB2138092E17A683B681B789B00134473
:103100001B887B827B8A03F48043002B1BD07A6868
:103110003B681B789B0013441B889BB223F4E0435D
:1031200023F070033B827A683B681B789B001A444B
:103130003B8A43F07F4343F47F0343F4404343F02F
:1031400080039BB213807A683B681B789B00134412
:103150001B889BB223F4804323F07003FB817A68C1
:103160003B681B789B001A44FB8943F07F4343F480
:103170007F0343F4004343F080039BB213804DE18F
:103180003B685B78002B40F0A5807A683B681B7831
:103190009B0013441B883B843B8C03F48043002B2F
:1031A0001BD07A683B681B789B0013441B889BB23A
:1031B00023F4E04323F07003FB837A683B681B78B9
:1031C0009B001A44FB8B43F07F4343F47F0343F49B
:1031D000404343F080039BB213807A683B681B78BE
:1031E0009B0013441B88BB83BB8B03F04003002B65
:1031F0001BD07A683B681B789B0013441B889BB2EA
:1032000023F4E04323F070037B837A683B681B78E8
:103210009B001A447B8B43F07F4343F47F0343F4CA
:10322000004343F0C0039BB213807A683B681B786D
:103230009B0013441B889BB223F4E04323F07003EC
:103240003B837A683B681B789B001A443B8B43F0B6
:103250007F4343F47F0343F4004343F0C0039BB236
:1032600013807A683B681B789B0013441B889BB2D1
:1032700023F4804323F07003FB827A683B681B7859
:103280009B001A44FB8A43F07F4343F47F0343F4DB
:10329000004343F080039BB213807A683B681B783D
:1032A0009B0013441B889BB223F4E04323F04003AC
:1032B000BB827A683B681B789B001A44BB8A43F048
:1032C0007F4343F47F0343F4004343F080039BB206
:1032D0001380A3E07A683B681B789B0013441B882B
:1032E000FB85FB8D03F48043002B1BD07A683B6881
:1032F0001B789B0013441B889BB223F4E04323F00C
:103300007003BB857A683B681B789B001A44BB8DB1
:1033100043F07F4343F47F0343F4404343F080038F
:103320009BB213807A683B681B789B0013441B8810
:103330007B857B8D03F04003002B1BD07A683B68B4
:103340001B789B0013441B889BB223F4E04323F0BB
:1033500070033B857A683B681B789B001A443B8D61
:1033600043F07F4343F47F0343F4004343F0C0033F
:103370009BB213807A683B681B789B0013441B88C0
:103380009BB223F4E04323F07003FB847A683B682C
:103390001B789B001A44FB8C43F07F4343F47F036C
:1033A00043F4404343F080039BB213807A683B6848
:1033B0001B789B0013441B889BB223F4E04323F04B
:1033C0004003BB847A683B681B789B001A44BB8C23
:1033D00043F07F4343F47F0343F4004343F080030F
:1033E0009BB213807A683B681B789B0013441B8850
:1033F0009BB223F4804323F070037B847A683B689C
:103400001B789B001A447B8C43F07F4343F47F037B
:1034100043F4004343F080039BB21380002318461B
:103420003437BD465DF8047B704780B5ACB000AF63
:10343000786039603B685B78012B40F0CA843B6858
:103440009A693B681B699A4204D93B681B69C7F8B3
:10345000AC3003E03B689B69C7F8AC303B681B7B32
:10346000002B22D13B6859693B68DA88D7F8AC3029
:103470009BB2786800F0E9FE7B683B617B68B3F83B
:1034800050309BB21A463B6913443B613B681B7842
:10349000DA003B69134403F20243FB60D7F8AC3017
:1034A0009AB2FB681A8000F06FBC3B68DB78022B95
:1034B00040F01E833B681A6A3B681B699A4240F2DF
:1034C000CF827A683B681B789B0013441B889BB2B1
:1034D00023F4E04323F07003A7F856307A683B6882
:1034E0001B789B001A44B7F8563043F07F4343F4EF
:1034F0007F0343F4014343F080039BB213803B6896
:103500001A6AD7F8AC30D21A3B681A627A683B68FC
:103510001B789B0013441B889BB203F04003002BD5
:1035200000F04F817B683B633B685B78002B6BD17D
:103530007B68BB627B68B3F850309BB21A46BB6AAB
:103540001344BB623B681B78DA00BB6A134403F286
:1035500006437B627B6A1B889BB2C3F309039AB262
:103560007B6A1A80D7F8AC30002B0AD17B6A1B88A3
:103570009BB26FEA43436FEA53439AB27B6A1A8065
:103580005BE0D7F8AC303E2B1CD8D7F8AC305B08EA
:10359000C7F8A830D7F8AC3003F00103002B04D0F3
:1035A000D7F8A8300133C7F8A8307B6A1B889AB2D5
:1035B000D7F8A8309BB29B029BB213439AB27B6AA6
:1035C0001A803AE0D7F8AC305B09C7F8A830D7F8D2
:1035D000AC3003F01F03002B04D1D7F8A830013B17
:1035E000C7F8A8307B6A1B889AB2D7F8A8309BB27C
:1035F0009B029BB213439BB26FEA43436FEA534370
:103600009AB27B6A1A8018E03B685B78012B14D170
:103610007B68B3F850309BB21A463B6B13443B6354
:103620003B681B78DA003B6B134403F20643FB62F2
:10363000D7F8AC309AB2FB6A1A803B685B89A7F86E
:1036400076303B685969D7F8AC309BB2B7F8762032
:10365000786800F0FAFD3B685A69D7F8AC301A4434
:103660003B685A613B681A6A3B681B699A4207D9F2
:103670003B681A6AD7F8AC30D21A3B681A6206E087
:103680003B681B6AC7F8AC303B6800221A623B6893
:103690005B78002B6BD17B68BB617B68B3F85030E3
:1036A0009BB21A46BB691344BB613B681B78DA00C6
:1036B000BB69134403F202437B617B691B889BB2A5
:1036C000C3F309039AB27B691A80D7F8AC30002B98
:1036D0000AD17B691B889BB26FEA43436FEA53436D
:1036E0009AB27B691A805DE0D7F8AC303E2B1CD8CB
:1036F000D7F8AC305B08C7F8A430D7F8AC3003F08B
:103700000103002B04D0D7F8A4300133C7F8A4304C
:103710007B691B889AB2D7F8A4309BB29B029BB2FC
:1037200013439AB27B691A803CE0D7F8AC305B094E
:10373000C7F8A430D7F8AC3003F01F03002B04D136
:10374000D7F8A430013BC7F8A4307B691B889AB234
:10375000D7F8A4309BB29B029BB213439BB26FEA93
:1037600043436FEA53439AB27B691A801AE03B687D
:103770005B78012B16D17B683B627B68B3F85030D5
:103780009BB21A463B6A13443B623B681B78DA00E3
:103790003B6A134403F20243FB61D7F8AC309AB2A0
:1037A000FB691A803B681B89A7F876303B6859692A
:1037B000D7F8AC309BB2B7F87620786800F045FDBA
:1037C000E2E23B685B78002B6BD17B68BB647B6873
:1037D000B3F850309BB21A46BB6C1344BB643B68D1
:1037E0001B78DA00BB6C134403F202437B647B6CEE
:1037F0001B889BB2C3F309039AB27B6C1A80D7F87B
:10380000AC30002B0AD17B6C1B889BB26FEA434320
:103810006FEA53439AB27B6C1A805DE0D7F8AC3004
:103820003E2B1CD8D7F8AC305B08C7F8A030D7F8CF
:10383000AC3003F00103002B04D0D7F8A0300133E3
:10384000C7F8A0307B6C1B889AB2D7F8A0309BB227
:103850009B029BB213439AB27B6C1A803CE0D7F870
:10386000AC305B09C7F8A030D7F8AC3003F01F03C9
:10387000002B04D1D7F8A030013BC7F8A0307B6CF7
:103880001B889AB2D7F8A0309BB29B029BB213431D
:103890009BB26FEA43436FEA53439AB27B6C1A8040
:1038A0001AE03B685B78012B16D17B683B657B682F
:1038B000B3F850309BB21A463B6D13443B653B68EE
:1038C0001B78DA003B6D134403F20243FB64D7F824
:1038D000AC309AB2FB6C1A803B681B89A7F8763033
:1038E0003B685969D7F8AC309BB2B7F87620786856
:1038F00000F0ABFC3B685A69D7F8AC301A443B681F
:103900005A613B681A6A3B681B699A4207D93B684F
:103910001A6AD7F8AC30D21A3B681A6206E03B68E4
:103920001B6AC7F8AC303B6800221A627B683B64B4
:103930003B685B78002B6BD17B68BB637B68B3F81B
:1039400050309BB21A46BB6B1344BB633B681B7879
:10395000DA00BB6B134403F206437B637B6B1B886B
:103960009BB2C3F309039AB27B6B1A80D7F8AC30D1
:10397000002B0AD17B6B1B889BB26FEA43436FEA33
:1039800053439AB27B6B1A805BE0D7F8AC303E2B86
:103990001CD8D7F8AC305B08C7F89C30D7F8AC30EF
:1039A00003F00103002B04D0D7F89C300133C7F893
:1039B0009C307B6B1B889AB2D7F89C309BB29B02E1
:1039C0009BB213439AB27B6B1A803AE0D7F8AC30C3
:1039D0005B09C7F89C30D7F8AC3003F01F03002B0D
:1039E00004D1D7F89C30013BC7F89C307B6B1B8817
:1039F0009AB2D7F89C309BB29B029BB213439BB206
:103A00006FEA43436FEA53439AB27B6B1A8018E024
:103A10003B685B78012B14D17B68B3F850309BB2C4
:103A20001A463B6C13443B643B681B78DA003B6CE2
:103A3000134403F20643FB63D7F8AC309AB2FB6B36
:103A40001A803B685B89A7F876303B685969D7F8DC
:103A5000AC309BB2B7F87620786800F0F6FB93E1C3
:103A60003B681B6AC7F8AC307A683B681B789B00E0
:103A700013441B889BB223F4E24323F07003A7F89E
:103A800062307A683B681B789B001A44B7F8623052
:103A900043F07F4343F47F0343F4004343F0800348
:103AA0009BB213807B68FB657B68B3F850309BB298
:103AB0001A46FB6D1344FB653B681B78DA00FB6D0F
:103AC000134403F20243BB65D7F8AC309AB2BB6D26
:103AD0001A803B681B89A7F876303B685969D7F88C
:103AE000AC309BB2B7F87620786800F0AEFB4BE1C3
:103AF0003B681A6AD7F8AC30D21A3B681A627A6807
:103B00003B681B789B0013441B889BB203F0400367
:103B1000002B00F09A807B683B673B685B78002B4A
:103B20006BD17B68BB667B68B3F850309BB21A469A
:103B3000BB6E1344BB663B681B78DA00BB6E134454
:103B400003F206437B667B6E1B889BB2C3F30903BB
:103B50009AB27B6E1A80D7F8AC30002B0AD17B6EFC
:103B60001B889BB26FEA43436FEA53439AB27B6E62
:103B70001A805BE0D7F8AC303E2B1CD8D7F8AC30BD
:103B80005B08C7F89830D7F8AC3003F00103002B7E
:103B900004D0D7F898300133C7F898307B6E1B8873
:103BA0009AB2D7F898309BB29B029BB213439AB259
:103BB0007B6E1A803AE0D7F8AC305B09C7F89830D2
:103BC000D7F8AC3003F01F03002B04D1D7F898309E
:103BD000013BC7F898307B6E1B889AB2D7F89830B3
:103BE0009BB29B029BB213439BB26FEA43436FEAC3
:103BF00053439AB27B6E1A8018E03B685B78012BC6
:103C000014D17B68B3F850309BB21A463B6F134413
:103C10003B673B681B78DA003B6F134403F20643B3
:103C2000FB66D7F8AC309AB2FB6E1A803B685B89B2
:103C3000A7F876303B685969D7F8AC309BB2B7F833
:103C40007620786800F001FB9EE03B685B78002BF3
:103C50006BD17B68FB677B68B3F850309BB21A4628
:103C6000FB6F1344FB673B681B78DA00FB6F134460
:103C700003F20243BB67BB6F1B889BB2C3F309030C
:103C80009AB2BB6F1A80D7F8AC30002B0AD1BB6F49
:103C90001B889BB26FEA43436FEA53439AB2BB6FF0
:103CA0001A8063E0D7F8AC303E2B1CD8D7F8AC3084
:103CB0005B08C7F89430D7F8AC3003F00103002B51
:103CC00004D0D7F894300133C7F89430BB6F1B8809
:103CD0009AB2D7F894309BB29B029BB213439AB22C
:103CE000BB6F1A8042E0D7F8AC305B09C7F894305C
:103CF000D7F8AC3003F01F03002B04D1D7F8943071
:103D0000013BC7F89430BB6F1B889AB2D7F8943048
:103D10009BB29B029BB213439BB26FEA43436FEA91
:103D200053439AB2BB6F1A8020E03B685B78012B4B
:103D30001CD17B68C7F884307B68B3F850309BB2E5
:103D40001A46D7F884301344C7F884303B681B7890
:103D5000DA00D7F88430134403F20243C7F8803006
:103D6000D7F8AC309AB2D7F880301A803B681B89FC
:103D7000A7F876303B685969D7F8AC309BB2B7F8F2
:103D80007620786800F061FA7A683B681B789B00BF
:103D900013441B889BB223F4E04323F040037B8150
:103DA0007B8983F010037B817B8983F020037B81F7
:103DB0007A683B681B789B001A447B8943F07F43F9
:103DC00043F47F0343F4004343F080039BB213802A
:103DD000D5E03B681B7B002B56D13B689B69002BD1
:103DE00022D13B68DB78002B1ED17A683B681B78B8
:103DF0009B0013441B889BB223F4E04323F0700321
:103E0000A7F88E307A683B681B789B001A44B7F895
:103E10008E3043F07F4343F47F0343F4014343F088
:103E200080039BB213801DE07A683B681B789B007F
:103E300013441B889BB223F4E24323F07003A7F8DA
:103E40008C307A683B681B789B001A44B7F88C303A
:103E500043F07F4343F47F0343F4004343F0800384
:103E60009BB213803B689A693B681B699A4207D9E9
:103E70003B689A693B681B69D21A3B689A6154E0B7
:103E80003B6800229A6150E03B68DB78022B42D10C
:103E90003B68DB69002B48D07A683B681B789B0045
:103EA00013441B88A7F89230B7F8923003F480438C
:103EB000002B05D0B7F8923003F04003002B0BD154
:103EC000B7F8923003F48043002B2ED1B7F892302C
:103ED00003F04003002B28D17A683B681B789B00D5
:103EE00013441B889BB223F4E04323F07003A7F82C
:103EF00090307A683B681B789B001A44B7F8903082
:103F000043F07F4343F47F0343F4004343F0C00393
:103F10009BB2138009E03B68DB78012B03D13B683F
:103F200000229A6101E001232AE07A683B681B784D
:103F30009B0013441B889BB223F4804323F070033F
:103F4000A7F88A30B7F88A3083F48053A7F88A300C
:103F5000B7F88A3083F40053A7F88A307A683B6850
:103F60001B789B001A44B7F88A3043F07F4343F430
:103F70007F0343F4004343F080039BB2138000238C
:103F80001846B037BD4680BD80B485B000AF7860BC
:103F900039603B685B78002B20D07A683B681B78DF
:103FA0009B0013441B889BB223F4E04323F040039F
:103FB000BB81BB8983F01003BB817A683B681B78A7
:103FC0009B001A44BB8943F07F4343F47F0343F4CF
:103FD000004343F080039BB213801FE07A683B6884
:103FE0001B789B0013441B889BB223F4804323F06F
:103FF0007003FB81FB8983F48053FB817A683B6803
:104000001B789B001A44FB8943F07F4343F47F03F2
:1040100043F4004343F080039BB21380002318460F
:104020001437BD465DF8047B704780B487B000AF9D
:10403000786039603B685B78002B4CD07A683B68CD
:104040001B789B0013441B883B823B8A03F0400390
:10405000002B1BD07A683B681B789B0013441B889D
:104060009BB223F4E04323F07003FB817A683B6842
:104070001B789B001A44FB8943F07F4343F47F0382
:1040800043F4004343F0C0039BB213803B68DB78EA
:10409000012B6CD07A683B681B789B0013441B880B
:1040A0009BB223F4E04323F04003BB81BB8983F040
:1040B0002003BB817A683B681B789B001A44BB894C
:1040C00043F07F4343F47F0343F4004343F0800312
:1040D0009BB213804BE07A683B681B789B001344CB
:1040E0001B88FB82FB8A03F48043002B1BD07A6879
:1040F0003B681B789B0013441B889BB223F4E0436E
:1041000023F07003BB827A683B681B789B001A44DB
:10411000BB8A43F07F4343F47F0343F4404343F0BF
:1041200080039BB213807A683B681B789B00134422
:104130001B889BB223F4804323F070037B827B8A2D
:1041400083F480537B827B8A83F400537B827A687A
:104150003B681B789B001A447B8A43F07F4343F4FF
:104160007F0343F4004343F080039BB2138000239A
:1041700018461C37BD465DF8047B704780B483B099
:1041800000AF78607B680122A3F840207B680022A2
:10419000A3F844207B680322A3F84020002318469C
:1041A0000C37BD465DF8047B704780B483B000AF28
:1041B00078600B46FB70FB78002B03D17B68802274
:1041C000A3F84C20002318460C37BD465DF8047B4D
:1041D000704780B483B000AF78607B68B3F8583024
:1041E0009BB26FEA43436FEA53439AB27B68A3F8EA
:1041F0005820002318460C37BD465DF8047B7047F5
:1042000080B483B000AF78607B68B3F858309BB25D
:10421000C3F30E039AB27B68A3F858200023184614
:104220000C37BD465DF8047B704780B485B000AFA5
:1042300078607B68B3F844309BB2FB60FB6818463B
:104240001437BD465DF8047B704780B48BB000AF77
:10425000F860B96011461A460B46FB801346BB80D6
:10426000BB8801335B08BB61FB687B61BB68FB619A
:10427000FA887B69134403F580633B62BB697B6208
:104280001CE0FB691B787B82FB6901331B781BB246
:104290001B021AB2B7F9123013431BB27B823B6A7E
:1042A0007A8A1A803B6A02333B62FB690133FB6105
:1042B000FB690133FB617B6A013B7B627B6A002BFC
:1042C000DFD100BF00BF2C37BD465DF8047B7047CF
:1042D00080B48BB000AFF860B96011461A460B4647
:1042E000FB801346BB80BB885B089BB2BB61FB684D
:1042F0007B61BB68FB61FA887B69134403F58063CB
:104300003B62BB697B6218E03B6A1B889BB23B61E6
:104310003B6A02333B623B69DAB2FB691A70FB69A4
:104320000133FB613B691B0ADAB2FB691A70FB6956
:104330000133FB617B6A013B7B627B6A002BE3D12B
:10434000BB8803F001039BB2002B07D03B6A1B889C
:104350009BB23B613B69DAB2FB691A7000BF2C3734
:10436000BD465DF8047B704780B582B000AF002386
:10437000FB71032002F03AF80F2000F00DF803461D
:10438000002B02D00123FB7101E007F05DFDFB79FA
:1043900018460837BD4680BD80B584B000AF786050
:1043A0000023FB73164B1B68002B22D0154B1A6899
:1043B000134B1B684FF47A71B1FBF3F3B2FBF3F3C9
:1043C000184602F054F80346002B0FD17B680F2BE0
:1043D00009D8002279684FF0FF3002F012F80A4A3B
:1043E0007B68136007E00123FB7304E00123FB7388
:1043F00001E00123FB73FB7B18461037BD4680BDEF
:1044000008000020000000200400002080B400AF5D
:10441000054B1A68054B1B681344034A136000BF21
:10442000BD465DF8047B7047740200200800002040
:1044300080B400AF034B1B681846BD465DF8047B93
:10444000704700BF7402002080B584B000AF786070
:10445000FFF7EEFFB8607B68FB60FB68B3F1FF3FDE
:1044600004D0094B1B68FA681344FB6000BFFFF7D8
:10447000DFFF0246BB68D31AFA689A42F7D800BF3A
:1044800000BF1037BD4680BD0800002080B400AFDB
:10449000034B1B681846BD465DF8047B704700BFA0
:1044A0009075FF1F80B400AF034B1B681846BD46D4
:1044B0005DF8047B704700BF9475FF1F80B400AFA8
:1044C000034B1B681846BD465DF8047B704700BF70
:1044D0009875FF1F80B588B000AF78607B68002BAF
:1044E00001D10123FEE27B681B6803F00103002B6E
:1044F00075D0974B9B6803F00C03BB61944BDB6852
:1045000003F003037B61BB690C2B02D17B69032B96
:1045100002D0BB69082B0BD18D4B1B6803F4003311
:10452000002B5BD07B685B68002B57D10123D9E25D
:104530007B685B68B3F5803F06D1854B1B68844A76
:1045400043F4803313601DE07B685B68B3F5A02FF4
:104550000CD17F4B1B687E4A43F4802313607C4B55
:104560001B687B4A43F4803313600BE0784B1B6875
:10457000774A23F480331360754B1B68744A23F425
:10458000802313607B685B68002B13D0FFF750FF1C
:10459000386108E0FFF74CFF02463B69D31A642BF1
:1045A00001D903239EE26A4B1B6803F40033002BFE
:1045B000F0D014E0FFF73CFF386108E0FFF738FF68
:1045C00002463B69D31A642B01D903238AE2604B6C
:1045D0001B6803F40033002BF0D100E000BF7B68C0
:1045E0001B6803F00203002B75D0594B9B6803F046
:1045F0000C03BB61564BDB6803F003037B61BB69B3
:104600000C2B02D17B69022B02D0BB69042B1FD17A
:104610004F4B1B6803F48063002B05D07B68DB687D
:10462000002B01D101235DE2494B5B6823F0FE4280
:104630007B681B691B06464913434B60454B1B684F
:104640001846FFF7A9FE0346002B43D0012349E299
:104650007B68DB68002B23D03D4B1B683C4A43F44E
:1046600080731360FFF7E4FE386108E0FFF7E0FEB7
:1046700002463B69D31A022B01D9032332E2344BA1
:104680001B6803F48063002BF0D0314B5B6823F090
:10469000FE427B681B691B062D4913434B601AE0E1
:1046A0002B4B1B682A4A23F480731360FFF7C0FE6C
:1046B000386108E0FFF7BCFE02463B69D31A022BC3
:1046C00001D903230EE2224B1B6803F48063002B05
:1046D000F0D100E000BF7B681B6803F00803002BEB
:1046E00041D07B685B69002B1CD0194BD3F8943008
:1046F000174A43F00103C2F89430FFF799FE38617E
:1047000008E0FFF795FE02463B69D31A022B01D958
:104710000323E7E10E4BD3F8943003F00203002BA0
:10472000EFD020E00A4BD3F89430094A23F001037C
:10473000C2F89430FFF77CFE38610DE0FFF778FE99
:1047400002463B69D31A022B06D90323CAE100BFF4
:1047500000100240040000208C4BD3F8943003F08A
:104760000203002BEAD17B681B6803F00403002BD3
:1047700000F0A6800023FB77844B9B6D03F08053F1
:10478000002B01D1012300E00023002B0DD07F4B33
:104790009B6D7E4A43F0805393657C4B9B6D03F089
:1047A0008053FB60FB680123FB77794B1B6803F4A4
:1047B0008073002B18D1764B1B68754A43F48073C5
:1047C0001360FFF735FE386108E0FFF731FE02465F
:1047D0003B69D31A022B01D9032383E16C4B1B687D
:1047E00003F48073002BF0D07B689B68012B08D109
:1047F000664BD3F89030654A43F00103C2F890301D
:1048000024E07B689B68052B10D1604BD3F8903077
:104810005E4A43F00403C2F890305C4BD3F890300A
:104820005A4A43F00103C2F890300FE0574BD3F8D7
:104830009030564A23F00103C2F89030534BD3F81E
:104840009030524A23F00403C2F890307B689B6892
:10485000002B16D0FFF7ECFD38610AE0FFF7E8FD0A
:1048600002463B69D31A41F28832934201D90323AD
:1048700038E1464BD3F8903003F00203002BEDD023
:1048800015E0FFF7D5FD38610AE0FFF7D1FD0246DC
:104890003B69D31A41F28832934201D9032321E1C3
:1048A0003A4BD3F8903003F00203002BEDD1FB7F9D
:1048B000012B05D1354B9B6D344A23F08053936512
:1048C0007B681B6803F02003002B3CD07B689B694E
:1048D000002B1CD02D4BD3F898302C4A43F0010309
:1048E000C2F89830FFF7A4FD386108E0FFF7A0FD9B
:1048F00002463B69D31A022B01D90323F2E0234B72
:10490000D3F8983003F00203002BEFD01BE01F4BCD
:10491000D3F898301D4A23F00103C2F89830FFF70E
:1049200087FD386108E0FFF783FD02463B69D31A33
:10493000022B01D90323D5E0144BD3F8983003F0B0
:104940000203002BEFD17B68DB69002B00F0C980EC
:104950000E4B9B6803F00C030C2B00F083807B68EC
:10496000DB69022B5ED1094B1B68084A23F0807378
:104970001360FFF75DFD38610CE0FFF759FD02465B
:104980003B69D31A022B05D90323ABE00010024088
:1049900000700040554B1B6803F00073002BECD1F6
:1049A000524BDA68524B13407A68116A7A68526A3D
:1049B000013A120111437A68926A120211437A682D
:1049C000126B5208013A520511437A68526B520831
:1049D000013A520611437A68D26AD2060A43434921
:1049E0001343CB60414B1B68404A43F08073136014
:1049F0003E4BDB683D4A43F08073D360FFF718FD00
:104A0000386108E0FFF714FD02463B69D31A022B18
:104A100001D9032366E0354B1B6803F00073002BBC
:104A2000F0D05EE0314B1B68304A23F08073136096
:104A3000FFF7FEFC386108E0FFF7FAFC02463B692D
:104A4000D31A022B01D903234CE0284B1B6803F037
:104A50000073002BF0D1254BDA682449254B134015
:104A6000CB603EE07B68DB69012B01D1012339E09B
:104A70001E4BDB687B617B6903F003027B681B6A6A
:104A80009A422CD17B6903F0F0027B685B6A013BA0
:104A90001B019A4223D17B6903F4FE427B689B6A27
:104AA0001B029A421BD17B6903F078427B68DB6A68
:104AB000DB069A4213D17B6903F4C0027B681B6B4F
:104AC0005B08013B5B059A4209D17B6903F0C06238
:104AD0007B685B6B5B08013B5B069A4201D001235C
:104AE00000E0002318462037BD4680BD001002407C
:104AF0000C809F01FCFFEEFE80B586B000AF7860B1
:104B0000396000237B617B68002B01D101231EE10A
:104B1000914B1B6803F00F033A689A4210D98E4BF1
:104B20001B6823F00F028C493B6813430B608A4BD0
:104B30001B6803F00F033A689A4201D0012306E193
:104B40007B681B6803F00103002B73D07B685B68F4
:104B5000032B29D1814B1B6803F00073002B01D17B
:104B60000123F4E000F066F938613B697C4A934226
:104B70003FD97A4B9B6803F0F003002B09D07B6888
:104B80001B6803F00203002B33D07B689B68002B6B
:104B90002FD1724B9B6823F0F003704A43F08003DF
:104BA000936080237B6124E07B685B68022B07D1E4
:104BB0006A4B1B6803F40033002B09D10123C6E0C4
:104BC000664B1B6803F48063002B01D10123BEE018
:104BD00000F0CEF838613B69614A934209D95F4BD6
:104BE0009B6823F0F0035D4A43F0800393608023C9
:104BF0007B615A4B9B6823F003027B685B685749D3
:104C000013438B60FFF714FCF8600AE0FFF710FC19
:104C10000246FB68D31A41F28832934201D903233A
:104C200095E04E4B9B6803F00C027B685B689B0031
:104C30009A42EBD17B681B6803F00203002B23D060
:104C40007B681B6803F00403002B05D0434B9B6873
:104C5000424A43F4E06393607B681B6803F00803F7
:104C6000002B07D03D4B9B6823F47C533B4A43F415
:104C7000E0639360394B9B6823F0F0027B689B688C
:104C8000364913438B6008E07B69802B05D1334B99
:104C90009B68324A23F0F00393602F4B1B6803F0AC
:104CA0000F033A689A421DD22B4B1B6823F00F0268
:104CB00029493B6813430B60FFF7BAFBF8600AE031
:104CC000FFF7B6FB0246FB68D31A41F288329342E3
:104CD00001D903233BE0204B1B6803F00F033A6824
:104CE0009A42EDD17B681B6803F00403002B08D0C7
:104CF0001A4B9B6823F4E0627B68DB681749134317
:104D00008B607B681B6803F00803002B09D0134BF2
:104D10009B6823F460527B681B69DB000F491343D7
:104D20008B6000F025F802460C4B9B681B0903F0D2
:104D30000F030C49CB5C03F01F0322FA03F30A4A6A
:104D400013600A4B1B681846FFF726FB03461846FC
:104D50001837BD4680BD00BF002002400010024051
:104D600000B4C404A448010800000020040000208E
:104D700080B487B000AF2C4B9B6803F00C03042B6E
:104D800002D12A4B3B6147E0274B9B6803F00C03A1
:104D9000082B02D1264B3B613EE0234B9B6803F07E
:104DA0000C030C2B36D1204BDB6803F00303FB60B4
:104DB0001D4BDB681B0903F00F030133BB60FB686D
:104DC000032B0CD11A4ABB68B2FBF3F3164AD26824
:104DD000120A02F07F0202FB03F37B610CE0134A2C
:104DE000BB68B2FBF3F3104AD268120A02F07F02EA
:104DF00002FB03F37B6100BF0B4BDB685B0E03F030
:104E0000030301335B007B607A697B68B2FBF3F3D9
:104E10003B6101E000233B613B6918461C37BD46FE
:104E20005DF8047B704700BF001002400024F400CE
:104E300000366E0180B487B000AF1E4BDB6803F014
:104E400003033B611B4BDB681B0903F00F030133BA
:104E5000FB603B69032B0CD1174AFB68B2FBF3F3F1
:104E6000144AD268120A02F07F0202FB03F37B614C
:104E70000CE0124AFB68B2FBF3F30E4AD268120A46
:104E800002F07F0202FB03F37B6100BF094BDB688A
:104E90005B0E03F0030301335B00BB607A69BB6800
:104EA000B2FBF3F37B607B6818461C37BD465DF8A8
:104EB000047B70470010024000366E010024F400AD
:104EC00080B586B000AF78600023FB740023BB740C
:104ED0007B681B6803F40023002B00F098800023FC
:104EE0007B74434B9B6D03F08053002B0DD1404BE3
:104EF0009B6D3F4A43F0805393653D4B9B6D03F0A0
:104F00008053BB60BB6801237B743A4B1B68394AF2
:104F100043F480731360FFF78BFAF86009E0FFF742
:104F200087FA0246FB68D31A022B02D90323FB74CB
:104F300005E0304B1B6803F48073002BEFD0FB7C43
:104F4000002B59D12A4BD3F8903003F440737B6186
:104F50007B69002B1ED07B681B6D7A699A4219D041
:104F6000234BD3F8903023F440737B61204BD3F86C
:104F700090301F4A43F48033C2F890301C4BD3F872
:104F800090301B4A23F48033C2F89030184A7B6972
:104F9000C2F890307B6903F00103002B16D0FFF7B5
:104FA00047FAF8600BE0FFF743FA0246FB68D31AB2
:104FB00041F28832934202D90323FB7406E00C4B82
:104FC000D3F8903003F00203002BECD0FB7C002BD5
:104FD0000BD1074BD3F8903023F440727B681B6DE4
:104FE00003491343C1F8903008E0FB7CBB7405E033
:104FF0000010024000700040FB7CBB747B7C012BE6
:1050000005D1A74B9B6DA64A23F0805393657B681F
:105010001B6803F00103002B0AD0A14BD3F88830A2
:1050200023F003027B685B689D491343C1F8883015
:105030007B681B6803F00203002B0AD0984BD3F85F
:10504000883023F00C027B689B6895491343C1F8B4
:1050500088307B681B6803F00403002B0AD0904B58
:10506000D3F8883023F030027B68DB688C49134327
:10507000C1F888307B681B6803F00803002B0AD056
:10508000874BD3F8883023F0C0027B681B698449C2
:105090001343C1F888307B681B6803F01003002BB2
:1050A0000AD07F4BD3F8883023F440727B685B6969
:1050B0007B491343C1F888307B681B6803F02003E9
:1050C000002B0AD0764BD3F8883023F440627B68FB
:1050D0009B6973491343C1F888307B681B6803F0F0
:1050E0004003002B0AD06E4BD3F8883023F4405293
:1050F0007B68DB696A491343C1F888307B681B68A9
:1051000003F08003002B0AD0654BD3F8883023F4DA
:1051100040427B681B6A62491343C1F888307B6850
:105120001B6803F48073002B0AD05D4BD3F88830E2
:1051300023F440327B685B6A59491343C1F88830D5
:105140007B681B6803F40033002B0AD0544BD3F860
:105150009C3023F003027B689B6A51491343C1F8DA
:105160009C307B681B6803F40073002B0AD04C4B07
:10517000D3F8883023F440227B68DB6A4849134324
:10518000C1F888307B681B6803F48063002B15D05E
:10519000434BD3F8883023F440127B681B6B4049A3
:1051A0001343C1F888307B681B6BB3F5801F05D1B2
:1051B0003B4BDB683A4A43F48013D3607B681B683F
:1051C00003F40063002B15D0354BD3F8883023F45B
:1051D00040027B685B6B32491343C1F888307B68BF
:1051E0005B6BB3F5800F05D12D4BDB682C4A43F484
:1051F0008013D3607B681B6803F48053002B15D0A9
:10520000274BD3F8883023F040727B689B6B24498E
:105210001343C1F888307B689B6BB3F1807F05D165
:105220001F4BDB681E4A43F48013D3607B681B6806
:1052300003F40053002B15D0194BD3F8883023F01A
:1052400040627B68DB6B16491343C1F888307B688A
:10525000DB6BB3F1006F05D1114BDB68104A43F4EF
:105260008013D3607B681B6803F48043002B19D044
:105270000B4BD3F8883023F040627B681B6C0849E5
:105280001343C1F888307B681B6CB3F1006F09D100
:10529000034BDB68024A43F48013D36002E000BF93
:1052A000001002407B681B6803F40043002B15D0FC
:1052B000294BD3F8883023F040527B685B6C264939
:1052C0001343C1F888307B685B6CB3F1805F05D114
:1052D000214BDB68204A43F48033D3607B681B6832
:1052E00003F48033002B15D01B4BD3F8883023F008
:1052F00040427B689B6C18491343C1F888307B6837
:105300009B6CB3F1804F05D1134BDB68124A43F419
:105310008033D3607B681B6803F48023002B15D097
:105320000D4BD3F89C3023F440127B68DB6C0A49A8
:105330001343C1F89C307B68DB6CB3F5001F05D1CB
:10534000054BDB68044A43F48013D360BB7C1846EA
:105350001837BD4680BD00BF0010024080B586B042
:1053600000AFF860B960C7E9002300233B612F4B11
:105370001B78012B01D1022353E02C4B01221A7020
:105380004FF47A7000F0E6F80346FB75FB7D002BC6
:1053900043D1264B00225A60254B1B6803F48063DF
:1053A000002B09D0224B1B68214A23F48063136031
:1053B0001E4B02221A7702E01C4B00221A77FB6870
:1053C000002B07D1D7E90023B86800F015F90123B5
:1053D0003B6110E0FB68012B02D0FB68022B0AD175
:1053E0003B681946B86800F02DF9FB68022B02D122
:1053F0004FF480233B614FF47A7000F0ABF8034622
:10540000FB753B69002B06D0094B5A693B69DB43AE
:10541000074913404B6100F0D3FA044B00221A7085
:10542000FB7D18461837BD4680BD00BF0C0000202C
:105430000020024080B483B000AF0023FB710B4B0F
:105440005B69002B0BDA094B094A9A60074B094A42
:105450009A60064B5B69002B01DA0123FB71FB7933
:1054600018460C37BD465DF8047B704700200240AB
:1054700023016745AB89EFCD80B483B000AF012332
:10548000FB71094B5B69084A43F000435361064BCB
:105490005B69002B01DA0023FB71FB7918460C379E
:1054A000BD465DF8047B70470020024080B483B0A5
:1054B00000AF0023FB710D4B5B6903F08043002BB1
:1054C0000DD00A4B0A4ADA60084B0A4ADA60074BE9
:1054D0005B6903F08043002B01D00123FB71FB7952
:1054E00018460C37BD465DF8047B7047002002402B
:1054F0003B2A19087F6E5D4C80B483B000AF012356
:10550000FB710A4B5B69094A43F080435361074BC7
:105510005B6903F08043002B01D00023FB71FB7912
:1055200018460C37BD465DF8047B704700200240EA
:1055300080B500AF064B5B69054A43F000635361D9
:105540004FF47A7000F006F80346184680BD00BF9D
:105550000020024080B584B000AF7860FEF768FF9D
:10556000F86009E0FEF764FF0246FB68D31A7A6828
:105570009A4201D2032337E01D4B1B6903F48033A9
:10558000B3F5803FEED01A4B1A694CF2FA33134050
:10559000BB60BB68002B1DD0164B5A68BB68134319
:1055A000144A5360BB68B3F1805F07D3104B9A690C
:1055B000BB6803F070430E4913438B61BB6823F053
:1055C0007043002B04D00A4ABB6823F07043136178
:1055D000012309E0064B1B6903F00103012B02D1F3
:1055E000034B01221A61002318461037BD4680BDC7
:1055F000002002400C00002080B485B000AFF860AD
:10560000C7E900230E4B5B690D4A43F00103536168
:10561000FB683A681A60BFF36F8F00BFD7E90001DB
:105620004FF000024FF000030A000023F968043134
:1056300013460B6000BF1437BD465DF8047B70470E
:105640000020024080B489B000AF78603960402308
:10565000FB777B68BB613B687B61144B5B69134ADA
:1056600043F480235361EFF31083FB60FB683B61DD
:1056700072B600BF7B691A68BB691A60BB690433E4
:10568000BB617B6904337B61FB7F013BFB77FB7F65
:10569000002BEFD13B69BB60BB6883F3108800BF70
:1056A00000BF2437BD465DF8047B704700200240F0
:1056B00080B584B000AF78603960494B1B78012B0E
:1056C00001D1022387E0464B01221A704FF47A7011
:1056D000FFF740FF0346FB73FB7B002B77D1404B6A
:1056E00000225A603F4B1B6803F40073002B13D059
:1056F0003C4B1B6803F48063002B09D0394B1B68BB
:10570000384A23F480631360354B03221A7716E07E
:10571000334B01221A7712E0324B1B6803F480638B
:10572000002B09D02F4B1B682E4A23F48063136093
:105730002B4B02221A7702E0294B00221A777B6852
:105740001B68012B13D17B685B68184600F0BCF81E
:105750004FF47A70FFF7FEFE0346FB73214B5B6943
:10576000204A23F4004323F0040353612DE03B68F7
:105770004FF0FF321A607B689B68BB601DE07B685E
:105780005B681946B86800F0D7F84FF47A70FFF7F5
:10579000E1FE0346FB73134B5B69124A23F47E73ED
:1057A00023F002035361FB7B002B03D03B68BA68F4
:1057B0001A600AE0BB680133BB607B689A687B684B
:1057C000DB681344BA689A42D9D300F0F9F8044B65
:1057D00000221A70FB7B18461037BD4680BD00BF03
:1057E0000C0000200020024080B582B000AF78603D
:1057F0007B6806221A607B685B68002B0BD07B6895
:105800005B68012B07D07B685B68022B03D07B6849
:105810005B68042B0FD17B681B6843F001027B6837
:105820001A607B6858687B6803F108017B680C3359
:105830001A4600F03BF900F08BF902467B681A61CA
:1058400000F09EF902467B689A617B68DB69012B58
:1058500003D07B68DB69022B10D17B681B6843F0A7
:1058600008027B681A607B6803F11C007B6803F107
:1058700020017B6824331A4600F096F97B681B6888
:1058800043F010027B681A6000F002F902467B6860
:105890009A627B68DB6A012B03D07B68DB6A022B90
:1058A0000DD17B681B6843F020027B681A607B681F
:1058B000DA6A7B6830331946104600F0CBF800BF37
:1058C0000837BD4680BD000080B483B000AF78606B
:1058D000184B1B6A03F48003002B16D07B6803F07F
:1058E0000103002B05D0134B5B69124A43F00403FC
:1058F00053617B6803F00203002B0ED00D4B5B69F4
:105900000C4A43F40043536107E00A4B5B69094AC0
:1059100043F4004343F004035361064B5B69054ABB
:1059200043F48033536100BF0C37BD465DF8047B00
:10593000704700BF0020024080B483B000AF7860A1
:1059400039601E4B1B6A03F48003002B06D11B4BEE
:105950005B691A4A23F40063536111E03B6803F06A
:105960000103002B06D0154B5B69144A23F4006336
:10597000536105E0114B5B69104A43F400635361C6
:105980000E4B5B6923F47E727B68DB0003F4FF63DC
:105990000A4913434B61094B5B69084A43F0020310
:1059A0005361064B5B69054A43F48033536100BF82
:1059B0000C37BD465DF8047B704700BF00200240F5
:1059C00080B483B000AF214B1B7FFB71FB79012BAF
:1059D00002D0FB79032B17D11D4B1B681C4A23F403
:1059E000007313601A4B1B68194A43F40063136079
:1059F000174B1B68164A23F400631360144B1B6893
:105A0000134A43F400731360FB79022B02D0FB7935
:105A1000032B11D10E4B1B680D4A43F480531360C6
:105A20000B4B1B680A4A23F480531360084B1B6816
:105A3000074A43F480631360044B00221A7700BFC7
:105A40000C37BD465DF8047B704700BF0C0000209A
:105A50000020024080B483B000AF786039607B687A
:105A6000012B05D1094B1B6FDAB23B681A6007E0C6
:105A70007B68022B04D1054B5B6FDAB23B681A607E
:105A800000BF0C37BD465DF8047B70470020024024
:105A900080B400AF044B1B6F03F480331846BD463F
:105AA0005DF8047B704700BF0020024080B485B0E1
:105AB00000AFF860B9607A60FB68002B0DD1234B12
:105AC000DB6A03F07F02BB681A60204BDB6A1B0CA9
:105AD00003F07F027B681A6031E0FB68012B0DD177
:105AE0001A4B1B6B03F07F02BB681A60174B1B6BD2
:105AF0001B0C03F07F027B681A6020E0FB68022B1E
:105B00000DD1124BDB6C03F07F02BB681A600F4BA8
:105B1000DB6C1B0C03F07F027B681A600FE0FB68F4
:105B2000042B0CD1094B1B6D03F07F02BB681A607C
:105B3000064B1B6D1B0C03F07F027B681A6000BFD5
:105B40001437BD465DF8047B704700BF002002405B
:105B500080B483B000AF094B1B6ADBB27B607B680B
:105B6000AA2B04D07B68CC2B01D0BB2300E07B6840
:105B700018460C37BD465DF8047B70470020024094
:105B800080B483B000AF074B1B6A7B607B6823F057
:105B9000FF037B607B6818460C37BD465DF8047BCD
:105BA000704700BF0020024080B489B000AFF860A9
:105BB000B9607A605B4B1B6803F48073002B14D1CF
:105BC0004FF00063FB61584B1B884FF6FF72934206
:105BD00008D0554B1B689B025A08544B134003F1E5
:105BE000006300E0524BBB6113E04F4B1B884FF644
:105BF000FF72934208D04C4B1B689B025A084B4BD8
:105C0000134003F1006300E0494BFB614FF0006378
:105C1000BB61484B1B6A03F48003002B39D1FB683E
:105C20001B6803F00303012B16D1424B5B6AC3F3DD
:105C30000E037B617B691B0103F10062BB681A6084
:105C40003C4B9B6AC3F30E037B617B691B0103F131
:105C500000627B681A6055E0FB681B6803F0030371
:105C6000022B4FD1334B5B6CC3F30E037B617B691B
:105C70001B0103F10062BB681A602E4B9B6CC3F3DF
:105C80000E037B617B691B0103F100627B681A6074
:105C900038E0FB681B6803F00303012B16D1254B8A
:105CA0005B6AC3F30E037B617B69DA00FB691A440C
:105CB000BB681A601F4B9B6AC3F30E037B617B6951
:105CC000DA00FB691A447B681A601BE0FB681B68FA
:105CD00003F00303022B15D1164B5B6CC3F30E03C9
:105CE0007B617B69DA00BB691A44BB681A60114B9F
:105CF0009B6CC3F30E037B617B69DA00BB691A44BA
:105D00007B681A600B4B9B6A03F00042FB681B68C0
:105D10001A43FB681A6000BF2437BD465DF8047B58
:105D2000704700BF00000140E075FF1F00FEFF014B
:105D3000000004080020024080B487B000AF786003
:105D4000396000237B615AE13B681A6801217B6955
:105D500001FA03F31340FB60FB68002B00F04C8159
:105D60003B685B6803F00303012B05D03B685B686D
:105D700003F00303022B30D17B689B683B617B6996
:105D80005B00032202FA03F3DB433A6913403B61F1
:105D90003B68DA687B695B0002FA03F33A691343F4
:105DA0003B617B683A699A607B685B683B61012272
:105DB0007B6902FA03F3DB433A6913403B613B68BA
:105DC0005B681B0903F001027B6902FA03F33A697D
:105DD00013433B617B683A695A603B685B6803F038
:105DE0000303032B17D07B68DB683B617B695B0097
:105DF000032202FA03F3DB433A6913403B613B6839
:105E00009A687B695B0002FA03F33A6913433B61CA
:105E10007B683A69DA603B685B6803F00303022B36
:105E200023D17B69DA087B68083253F822303B6162
:105E30007B6903F007039B000F2202FA03F3DB43A5
:105E40003A6913403B613B681A697B6903F00703B9
:105E50009B0002FA03F33A6913433B617B69DA085A
:105E60007B680832396943F822107B681B683B6104
:105E70007B695B00032202FA03F3DB433A691340B8
:105E80003B613B685B6803F003027B695B0002FADD
:105E900003F33A6913433B617B683A691A603B68D4
:105EA0005B6803F44033002B00F0A6805B4B1B6E55
:105EB0005A4A43F001031366584B1B6E03F001036B
:105EC000BB60BB68564A7B699B08023352F823309B
:105ED0003B617B6903F003039B000F2202FA03F38B
:105EE000DB433A6913403B617B68B3F1904F1FD0AD
:105EF0007B684C4A934219D07B684B4A934213D03B
:105F00007B684A4A93420DD07B68494A934207D046
:105F10007B68484A934201D105230AE0062308E042
:105F2000042306E0032304E0022302E0012300E04F
:105F300000237A6902F00302920093403A69134306
:105F40003B6137497B699B0802333A6941F823205A
:105F5000394B9B683B61FB68DB433A6913403B610B
:105F60003B685B6803F48013002B03D03A69FB683D
:105F700013433B61304A3B6993602F4BDB683B61C5
:105F8000FB68DB433A6913403B613B685B6803F4A1
:105F90000013002B03D03A69FB6813433B61264A88
:105FA0003B69D360244B5B683B61FB68DB433A6928
:105FB00013403B613B685B6803F40033002B03D064
:105FC0003A69FB6813433B611B4A3B6953601A4BB8
:105FD0001B683B61FB68DB433A6913403B613B68EC
:105FE0005B6803F48033002B03D03A69FB681343EA
:105FF0003B61114A3B6913607B6901337B613B68FC
:106000001A687B6922FA03F3002B7FF49DAE00BF70
:1060100000BF1C37BD465DF8047B7047001002408E
:10602000000001400004004800080048000C00483F
:1060300000100048001400480004014080B483B000
:1060400000AF78600B467B8013467B707B78002B1B
:1060500003D07A887B689A6102E07A887B689A62CA
:1060600000BF0C37BD465DF8047B704780B582B039
:1060700000AF0346FB80084B5A69FB881340002B96
:1060800006D0054AFB885361FB88184606F0C0FD20
:1060900000BF0837BD4680BD0004014080B485B014
:1060A00000AF78607B68002B41D14B4B1B6803F439
:1060B000C063B3F5806F31D1474BD3F88030464A87
:1060C00023F48073C2F88030434B1B6823F4C06311
:1060D000414A43F400731360404B1B68322202FBB9
:1060E00003F33F4AA2FB03239B0C0133FB6002E056
:1060F000FB68013BFB60384B5B6903F48063B3F5DD
:10610000806F02D1FB68002BF2D1334B5B6903F443
:106110008063B3F5806F58D1032357E02E4BD3F83B
:1061200080302D4A23F48073C2F880304DE07B68C4
:10613000B3F5007F41D1284B1B6803F4C063B3F56E
:10614000806F31D1244BD3F88030234A43F48073DD
:10615000C2F88030204B1B6823F4C0631E4A43F40E
:10616000007313601D4B1B68322202FB03F31C4AB1
:10617000A2FB03239B0C0133FB6002E0FB68013BA5
:10618000FB60154B5B6903F48063B3F5806F02D14C
:10619000FB68002BF2D1104B5B6903F48063B3F50D
:1061A000806F12D1032311E00B4BD3F880300A4AE1
:1061B00043F48073C2F8803007E0074B1B6823F478
:1061C000C063054A43F48063136000231846143704
:1061D000BD465DF8047B7047007000400000002061
:1061E00083DE1B4380B400AF054B9B68044A43F435
:1061F0008043936000BFBD465DF8047B704700BFDD
:106200000070004080B485B000AF78607B6803F018
:106210000703FB600C4BDB68BB60BA684FF6FF03FB
:106220001340BB60FB681A02BB68134343F0BF63B3
:1062300043F40033BB60044ABB68D36000BF14372B
:10624000BD465DF8047B704700ED00E080B400AF10
:10625000044BDB681B0A03F007031846BD465DF8D4
:10626000047B704700ED00E080B483B000AF0346CC
:10627000FB7197F90730002B0BDBFB7903F01F0252
:10628000074997F907305B09012000FA02F241F84B
:10629000232000BF0C37BD465DF8047B704700BF6C
:1062A00000E100E080B483B000AF0346FB7197F9D2
:1062B0000730002B12DBFB7903F01F020A4997F924
:1062C00007305B09012000FA02F2203341F8232055
:1062D000BFF34F8F00BFBFF36F8F00BF00BF0C37FE
:1062E000BD465DF8047B704700E100E080B483B0F8
:1062F00000AF03463960FB7197F90730002B0ADBCA
:106300003B68DAB20C4997F907301201D2B20B445C
:1063100083F800230AE03B68DAB20849FB7903F00E
:106320000F03043B1201D2B20B441A7600BF0C37A4
:10633000BD465DF8047B704700E100E000ED00E041
:1063400080B489B000AFF860B9607A60FB6803F090
:106350000703FB61FB69C3F10703042B28BF042378
:10636000BB61FB690433062B02D9FB69033B00E0E8
:1063700000237B614FF0FF32BB6902FA03F3DA437B
:10638000BB681A407B699A404FF0FF317B6901FA84
:1063900003F3D9437B680B40134318462437BD46AB
:1063A0005DF8047B7047000080B582B000AF786074
:1063B0007B68013BB3F1807F01D301230FE00A4AE0
:1063C0007B68013B53600F214FF0FF30FFF78EFFDA
:1063D000054B00229A60044B07221A6000231846DE
:1063E0000837BD4680BD00BF10E000E080B582B038
:1063F00000AF78607868FFF705FF00BF0837BD463B
:1064000080BD80B586B000AF0346B9607A60FB738B
:10641000FFF71CFF78617A68B9687869FFF790FF29
:10642000024697F90F3011461846FFF75FFF00BF8D
:106430001837BD4680BD80B582B000AF0346FB7102
:1064400097F907301846FFF70FFF00BF0837BD4622
:1064500080BD80B582B000AF0346FB7197F907306D
:106460001846FFF71FFF00BF0837BD4680BD80B547
:1064700082B000AF78607868FFF796FF0346184651
:106480000837BD4680BD000080B584B000AF78609D
:106490007B68002B01D1012347E17B6893F85C30D6
:1064A000DBB2002B06D17B68002283F85D20786880
:1064B00005F0C4FA7B681B689A697B681B6822F048
:1064C00010029A61FDF7B4FFF86012E0FDF7B0FF2B
:1064D0000246FB68D31A0A2B0BD97B681B6E43F06C
:1064E00001027B681A667B68032283F85C20012323
:1064F0001BE17B681B689B6903F00803082BE5D050
:106500007B681B689A697B681B6842F001029A618C
:10651000FDF78EFFF86012E0FDF78AFF0246FB6888
:10652000D31A0A2B0BD97B681B6E43F001027B68E0
:106530001A667B68032283F85C200123F5E07B6800
:106540001B689B6903F00103002BE5D07B681B6887
:106550009A697B681B6842F002029A617B681B683B
:10656000744A934203D1744A7B685B6813607B680A
:106570001B7C012B08D17B681B689A697B681B68B0
:1065800022F040029A6107E07B681B689A697B6889
:106590001B6842F040029A617B685B7C012B08D14A
:1065A0007B681B689A697B681B6842F480429A6129
:1065B00007E07B681B689A697B681B6822F480424D
:1065C0009A617B689B7C012B08D17B681B689A6968
:1065D0007B681B6822F480529A6107E07B681B6825
:1065E0009A697B681B6842F480529A617B681B68D9
:1065F0009B6923F440717B689A687B681B680A4337
:106600009A617B681B689A697B681B6822F0A40208
:106610009A617B681B681A697B681B6822F010020C
:106620001A617B68DB68012B08D17B681B689A695B
:106630007B681B6842F004029A612CE07B68DB688F
:10664000002B28D07B68DB68022B1CD07B681B6882
:106650009A697B681B6842F080029A617B681B68BC
:106660001A697B681B6842F010021A617B68DB685C
:10667000032B10D17B681B689A697B681B6842F00A
:1066800020029A6107E07B681B689A697B681B6837
:1066900042F020029A617B689B69013B5A067B6845
:1066A000DB69013B1B021A437B681B6A013B42EA20
:1066B00003017B685B69013B1A047B681B680A4322
:1066C000DA617B689B68B3F5407F15D17B689B6A74
:1066D0005A1E7B68DB6A013B1B021A437B681B6BFB
:1066E000013B1B0142EA03017B685B6A013B1A0420
:1066F0007B681B680A43DA607B681B68D3F8C010AC
:106700007B68DA6B7B681B680A43C3F8C020786833
:1067100000F06CFC7B6800229A657B6800221A6698
:106720007B68012283F85C20002318461037BD46A1
:1067300080BD00BF006400400065004080B487B0A9
:1067400000AF786039607B6893F85C30FB75FB7D47
:10675000012B02D0FB7D022B3DD13B681B68002B37
:1067600019D13B689B689A073B68DB68DB061A43D4
:106770003B681B691B041A433B685B6913433B611D
:106780007B681A6C3B685B689B001344BB60BB680A
:106790003A691A601DE03B68DB685A073B681B6971
:1067A00013433B613B689B689A073B685B691343F3
:1067B000FB607B685A6C3B685B68DB001344BB6022
:1067C000BB683A691A60BB680433BB60BB68FA688F
:1067D0001A60002306E07B681B6E43F002027B68B0
:1067E0001A66012318461C37BD465DF8047B7047C6
:1067F00080B483B000AF78607B6893F85C30DBB224
:10680000012B10D17B68022283F85C207B681B6817
:106810009A697B681B6822F001029A617B680022FA
:106820001A66002306E07B681B6E43F004027B6857
:106830001A66012318460C37BD465DF8047B704785
:1068400080B586B000AFF860B9607A60FB6893F8F5
:106850005C30DBB2022B2CD1FB681B68D3F8C43050
:1068600003F40013002B07D0FB681B6E43F4007287
:10687000FB681A66012323E0FB681B68D3F8C43069
:106880001B0C03F003037B617B697A68B968F868C5
:1068900000F018FCFB681B6801217A6901FA02F21A
:1068A000C3F8CC2001227B699A40FB689A650023DB
:1068B00006E0FB681B6E43F00802FB681A660123C2
:1068C00018461837BD4680BD80B48BB000AFF86065
:1068D000B9607A603B600023FB61FB6893F85C3031
:1068E000FB76FB7E022B40F0E880BB68402B37D163
:1068F000FB681B68D3F8903003F00F03002B07D11F
:10690000FB681B6E43F48072FB681A660123DBE0B0
:10691000FB681B68D3F8903003F08073B3F1807F7D
:106920000AD1FB681B68D3F8803003F40073B3F519
:10693000007F01D10123FB61FB681B68D3F8903015
:106940001B0A03F00303FA691344FB61FB68996CAB
:10695000FA691346DB001344DB000B447B6236E02C
:10696000FB681B68D3F8983003F00F03002B07D1A6
:10697000FB681B6E43F48072FB681A660123A3E078
:10698000FB681B68D3F8983003F08073B3F1807F05
:106990000AD1FB681B68D3F8803003F48073B3F529
:1069A000807F01D10123FB61FB681B68D3F898301D
:1069B0001B0A03F00303FA691344FB61FB68D96CFB
:1069C000FA691346DB001344DB000B447B627B6AED
:1069D0001B6803F080427B685A607B685B68002B11
:1069E00007D17B6A1B689B0CC3F30A027B681A60A1
:1069F00005E07B6A1B6823F060427B681A607B6A53
:106A00001B6803F000527B689A607B6A1B6803F086
:106A100000427B681A617B6A04337B627B6A1B6875
:106A20009AB27B68DA617B6A1B681B0C03F00F0269
:106A30007B68DA607B6A1B6803F480127B685A61AA
:106A40007B6A1B6803F400127B689A617B6A1B688F
:106A50001B0E03F07F027B681A627B6A1B68DA0FE9
:106A60007B685A627B6A04337B627B6A7B610023AA
:106A70003B620AE07A693B6A1A4439683B6A0B4414
:106A800012781A703B6A01333B627B68DB68114AFB
:106A9000D35C1A463B6A9342ECD3BB68402B05D1CA
:106AA000FB681B68FA69C3F8942004E0FB681B6864
:106AB000FA69C3F89C20002306E0FB681B6E43F0D4
:106AC0000802FB681A66012318462C37BD465DF89C
:106AD000047B7047B448010880B485B000AF78608B
:106AE0007B681B68D3F8C43003F00703FB60FB68C6
:106AF00018461437BD465DF8047B704780B487B0F4
:106B000000AFF860B9607A60FB6893F85C30FB75A1
:106B1000FB7D012B03D0FB7D022B40F0C880FB687E
:106B20001B689B6D3B61BB6803F00703002B04D01F
:106B30003B6903F00103002B3BD0BB6803F0380333
:106B4000002B04D03B6903F00203002B31D0BB685B
:106B500003F4E073002B04D03B6903F00403002B23
:106B600027D0BB6803F4F053002B04D03B6903F03B
:106B70000803002B1DD0BB6803F46043002B04D036
:106B80003B6903F01003002B13D0BB6803F44033C0
:106B9000002B04D03B6903F02003002B09D0BB6815
:106BA00003F47C03002B0CD03B6903F04003002B63
:106BB00007D1FB681B68DA6DFB681B6842F00102B5
:106BC000DA65BB6803F00703002B04D03B6903F0D0
:106BD0000103002B3BD1BB6803F03803002B04D02A
:106BE0003B6903F00203002B31D1BB6803F4E0736F
:106BF000002B04D03B6903F00403002B27D1BB68B2
:106C000003F4F053002B04D03B6903F00803002B7E
:106C10001DD1BB6803F46043002B04D03B6903F033
:106C20001003002B13D1BB6803F44033002B04D0B6
:106C30003B6903F02003002B09D1BB6803F47C03FC
:106C4000002B0CD03B6903F04003002B07D0FB68FE
:106C50001B68DA6DFB681B6842F00202DA65BB68EC
:106C600003F08003002B09D0FB681B68D3F8DC100D
:106C7000FB681B687A680A43C3F8DC20BB6803F42E
:106C80008073002B09D0FB681B68D3F8E010FB6809
:106C90001B687A680A43C3F8E020FB681B68596DDB
:106CA000FB681B68BA680A435A65002306E0FB6864
:106CB0001B6E43F00202FB681A66012318461C375C
:106CC000BD465DF8047B704780B58CB000AF78603E
:106CD0007B681B681B6D03F4E053FB627B681B68D9
:106CE0005B6DFA6A1340FB627B681B681B6D03F0E7
:106CF0000703BB627B681B685B6DBA6A1340BB62AB
:106D00007B681B681B6D03F038037B627B681B6824
:106D10005B6D7A6A13407B627B681B681B6D03F4B2
:106D200071033B627B681B685B6D3A6A13403B6290
:106D30007B681B681B6D03F46023FB617B681B6829
:106D40005B6DFA691340FB617B681B685B6DBB611F
:106D50007B681B681B6D7B617B699B0903F00103EA
:106D6000002B0CD0BB699B0903F00103002B06D05C
:106D70007B681B6840221A65786800F017F97B6908
:106D80001B0A03F00103002B1AD0BB691B0A03F096
:106D90000103002B14D07B681B68D3F8D8303B610B
:106DA0007B681B68D3F8E0303A6913403B617B682D
:106DB0001B684FF480721A653969786800F0D7F85B
:106DC000FB6A002B07D07B681B68FA6A1A65F96AB0
:106DD000786800F0ACF8BB6A002B07D07B681B68B2
:106DE000BA6A1A65B96A786807F07AF87B6A002B84
:106DF00007D07B681B687A6A1A65796A786800F040
:106E0000A1F87B695B0A03F00103002B0DD0BB697D
:106E10005B0A03F00103002B07D07B681B684FF46B
:106E200000721A65786800F098F87B69DB0903F056
:106E30000103002B19D0BB69DB0903F00103002B10
:106E400013D07B681B68D3F8D430FB607B681B6869
:106E5000D3F8DC30FA681340FB607B681B68802243
:106E60001A65F968786807F0E1FA7B695B0B03F053
:106E70000103002B0DD0BB695B0B03F00103002B5A
:106E800007D07B681B684FF400521A65786800F0E1
:106E900079F87B69DB0B03F00103002B0DD0BB6994
:106EA000DB0B03F00103002B07D07B681B684FF45A
:106EB00000421A65786800F06FF87B699B0B03F05D
:106EC0000103002B10D0BB699B0B03F00103002BC7
:106ED0000AD07B681B684FF480421A657B681B6E82
:106EE00043F080027B681A66FB69002B07D07B6841
:106EF0001B68FA691A65F969786800F06BF83B6AF3
:106F0000002B09D07B681B683A6A1A657B681A6E89
:106F10003B6A1A437B681A667B681B6E002B02D0A3
:106F2000786800F04DF800BF3037BD4680BD80B4B2
:106F300083B000AF7860396000BF0C37BD465DF8A4
:106F4000047B704780B483B000AF7860396000BFC5
:106F50000C37BD465DF8047B704780B483B000AF4A
:106F6000786000BF0C37BD465DF8047B704780B485
:106F700083B000AF7860396000BF0C37BD465DF864
:106F8000047B704780B483B000AF786000BF0C37DB
:106F9000BD465DF8047B704780B483B000AF786075
:106FA00000BF0C37BD465DF8047B704780B483B0EA
:106FB00000AF786000BF0C37BD465DF8047B7047BA
:106FC00080B483B000AF786000BF0C37BD465DF879
:106FD000047B704780B483B000AF7860396000BF35
:106FE0000C37BD465DF8047B7047000080B485B067
:106FF00000AF7860304BBB607B681B682F4A9342C0
:1070000003D1BB6803F55473BB607B681B682C4AD3
:10701000934203D1BB6803F5D463BB607B68BA6855
:107020001A647B681B68D3F8803023F4F8117B68FE
:107030005B6B1A047B681B680A43C3F88020BB683B
:1070400003F170027B685A647B681B68D3F8803058
:1070500023F070617B689B6B1A067B681B680A4390
:10706000C3F88020BB6803F1B0027B689A64BB68F8
:1070700003F5C4727B68DA64BB6803F518727B6839
:107080001A65BB6803F51E727B685A65BB68FB60B6
:1070900005E0FB6800221A60FB680433FB60BB68F4
:1070A00003F55473FA689A42F3D300BF00BF143754
:1070B000BD465DF8047B704700A4004000680040B6
:1070C000006C004080B489B000AFF860B9607A60AD
:1070D0003B60BB685B68002B0AD1BB681A69BB6860
:1070E0009B681A43BB681B689B041343FB610AE05F
:1070F000BB681A69BB689B681A43BB681B6813436B
:1071000043F08043FB61BB681B6A1A06BB68DB69FE
:107110001A43BB689B691A43BB685B691A43BB6827
:10712000DB681B0413433B61FB68596D3A681346E7
:10713000DB001344DB000B44BB61BB69FA691A60D6
:10714000BB690433BB61BB693A691A60BB6904332C
:10715000BB6100237B6120E07B6903337A681344C1
:107160001B781A067B69023379680B441B781B0471
:107170001A437B69013379680B441B781B02134364
:1071800079687A690A4412781A43BB691A60BB6944
:107190000433BB617B6904337B61BB68DB68064AEF
:1071A000D35C1A467B699342D6D300BF00BF243715
:1071B000BD465DF8047B7047B448010880B584B0D3
:1071C00000AF78607B68002B01D101239DE07B68D4
:1071D0005B6A002B08D17B685B68B3F5827F09D0BE
:1071E0007B680022DA6105E07B6800221A617B6817
:1071F00000225A617B6800229A627B6893F85D30B6
:10720000DBB2002B06D17B68002283F85C20786813
:1072100004F0BEFC7B68022283F85D207B681B685B
:107220001A687B681B6822F040021A607B68DB6882
:10723000B3F5E06F02D90023FB6002E04FF4805306
:10724000FB607B68DB68B3F5706F07D07B68DB6839
:10725000B3F5E06F02D07B6800229A627B685B68BE
:1072600003F482727B689B6803F404431A437B68CF
:107270001B6903F002031A437B685B6903F0010397
:107280001A437B689B6903F400731A437B68DB69CC
:1072900003F038031A437B681B6A03F0800342EA59
:1072A00003017B689B6A03F400527B681B680A43F6
:1072B0001A607B689B691B0C03F004027B685B6AA5
:1072C00003F010031A437B685B6B03F008031A4357
:1072D0007B68DB6803F4706342EA0301FB6803F434
:1072E00080527B681B680A435A607B681B68DA69B6
:1072F0007B681B6822F40062DA617B6800221A66F0
:107300007B68012283F85D20002318461037BD46B4
:1073100080BD80B588B000AFF860B9603B601346AF
:10732000FB80FDF785F8F861FB887B83FB6893F8A9
:107330005D30DBB2012B01D002235CE1BB68002B86
:1073400002D0FB88002B01D1012354E1FB6893F8A4
:107350005C30012B01D102234DE1FB68012283F84F
:107360005C20FB68032283F85D20FB6800221A661C
:10737000FB68BA689A63FB68FA889A87FB68FA88A0
:10738000DA87FB6800221A64FB680022A3F8442015
:10739000FB680022A3F84620FB6800221A65FB6800
:1073A0000022DA64FB689B68B3F5004F0FD1FB68DD
:1073B0001B681A68FB681B6822F040021A60FB68B1
:1073C0001B681A68FB681B6842F480421A60FB68FD
:1073D0001B681B6803F04003402B07D0FB681B6849
:1073E0001A68FB681B6842F040021A60FB68DB68A1
:1073F000B3F5E06F52D9FB685B68002B02D07B8B42
:10740000012B45D1FB689B6B1A88FB681B68DA600F
:10741000FB689B6B9A1CFB689A63FB68DB8F9BB2D3
:10742000013B9AB2FB68DA8732E0FB681B689B6815
:1074300003F00203022B12D1FB689B6B1A88FB68D6
:107440001B68DA60FB689B6B9A1CFB689A63FB689D
:10745000DB8F9BB2013B9AB2FB68DA8718E0FCF73E
:10746000E7FF0246FB69D31A3A689A4203D83B68A1
:10747000B3F1FF3F02D13B68002B09D1FB68012229
:1074800083F85D20FB68002283F85C200323B2E0D0
:10749000FB68DB8F9BB2002BC7D183E0FB685B6886
:1074A000002B02D07B8B012B77D1FB68DB8F9BB24B
:1074B000012B12D9FB689B6B1A88FB681B68DA608A
:1074C000FB689B6B9A1CFB689A63FB68DB8F9BB223
:1074D000023B9AB2FB68DA875FE0FB689A6BFB6855
:1074E0001B680C3312781A70FB689B6B5A1CFB6884
:1074F0009A63FB68DB8F9BB2013B9AB2FB68DA8729
:107500004BE0FB681B689B6803F00203022B2BD146
:10751000FB68DB8F9BB2012B12D9FB689B6B1A882F
:10752000FB681B68DA60FB689B6B9A1CFB689A63BC
:10753000FB68DB8F9BB2023B9AB2FB68DA872CE0D8
:10754000FB689A6BFB681B680C3312781A70FB6837
:107550009B6B5A1CFB689A63FB68DB8F9BB2013BF9
:107560009AB2FB68DA8718E0FCF762FF0246FB6913
:10757000D31A3A689A4203D83B68B3F1FF3F02D16D
:107580003B68002B09D1FB68012283F85D20FB6872
:10759000002283F85C2003232DE0FB68DB8F9BB285
:1075A000002BAED1FA693968F86800F0F5FC0346A3
:1075B000002B02D0FB6820221A66FB689B68002B18
:1075C0000AD100237B61FB681B68DB687B61FB6879
:1075D0001B689B687B617B69FB68012283F85D20E7
:1075E000FB68002283F85C20FB681B6E002B01D037
:1075F000012300E0002318462037BD4680BD80B53A
:1076000088B002AFF860B9603B601346FB80FB684E
:1076100093F85D30DBB2012B01D0022323E1BB687C
:10762000002B02D0FB88002B01D101231BE1FB685A
:107630005B68B3F5827F12D1FB689B68002B0ED18B
:10764000FB68042283F85D20FA883B6800931346A8
:10765000BA68B968F86800F00AF9034603E1FCF774
:10766000E7FE7861FB6893F85C30012B01D10223BF
:10767000F9E0FB68012283F85C20FB68042283F8B0
:107680005D20FB6800221A66FB68BA681A64FB6812
:10769000FA88A3F84420FB68FA88A3F84620FB6820
:1076A00000229A63FB6800229A87FB680022DA872F
:1076B000FB680022DA64FB6800221A65FB68DB685D
:1076C000B3F5E06F08D9FB681B685A68FB681B6854
:1076D00022F480525A6007E0FB681B685A68FB6816
:1076E0001B6842F480525A60FB689B68B3F5004FF8
:1076F0000FD1FB681B681A68FB681B6822F0400208
:107700001A60FB681B681A68FB681B6822F48042D9
:107710001A60FB681B681B6803F04003402B07D00E
:10772000FB681B681A68FB681B6842F040021A601D
:10773000FB68DB68B3F5E06F75D837E0FB681B6862
:107740009B6803F00103012B17D1FB681B6803F151
:107750000C02FB681B6C1278D2B21A70FB681B6CAF
:107760005A1CFB681A64FB68B3F846309BB2013BB5
:107770009AB2FB68A3F8462018E0FCF759FE0246CF
:107780007B69D31A3A689A4203D83B68B3F1FF3F4A
:1077900002D13B68002B09D1FB68012283F85D20F0
:1077A000FB68002283F85C2003235CE0FB68B3F8ED
:1077B00046309BB2002BC1D13BE0FB681B689B6845
:1077C00003F00103012B15D1FB681B68DA68FB6825
:1077D0001B6C92B21A80FB681B6C9A1CFB681A64C3
:1077E000FB68B3F846309BB2013B9AB2FB68A3F842
:1077F000462018E0FCF71CFE02467B69D31A3A6863
:107800009A4203D83B68B3F1FF3F02D13B68002B9B
:1078100009D1FB68012283F85D20FB68002283F810
:107820005C2003231FE0FB68B3F846309BB2002BBB
:10783000C3D17A693968F86800F056FB0346002B1B
:1078400002D0FB6820221A66FB68012283F85D20C3
:10785000FB68002283F85C20FB681B6E002B01D0C4
:10786000012300E0002318461837BD4680BD80B5CF
:107870008AB000AFF860B9607A607B8001237B62D8
:10788000FCF7D6FD3862FB6893F85D30FB77FB6848
:107890005B68BB617B88FB827B88BB82FB7F012BA3
:1078A0000CD0BB69B3F5827F06D1FB689B68002BC7
:1078B00002D1FB7F042B01D00223F3E1BB68002B34
:1078C00005D07B68002B02D07B88002B01D10123DF
:1078D000E8E1FB6893F85C30012B01D10223E1E180
:1078E000FB68012283F85C20FB6893F85D30DBB213
:1078F000042B03D0FB68052283F85D20FB6800227F
:107900001A66FB687A681A64FB687A88A3F84620CE
:10791000FB687A88A3F84420FB68BA689A63FB681E
:107920007A88DA87FB687A889A87FB680022DA64AB
:10793000FB6800221A65FB68DB68B3F5E06F02D8CC
:10794000BB8A012B08D9FB681B685A68FB681B6857
:1079500022F480525A6007E0FB681B685A68FB6893
:107960001B6842F480525A60FB681B681B6803F076
:107970004003402B07D0FB681B681A68FB681B6834
:1079800042F040021A60FB68DB68B3F5E06F40F23A
:107990008380FB685B68002B02D0FB8A012B6FD1D0
:1079A000FB689B6B1A88FB681B68DA60FB689B6B43
:1079B0009A1CFB689A63FB68DB8F9BB2013B9AB20F
:1079C000FB68DA875CE0FB681B689B6803F00203D6
:1079D000022B1BD1FB68DB8F9BB2002B16D07B6A7E
:1079E000012B13D1FB689B6B1A88FB681B68DA605C
:1079F000FB689B6B9A1CFB689A63FB68DB8F9BB2EE
:107A0000013B9AB2FB68DA8700237B62FB681B6844
:107A10009B6803F00103012B1CD1FB68B3F84630CF
:107A20009BB2002B16D0FB681B68DA68FB681B6CE6
:107A300092B21A80FB681B6C9A1CFB681A64FB6884
:107A4000B3F846309BB2013B9AB2FB68A3F84620DC
:107A500001237B62FCF7ECFC02463B6AD31A3A6BCB
:107A60009A420DD83B6BB3F1FF3F09D0FB6801226E
:107A700083F85D20FB68002283F85C20032311E17A
:107A8000FB68DB8F9BB2002B9DD1FB68B3F84630BF
:107A90009BB2002B97D1E5E0FB685B68002B03D01D
:107AA000FB8A012B40F0D180FB68DB8F9BB2012B5E
:107AB00012D9FB689B6B1A88FB681B68DA60FB684D
:107AC0009B6B9A1CFB689A63FB68DB8F9BB2023B43
:107AD0009AB2FB68DA87B8E0FB689A6BFB681B68B0
:107AE0000C3312781A70FB689B6B5A1CFB689A6304
:107AF000FB68DB8F9BB2013B9AB2FB68DA87A4E09C
:107B0000FB681B689B6803F00203022B34D1FB68FF
:107B1000DB8F9BB2002B2FD07B6A012B2CD1FB6813
:107B2000DB8F9BB2012B12D9FB689B6B1A88FB6819
:107B30001B68DA60FB689B6B9A1CFB689A63FB68A6
:107B4000DB8F9BB2023B9AB2FB68DA8712E0FB68DC
:107B50009A6BFB681B680C3312781A70FB689B6B7E
:107B60005A1CFB689A63FB68DB8F9BB2013B9AB29D
:107B7000FB68DA8700237B62FB681B689B6803F065
:107B80000103012B48D1FB68B3F846309BB2002BB0
:107B900042D0FB68B3F846309BB2012B23D9FB6877
:107BA0001B68DA68FB681B6C92B21A80FB681B6C5E
:107BB0009A1CFB681A64FB68B3F846309BB2023B20
:107BC0009AB2FB68A3F84620FB68B3F846309BB234
:107BD000012B1FD8FB681B685A68FB681B6842F4BE
:107BE00080525A6016E0FB681B6803F10C02FB68C8
:107BF0001B6C1278D2B21A70FB681B6C5A1CFB68A3
:107C00001A64FB68B3F846309BB2013B9AB2FB683A
:107C1000A3F8462001237B62FCF70AFC02463B6A7C
:107C2000D31A3A6B9A4203D83B6BB3F1FF3F02D1B0
:107C30003B6B002B09D1FB68012283F85D20FB68B8
:107C4000002283F85C2003232CE0FB68DB8F9BB2CF
:107C5000002B7FF455AFFB68B3F846309BB2002B86
:107C60007FF44EAF3A6A396BF86800F095F9034635
:107C7000002B08D0FB6820221A66FB68002283F8DC
:107C80005C2001230EE0FB68012283F85D20FB6885
:107C9000002283F85C20FB681B6E002B01D00123BF
:107CA00000E0002318462837BD4680BD80B588B067
:107CB00000AFF860B9603B601346FB71FCF7B8FB9E
:107CC0000246BB6A9B1A3A681344FB61FCF7B0FB9F
:107CD000B861394B1B685B011B0DFA6902FB03F3AA
:107CE0007B6154E03B68B3F1FF3F50D0FCF7A0FB51
:107CF0000246BB69D31AFA699A4202D9FB69002B82
:107D00003DD1FB681B685A68FB681B6822F0E002E3
:107D10005A60FB685B68B3F5827F11D1FB689B6892
:107D2000B3F5004F04D0FB689B68B3F5806F07D1B3
:107D3000FB681B681A68FB681B6822F040021A6027
:107D4000FB689B6AB3F5005F0FD1FB681B681A687C
:107D5000FB681B6822F400521A60FB681B681A68F3
:107D6000FB681B6842F400521A60FB68012283F82A
:107D70005D20FB68002283F85C20032317E07B6909
:107D8000002B01D10023FB617B69013B7B61FB6818
:107D90001B689A68BB681340BA689A420CBF0123FB
:107DA0000023DBB21A46FB799A429BD10023184686
:107DB0002037BD4680BD00BF0000002080B58AB0DE
:107DC00000AFF860B9607A603B600023FB75FCF798
:107DD0002FFB02463B6B9B1A3A6813447B62FCF70D
:107DE00027FB3862FB681B680C33FB613D4B1A684C
:107DF00013469B001344DA00D31A1B0D7A6A02FB68
:107E000003F3BB6160E0BB68B3F5C06F07D17B686B
:107E1000002B04D1FB691B78DBB2FB75FB7D3B6853
:107E2000B3F1FF3F50D0FCF703FB02463B6AD31A85
:107E30007A6A9A4202D97B6A002B3DD1FB681B68A3
:107E40005A68FB681B6822F0E0025A60FB685B68B6
:107E5000B3F5827F11D1FB689B68B3F5004F04D066
:107E6000FB689B68B3F5806F07D1FB681B681A68D5
:107E7000FB681B6822F040021A60FB689B6AB3F53E
:107E8000005F0FD1FB681B681A68FB681B6822F44F
:107E900000521A60FB681B681A68FB681B6842F492
:107EA00000521A60FB68012283F85D20FB68002203
:107EB00083F85C20032310E0BB69002B01D1002371
:107EC0007B62BB69013BBB61FB681B689A68BB684E
:107ED00013407A689A4296D1002318462837BD4647
:107EE00080BD00BF0000002080B586B002AFF86002
:107EF000B9607A60FB685B68B3F5827F11D1FB687B
:107F00009B68B3F5004F04D0FB689B68B3F5806FA6
:107F100007D1FB681B681A68FB681B6822F04002E7
:107F20001A607B680093BB6800228021F868FFF725
:107F3000BDFE0346002B07D0FB681B6E43F02002FA
:107F4000FB681A66032323E0FB685B68B3F5827F56
:107F50001DD1FB689B68B3F5004F04D0FB689B689C
:107F6000B3F5806F13D17B680093BB6800224FF498
:107F7000C061F868FFF722FF0346002B07D0FB68BB
:107F80001B6E43F02002FB681A66032300E0002307
:107F900018461037BD4680BD80B586B002AFF86088
:107FA000B9607A607B680093BB6800224FF4C051CF
:107FB000F868FFF703FF0346002B07D0FB681B6E32
:107FC00043F02002FB681A66032327E07B680093D6
:107FD000BB6800228021F868FFF768FE0346002B8B
:107FE00007D0FB681B6E43F02002FB681A66032370
:107FF00014E07B680093BB6800224FF4C061F8680E
:10800000FFF7DCFE0346002B07D0FB681B6E43F036
:108010002002FB681A66032300E00023184610378D
:10802000BD4680BD80B582B000AF78607B68002B14
:1080300001D1012349E07B6893F83D30DBB2002B8E
:1080400006D17B68002283F83C20786803F054FE58
:108050007B68022283F83D207B681A687B680433C2
:108060001946104600F05CFA7B68012283F848202C
:108070007B68012283F83E207B68012283F83F2041
:108080007B68012283F840207B68012283F841202D
:108090007B68012283F842207B68012283F8432019
:1080A0007B68012283F844207B68012283F8452005
:1080B0007B68012283F846207B68012283F84720F1
:1080C0007B68012283F83D20002318460837BD460F
:1080D00080BD000080B584B000AF786039603B6837
:1080E000002B09D17B6893F83E30DBB2012B14BF23
:1080F00001230023DBB23CE03B68042B09D17B6801
:1081000093F83F30DBB2012B14BF01230023DBB215
:108110002FE03B68082B09D17B6893F84030DBB235
:10812000012B14BF01230023DBB222E03B680C2BA0
:1081300009D17B6893F84130DBB2012B14BF0123D6
:108140000023DBB215E03B68102B09D17B6893F864
:108150004230DBB2012B14BF01230023DBB208E065
:108160007B6893F84330DBB2012B14BF012300235B
:10817000DBB2002B01D00123A6E03B68002B04D129
:108180007B68022283F83E2023E03B68042B04D165
:108190007B68022283F83F201BE03B68082B04D158
:1081A0007B68022283F8402013E03B680C2B04D14B
:1081B0007B68022283F841200BE03B68102B04D13E
:1081C0007B68022283F8422003E07B68022283F866
:1081D00043207B681B6801223968184600F07EFD49
:1081E0007B681B683A4A934218D07B681B68394AFF
:1081F000934213D07B681B68374A93420ED07B684A
:108200001B68364A934209D07B681B68344A934204
:1082100004D07B681B68334A934201D1012300E0FC
:108220000023002B07D07B681B685A6C7B681B6897
:1082300042F400425A647B681B68254A934222D06C
:108240007B681B68B3F1804F1DD07B681B68264A92
:10825000934218D07B681B68244A934213D07B68F2
:108260001B68234A93420ED07B681B68194A9342CD
:1082700009D07B681B68184A934204D07B681B684E
:10828000184A934215D17B681B689A68194B1340B2
:10829000FB60FB68062B15D0FB68B3F5803F11D05F
:1082A0007B681B681A687B681B6842F001021A60D1
:1082B00008E07B681B681A687B681B6842F0010253
:1082C0001A6000E000BF002318461037BD4680BD8D
:1082D000002C0140003401400040014000440140B6
:1082E00000480140005001400004004000080040E8
:1082F000000C00400700010080B586B000AFF860B8
:10830000B9607A600023FB75FB6893F83C30012B61
:1083100001D10223FFE0FB68012283F83C207B6847
:10832000142B00F2F08001A252F823F081830008A0
:10833000078500080785000807850008C183000835
:1083400007850008078500080785000803840008E2
:108350000785000807850008078500084384000892
:108360000785000807850008078500088584000840
:10837000078500080785000807850008C5840008F0
:10838000FB681B68B968184600F07EF9FB681B683B
:108390009A69FB681B6842F008029A61FB681B68D7
:1083A0009A69FB681B6822F004029A61FB681B68EB
:1083B0009969BB681A69FB681B680A439A61A5E062
:1083C000FB681B68B968184600F0F8F9FB681B6881
:1083D0009A69FB681B6842F400629A61FB681B683B
:1083E0009A69FB681B6822F480629A61FB681B68CB
:1083F0009969BB681B691A02FB681B680A439A618A
:1084000084E0FB681B68B968184600F06BFAFB68EB
:108410001B68DA69FB681B6842F00802DA61FB68D6
:108420001B68DA69FB681B6822F00402DA61FB68EA
:108430001B68D969BB681A69FB681B680A43DA6163
:1084400064E0FB681B68B968184600F0DDFAFB6859
:108450001B68DA69FB681B6842F40062DA61FB683A
:108460001B68DA69FB681B6822F48062DA61FB68CA
:108470001B68D969BB681B691A02FB681B680A4341
:10848000DA6143E0FB681B68B968184600F050FBEE
:10849000FB681B681A6DFB681B6842F008021A65CE
:1084A000FB681B681A6DFB681B6822F004021A65E2
:1084B000FB681B68196DBB681A69FB681B680A4377
:1084C0001A6523E0FB681B68B968184600F09AFB40
:1084D000FB681B681A6DFB681B6842F400621A6532
:1084E000FB681B681A6DFB681B6822F480621A65C2
:1084F000FB681B68196DBB681B691A02FB681B6867
:108500000A431A6502E00123FB7500BFFB680022E5
:1085100083F83C20FB7D18461837BD4680BD00BF60
:1085200080B485B000AF786039607B681B68FB6001
:108530007B684C4A934217D07B68B3F1804F13D0CD
:108540007B68494A93420FD07B68484A93420BD0DC
:108550007B68474A934207D07B68464A934203D0E0
:108560007B68454A934208D1FB6823F07003FB60A7
:108570003B685B68FA681343FB607B68394A934247
:1085800023D07B68B3F1804F1FD07B68364A93427B
:108590001BD07B68354A934217D07B68344A93429C
:1085A00013D07B68334A93420FD07B68334A93429F
:1085B0000BD07B68324A934207D07B68314A9342A2
:1085C00003D07B682C4A934208D1FB6823F44073A4
:1085D000FB603B68DB68FA681343FB60FB6823F0D1
:1085E00080023B685B691343FB607B68FA681A6032
:1085F0003B689A687B68DA623B681A687B689A62B3
:108600007B68184A934213D07B681A4A93420FD072
:108610007B681A4A93420BD07B68194A934207D071
:108620007B68184A934203D07B68134A934203D174
:108630003B681A697B681A637B6801225A617B6810
:108640001B6903F00103012B05D17B681B6923F033
:1086500001027B681A6100BF1437BD465DF8047BD8
:10866000704700BF002C014000040040000800409B
:10867000000C004000340140005001400040014027
:10868000004401400048014080B487B000AF7860EA
:1086900039607B681B6A7B617B681B6A23F001027F
:1086A0007B681A627B685B683B617B689B69FB60E7
:1086B000FB6823F4803323F07003FB60FB6823F036
:1086C0000303FB603B681B68FA681343FB607B692C
:1086D00023F002037B613B689B687A6913437B61EB
:1086E0007B68304A934213D07B682F4A93420FD065
:1086F0007B682E4A93420BD07B682D4A934207D069
:108700007B682C4A934203D07B682B4A93420CD15E
:108710007B6923F008037B613B68DB687A6913435C
:108720007B617B6923F004037B617B681D4A934274
:1087300013D07B681C4A93420FD07B681B4A93423C
:108740000BD07B681A4A934207D07B68194A934240
:1087500003D07B68184A934211D13B6923F480739C
:108760003B613B6923F400733B613B685B693A6999
:1087700013433B613B689B693A6913433B617B68E8
:108780003A695A607B68FA689A613B685A687B6804
:108790005A637B687A691A6200BF1C37BD465DF870
:1087A000047B7047002C0140003401400040014030
:1087B00000440140004801400050014080B487B0AF
:1087C00000AF786039607B681B6A7B617B681B6ADD
:1087D00023F010027B681A627B685B683B617B68F0
:1087E0009B69FB60FB6823F0807323F4E043FB602C
:1087F000FB6823F44073FB603B681B681B02FA684C
:108800001343FB607B6923F020037B613B689B681B
:108810001B017A6913437B617B682C4A934207D022
:108820007B682B4A934203D07B682A4A93420DD13E
:108830007B6923F080037B613B68DB681B017A69FD
:1088400013437B617B6923F040037B617B681F4A94
:10885000934213D07B681E4A93420FD07B681E4A16
:1088600093420BD07B681D4A934207D07B681C4A19
:10887000934203D07B68174A934213D13B6923F498
:1088800080633B613B6923F400633B613B685B6948
:108890009B003A6913433B613B689B699B003A69C3
:1088A00013433B617B683A695A607B68FA689A6156
:1088B0003B685A687B689A637B687A691A6200BF72
:1088C0001C37BD465DF8047B704700BF002C01409B
:1088D000003401400050014000400140004401408C
:1088E0000048014080B487B000AF786039607B6891
:1088F0001B6A7B617B681B6A23F480727B681A6247
:108900007B685B683B617B68DB69FB60FB6823F429
:10891000803323F07003FB60FB6823F00303FB60EC
:108920003B681B68FA681343FB607B6923F40073A0
:108930007B613B689B681B027A6913437B617B68A0
:108940002B4A934207D07B682A4A934203D07B6824
:10895000294A93420DD17B6923F400637B613B6814
:10896000DB681B027A6913437B617B6923F48063B4
:108970007B617B681E4A934213D07B681D4A9342F9
:108980000FD07B681D4A93420BD07B681C4A9342F0
:1089900007D07B681B4A934203D07B68164A9342F8
:1089A00013D13B6923F480533B613B6923F40053AB
:1089B0003B613B685B691B013A6913433B613B6860
:1089C0009B691B013A6913433B617B683A695A60B2
:1089D0007B68FA68DA613B685A687B68DA637B68AF
:1089E0007A691A6200BF1C37BD465DF8047B704788
:1089F000002C014000340140005001400040014083
:108A0000004401400048014080B487B000AF786066
:108A100039607B681B6A7B617B681B6A23F4805228
:108A20007B681A627B685B683B617B68DB69FB6023
:108A3000FB6823F0807323F4E043FB60FB6823F4BE
:108A40004073FB603B681B681B02FA681343FB60C2
:108A50007B6923F400537B613B689B681B037A6945
:108A600013437B617B682C4A934207D07B682B4A77
:108A7000934203D07B682A4A93420DD17B6923F449
:108A800000437B613B68DB681B037A6913437B61AE
:108A90007B6923F480437B617B681F4A934213D038
:108AA0007B681E4A93420FD07B681E4A93420BD0CC
:108AB0007B681D4A934207D07B681C4A934203D0CF
:108AC0007B68174A934213D13B6923F480433B618F
:108AD0003B6923F400433B613B685B699B013A6956
:108AE00013433B613B689B699B013A6913433B61BC
:108AF0007B683A695A607B68FA68DA613B685A6851
:108B00007B681A647B687A691A6200BF1C37BD46AD
:108B10005DF8047B704700BF002C01400034014029
:108B20000050014000400140004401400048014025
:108B300080B487B000AF786039607B681B6A3B61A6
:108B40007B681B6A23F480327B681A627B685B68EF
:108B50007B617B681B6DFB60FB6823F4803323F033
:108B60007003FB603B681B68FA681343FB603B695A
:108B700023F400333B613B689B681B043A69134351
:108B80003B617B68194A934213D07B68184A934231
:108B90000FD07B68174A93420BD07B68164A9342EA
:108BA00007D07B68154A934203D07B68144A9342EE
:108BB00009D17B6923F480337B613B685B691B02CD
:108BC0007A6913437B617B687A695A607B68FA68CB
:108BD0001A653B685A687B689A647B683A691A62CE
:108BE00000BF1C37BD465DF8047B7047002C014078
:108BF0000034014000400140004401400048014071
:108C00000050014080B487B000AF786039607B6865
:108C10001B6A3B617B681B6A23F480127B681A62C3
:108C20007B685B687B617B681B6DFB60FB6823F086
:108C3000807323F4E043FB603B681B681B02FA6807
:108C40001343FB603B6923F400133B613B689B6863
:108C50001B053A6913433B617B681A4A934213D060
:108C60007B68194A93420FD07B68184A93420BD015
:108C70007B68174A934207D07B68164A934203D019
:108C80007B68154A934209D17B6923F480237B6179
:108C90003B685B699B027A6913437B617B687A69F5
:108CA0005A607B68FA681A653B685A687B68DA64C0
:108CB0007B683A691A6200BF1C37BD465DF8047BC9
:108CC000704700BF002C01400034014000400140CB
:108CD00000440140004801400050014080B487B08A
:108CE00000AFF860B9607A60BB6803F01F0301222F
:108CF00002FA03F37B61FB681A6A7B69DB431A4063
:108D0000FB681A62FB681A6ABB6803F01F03796884
:108D100001FA03F31A43FB681A6200BF1C37BD4611
:108D20005DF8047B7047000080B485B000AF7860C8
:108D300039607B6893F83C30012B01D1022374E049
:108D40007B68012283F83C207B68022283F83D2067
:108D50007B681B685B68FB607B681B689B68BB600B
:108D60007B681B68344A934209D07B681B68334A8E
:108D7000934204D07B681B68314A934208D1FB6858
:108D800023F47003FB603B685B68FA681343FB6085
:108D9000FB6823F0007323F07003FB603B681B68E3
:108DA000FA681343FB607B681B68FA685A607B684B
:108DB0001B68214A934222D07B681B68B3F1804F25
:108DC0001DD07B681B681F4A934218D07B681B68C4
:108DD0001D4A934213D07B681B681C4A93420ED0F5
:108DE0007B681B68154A934209D07B681B68184A48
:108DF000934204D07B681B68114A93420CD1BB6834
:108E000023F08003BB603B689B68BA681343BB6078
:108E10007B681B68BA689A607B68012283F83D20F2
:108E20007B68002283F83C20002318461437BD4697
:108E30005DF8047B704700BF002C01400034014006
:108E4000005001400004004000080040000C0040B9
:108E50000040014080B586B000AFF860B9601346AD
:108E6000FB71FB68002B01D103231FE0FB6800228C
:108E7000C3F8B822FB680022C3F8C022FB680022B6
:108E8000C3F8CC22BB68002B03D0FB68BA68C3F8D8
:108E9000B422FB68012283F89C22FB68FA791A70DD
:108EA000F86802F027F80346FB75FB7D1846183773
:108EB000BD4680BD80B584B000AF7860786802F0B0
:108EC000AFF87B68012283F89C227B68D3F8B83224
:108ED000002B11D07B68D3F8B8325B687A6852688F
:108EE000D2B21146786898477B680022C3F8B8224E
:108EF0007B680022C3F8C0227B680022C3F8B4223A
:108F00007B680022C3F8CC22786802F053F803464D
:108F1000FB73FB7B18461037BD4680BD80B584B01F
:108F200000AF786039600023FB813B68002B01D1E2
:108F3000032316E07B683A68C3F8B8227B68D3F84D
:108F4000B832DB6A002B0BD07B68D3F8B832DB6A0F
:108F500007F10E021046984702467B68C3F8CC2200
:108F6000002318461037BD4680BD80B582B000AFE3
:108F70007860786802F039F8034618460837BD462D
:108F800080BD80B483B000AF7860002318460C37F2
:108F9000BD465DF8047B704780B584B000AF786053
:108FA0000B46FB700323FB737B68D3F8B832002BAE
:108FB00009D07B68D3F8B8321B68FA781146786814
:108FC00098470346FB73FB7B18461037BD4680BDB0
:108FD00080B582B000AF78600B46FB707B68D3F839
:108FE000B832002B07D07B68D3F8B8325B68FA78C8
:108FF000114678689847002318460837BD4680BD5B
:1090000080B584B000AF786039607B6803F2AA2332
:109010003968184600F048FF7B680122C3F89422A3
:109020007B68B3F8B0321A467B68C3F898227B6835
:1090300093F8AA3203F01F03022B1AD0022B22D876
:10904000002B02D0012B0AD01DE07B6803F2AA237B
:109050001946786800F0F0F90346FB7320E07B685E
:1090600003F2AA231946786800F054FA0346FB730A
:1090700016E07B6803F2AA231946786800F093FA99
:109080000346FB730CE07B6893F8AA3223F07F035E
:10909000DBB21946786802F023F80346FB7300BF81
:1090A000FB7B18461037BD4680BD80B586B000AF4B
:1090B000F8600B467A60FB72FB7A002B38D1FB68B4
:1090C00003F5AA733B61FB68D3F89432032B4AD1B2
:1090D0003B699A683B69DB689A4213D93B699A6895
:1090E0003B69DB68D21A3B699A603B69DA683B6985
:1090F0009B68934228BF13461A467968F86800F0C7
:10910000C7FF30E0FB6893F89C32DBB2032B0BD136
:10911000FB68D3F8B8321B69002B05D0FB68D3F885
:10912000B8321B69F8689847F86800F0C2FF1AE087
:10913000FB6893F89C32DBB2032B14D1FB68D3F8A5
:10914000B8329B69002B0ED0FB68D3F8B8329B690C
:10915000FA7A1146F86898470346FB75FB7D002BA9
:1091600001D0FB7D00E0002318461837BD4680BDC6
:1091700080B586B000AFF8600B467A60FB72FB7A70
:10918000002B6BD1FB6814333B61FB68D3F894323E
:10919000022B56D13B699A683B69DB689A4214D925
:1091A0003B699A683B69DB68D21A3B699A603B6904
:1091B0009B681A467968F86800F03CFF002300229B
:1091C0000021F86802F036F83BE03B69DA683B6959
:1091D0009B689A421CD13B695A683B69DB689A429A
:1091E00016D33B695A68FB68D3F898329A420FD27B
:1091F00000220021F86800F01DFFFB680022C3F880
:109200009822002300220021F86802F013F818E0E9
:10921000FB6893F89C32DBB2032B0BD1FB68D3F8CD
:10922000B832DB68002B05D0FB68D3F8B832DB68B6
:10923000F86898478021F86801F052FFF86800F05C
:109240004BFFFB6893F8A032012B22D1F868FFF79F
:1092500098FEFB68002283F8A0221AE0FB6893F8CE
:109260009C32DBB2032B14D1FB68D3F8B8325B69B4
:10927000002B0ED0FB68D3F8B8325B69FA7A11463E
:10928000F86898470346FB75FB7D002B01D0FB7DFA
:1092900000E0002318461837BD4680BD80B582B077
:1092A00000AF78607B68012283F89C227B680022F3
:1092B000C3F894227B6800225A607B680022C3F8BE
:1092C000A4227B68D3F8B832002B01D103232FE00E
:1092D0007B68D3F8BC32002B0FD07B68D3F8B83250
:1092E0005B68002B09D07B68D3F8B8325B687A687A
:1092F0005268D2B211467868984740230022002174
:10930000786801F0A8FE7B680122A3F864217B68DD
:109310004022C3F86021402300228021786801F0B8
:109320009AFE7B6801229A847B6840221A6200239D
:1093300018460837BD4680BD80B483B000AF786062
:109340000B46FB707B68FA781A74002318460C37BA
:10935000BD465DF8047B704780B483B000AF786091
:109360007B6893F89C32DAB27B6883F89D227B6835
:10937000042283F89C22002318460C37BD465DF872
:10938000047B704780B483B000AF78607B6893F84B
:109390009C32DBB2042B06D17B6893F89D32DAB2A3
:1093A0007B6883F89C22002318460C37BD465DF885
:1093B000047B704780B582B000AF78607B68D3F8DB
:1093C000B832002B01D1032312E07B6893F89C3262
:1093D000DBB2032B0BD17B68D3F8B832DB69002BEF
:1093E00005D07B68D3F8B832DB69786898470023EA
:1093F00018460837BD4680BD80B487B000AF78609E
:109400007B687B617B691B787B827B6901337B6135
:109410007B691B783B82B7F910301B021AB2B7F98F
:10942000123013431BB2FB81FB8918461C37BD4623
:109430005DF8047B7047000080B584B000AF7860B1
:1094400039600023FB733B681B7803F06003402BFB
:1094500005D0402B53D8002B0BD0202B4FD17B684D
:10946000D3F8B8329B683968786898470346FB732D
:109470004AE03B685B78092B3BD801A252F823F005
:10948000D5940008E9940008F3940008DF940008DC
:10949000F3940008B3940008A9940008F39400081A
:1094A000CB940008BD9400083968786800F0DEF9B4
:1094B00024E03968786800F06DFB1FE0396878684F
:1094C00000F0ACFB0346FB7318E03968786800F0E5
:1094D0004BFC13E03968786800F07CFC0EE03968DA
:1094E000786800F0ABFC09E03968786800F0BAFCF5
:1094F00004E03968786800F011FD00BF04E03968C5
:10950000786800F00BFD00BFFB7B18461037BD46A6
:1095100080BD00BF80B584B000AF786039600023A3
:10952000FB733B681B7803F06003402B05D0402B96
:109530002FD8002B01D0202B2BD17B6893F89C32A5
:10954000DBB2013B022B1DD83B689B88DBB2012BB1
:1095500013D87B68D3F8B8329B6839687868984725
:109560000346FB733B68DB88002B10D1FB7B002B91
:109570000DD1786800F09DFD09E03968786800F049
:10958000CDFC04E03968786800F0C8FC00E000BF5A
:1095900004E03968786800F0C1FC00BFFB7B184626
:1095A0001037BD4680BD80B584B000AF78603960AB
:1095B0000023FB733B689B88BB733B681B7803F0FD
:1095C0006003402B07D0402B00F24581002B0CD0CC
:1095D000202B40F040817B68D3F8B8329B68396813
:1095E000786898470346FB733AE13B685B78032B46
:1095F00007D0032B00F32981002B7FD0012B3CD017
:1096000023E17B6893F89C32DBB2022B02D0032B60
:1096100016D02CE0BB7B002B0DD0BB7B802B0AD05F
:10962000BB7B1946786801F05BFD8021786801F00A
:1096300057FD00BF20E03968786800F06FFC1BE040
:109640003B685B88002B0ED1BB7B002B0BD0BB7B18
:10965000802B08D03B68DB88002B04D1BB7B1946EC
:10966000786801F03DFD786800F023FD04E039687A
:10967000786800F053FC00BFECE07B6893F89C3204
:10968000DBB2022B02D0032B16D030E0BB7B002BC9
:109690000DD0BB7B802B0AD0BB7B1946786801F0CC
:1096A0001FFD8021786801F01BFD00BF25E03968AF
:1096B000786800F033FC20E03B685B88002B1BD10E
:1096C000BB7B03F07F03002B04D0BB7B194678687B
:1096D00001F025FD786800F0ECFC7B68D3F8B83227
:1096E0009B683968786898470346FB7304E03968DB
:1096F000786800F013FC00E000BFABE07B6893F8F3
:109700009C32DBB2022B02D0032B32D097E0BB7B22
:10971000002B07D0BB7B802B04D03968786800F021
:10972000FDFB91E097F90E30002B0BDABB7B03F0C9
:109730007F0213469B0013449B0010337A68134446
:1097400004330BE0BB7B03F07F0213469B00134402
:109750009B0003F5A8737A6813440433BB60BB68AD
:1097600000221A60BB6802221946786800F047FCA4
:109770006AE097F90E30002B11DABB7B03F00F0281
:10978000796813469B0013449B000B4424331B88C9
:10979000002B17D13968786800F0C0FB54E0BB7B20
:1097A00003F00F02796813469B0013449B000B449F
:1097B00003F5B2731B88002B04D13968786800F078
:1097C000ADFB41E097F90E30002B0BDABB7B03F0C9
:1097D0007F0213469B0013449B0010337A681344A6
:1097E00004330BE0BB7B03F07F0213469B00134462
:1097F0009B0003F5A8737A6813440433BB60BB7BFA
:10980000002B02D0BB7B802B03D1BB6800221A60E7
:109810000EE0BB7B1946786801F0A0FC0346002BE4
:1098200003D0BB6801221A6002E0BB6800221A6004
:10983000BB6802221946786800F0E1FB04E0396851
:10984000786800F06BFB00BF04E03968786800F0CE
:1098500065FB00BF04E03968786800F05FFB00BF7B
:10986000FB7B18461037BD4680BD000080B584B034
:1098700000AF7860396000233B810023FB60002348
:10988000FB723B685B881B0A9BB2013B0E2B00F20C
:10989000528101A252F823F0099900082199000889
:1098A00061990008379B0008379B0008D79A000889
:1098B000039B0008379B0008379B0008379B000874
:1098C000379B0008379B0008379B0008379B000830
:1098D000D59800087B68D3F8B432DB69002B0BD035
:1098E0007B68D3F8B432DB697A68127C07F108012F
:1098F00010469847F86026E13968786800F00EFB5A
:10990000FB7A0133FB721EE17B68D3F8B4321B682B
:109910007A68127C07F1080110469847F86012E156
:109920007B681B7C002B0DD17B68D3F8B8329B6A17
:1099300007F1080210469847F860FB6801330222DD
:109940001A7000E17B68D3F8B832DB6A07F10802CD
:1099500010469847F860FB68013302221A70F2E063
:109960003B685B88DBB2052B00F2AC8001A252F8A9
:1099700023F000BF8D990008C1990008F5990008EF
:10998000299A00085D9A0008919A00087B68D3F82C
:10999000B4325B68002B0BD07B68D3F8B4325B68C1
:1099A0007A68127C07F1080110469847F86091E048
:1099B0003968786800F0B2FAFB7A0133FB7289E00B
:1099C0007B68D3F8B4329B68002B0BD07B68D3F84C
:1099D000B4329B687A68127C07F1080110469847F8
:1099E000F86077E03968786800F098FAFB7A01331C
:1099F000FB726FE07B68D3F8B432DB68002B0BD0CE
:109A00007B68D3F8B432DB687A68127C07F108010E
:109A100010469847F8605DE03968786800F07EFA93
:109A2000FB7A0133FB7255E07B68D3F8B4321B69D3
:109A3000002B0BD07B68D3F8B4321B697A68127C98
:109A400007F1080110469847F86043E039687868E4
:109A500000F064FAFB7A0133FB723BE07B68D3F8D9
:109A6000B4325B69002B0BD07B68D3F8B4325B69EE
:109A70007A68127C07F1080110469847F86029E0DF
:109A80003968786800F04AFAFB7A0133FB7221E00A
:109A90007B68D3F8B4329B69002B0BD07B68D3F87A
:109AA000B4329B697A68127C07F108011046984726
:109AB000F8600FE03968786800F030FAFB7A01331B
:109AC000FB7207E03968786800F028FAFB7A013306
:109AD000FB7200BF37E07B681B7C002B09D17B68E1
:109AE000D3F8B8325B6B07F1080210469847F8606C
:109AF00029E03968786800F011FAFB7A0133FB72CB
:109B000021E07B681B7C002B0DD17B68D3F8B83239
:109B10001B6B07F1080210469847F860FB68013399
:109B200007221A700FE03968786800F0F7F9FB7ABD
:109B30000133FB7207E03968786800F0EFF9FB7ACF
:109B40000133FB7200BFFB7A002B1ED13B68DB8820
:109B5000002B16D03B89002B0ED03B68DA883B895E
:109B6000934228BF13469BB23B813B891A46F96852
:109B7000786800F044FA09E03968786800F0CEF9B6
:109B800004E0786800F095FA00E000BF1037BD46A9
:109B900080BD00BF80B584B000AF786039603B689D
:109BA0009B88002B31D13B68DB88002B2DD13B6893
:109BB0005B887F2B29D83B685B88DBB203F07F038F
:109BC000FB737B6893F89C32DBB2032B04D13968BA
:109BD000786800F0A3F91DE07B68FA7B83F89E2289
:109BE000FB7B1946786801F0E5FA786800F061FAC5
:109BF000FB7B002B04D07B68022283F89C2209E0C7
:109C00007B68012283F89C2204E03968786800F0C0
:109C100085F900BF00BF1037BD4680BD80B584B058
:109C200000AF786039600023FB733B685B88DAB271
:109C30004C4B1A704B4B1B78012B05D9396878684F
:109C400000F06CF9032388E07B6893F89C32DBB268
:109C5000022B02D0032B25D071E0424B1B78002B46
:109C60001CD0404B1B781A467B685A603D4B1B78D2
:109C700019467868FFF790F90346FB73FB7B002BCE
:109C800004D03968786800F049F965E0786800F038
:109C900010FA7B68032283F89C225DE0786800F06C
:109CA00008FA59E02F4B1B78002B12D17B68022257
:109CB00083F89C222B4B1B781A467B685A60294BF1
:109CC0001B7819467868FFF783F9786800F0F1F996
:109CD00042E0244B1B781A467B685B689A422AD084
:109CE0007B685B68DBB219467868FFF771F91D4B3A
:109CF0001B781A467B685A601A4B1B78194678689D
:109D0000FFF74AF90346FB73FB7B002B0FD0396842
:109D1000786800F003F97B685B68DBB21946786805
:109D2000FFF756F97B68022283F89C2214E07868DA
:109D300000F0BFF910E0786800F0BBF90CE039687A
:109D4000786800F0EBF8074B1B7819467868FFF746
:109D50003FF90323FB7300BFFB7B18461037BD465A
:109D600080BD00BF7802002080B582B000AF78606F
:109D700039603B68DB88012B04D03968786800F0D3
:109D8000CDF823E07B6893F89C32DBB2022B02DC37
:109D9000002B03DC15E0032B0BD012E07B680022C4
:109DA0009A607B68083301221946786800F027F929
:109DB0000CE07B68043301221946786800F01FF933
:109DC00004E03968786800F0A9F800BF00BF0837E0
:109DD000BD4680BD80B582B000AF786039607B68D9
:109DE00093F89C32DBB2013B022B1ED83B68DB8828
:109DF000022B04D03968786800F090F81AE07B688C
:109E00000122DA607B68D3F8A432002B05D07B688E
:109E1000DB6843F002027B68DA607B680C33022265
:109E20001946786800F0EBF804E03968786800F0CB
:109E300075F800BF00BF0837BD4680BD80B582B051
:109E400000AF786039603B685B88012B06D17B6886
:109E50000122C3F8A422786800F02BF900BF08376C
:109E6000BD4680BD80B582B000AF786039607B6848
:109E700093F89C32DBB2013B022B0BD83B685B882A
:109E8000012B0CD17B680022C3F8A422786800F073
:109E900010F904E03968786800F040F800E000BF8D
:109EA00000BF0837BD4680BD80B584B000AF786084
:109EB00039603B68FB60FB681A787B681A70FB6846
:109EC0000133FB60FB681A787B685A70FB680133CA
:109ED000FB60F868FFF790FA03461A467B685A80E1
:109EE000FB680133FB60FB680133FB60F868FFF738
:109EF00083FA03461A467B689A80FB680133FB604D
:109F0000FB680133FB60F868FFF776FA03461A46F0
:109F10007B68DA8000BF1037BD4680BD80B582B057
:109F200000AF786039608021786801F0D9F80021AD
:109F3000786801F0D5F800BF0837BD4680BD80B510
:109F400086B000AFF860B9607A600023FB75FB68EB
:109F5000002B36D0FB683B61386900F036F80346C9
:109F600001339BB25B009AB27B681A80FB7DBA68B2
:109F700013447A6812781A70FB7D0133FB75FB7D00
:109F8000BA68134403221A70FB7D0133FB7513E09A
:109F9000FB7DBA6813443A6912781A703B69013341
:109FA0003B61FB7D0133FB75FB7DBA6813440022E6
:109FB0001A70FB7D0133FB753B691B78002BE7D1E1
:109FC00000E000BF1837BD4680BD80B485B000AF4B
:109FD00078600023FB737B68BB6005E0FB7B01338B
:109FE000FB73BB680133BB60BB681B78002BF5D1EA
:109FF000FB7B18461437BD465DF8047B704780B57F
:10A0000084B000AFF860B9607A60FB680222C3F8E0
:10A010009422FB687A689A61FB687A68DA617B68E7
:10A02000BA680021F86801F0E4F8002318461037F8
:10A03000BD4680BD80B584B000AFF860B9607A607D
:10A040007B68BA680021F86801F0D3F8002318464D
:10A050001037BD4680BD80B584B000AFF860B960F0
:10A060007A60FB680322C3F89422FB687A68C3F81D
:10A070005821FB687A68C3F85C217B68BA680021C4
:10A08000F86801F0D7F8002318461037BD4680BDA8
:10A0900080B584B000AFF860B9607A607B68BA6858
:10A0A0000021F86801F0C6F8002318461037BD46B5
:10A0B00080BD80B582B000AF78607B680422C3F8B1
:10A0C0009422002300220021786801F092F80023F6
:10A0D00018460837BD4680BD80B582B000AF7860B5
:10A0E0007B680522C3F894220023002200217868AF
:10A0F00001F0A0F8002318460837BD4680BD80B5A2
:10A1000084B000AF78600B46FB704FF4077001F02D
:10A11000FBF8F860FB68002B05D17B680022C3F8D0
:10A12000BC22022366E07B68FA68C3F8BC227B6825
:10A130001B7C002B19D14FF4007302228121786817
:10A1400000F089FF7B6801221A874FF40073022216
:10A150000121786800F07FFF7B680122A3F8782155
:10A160007B681022A3F84E2016E0402302228121B2
:10A17000786800F070FF7B6801221A874023022272
:10A180000121786800F067FF7B680122A3F878213D
:10A190007B681022A3F84E200823032282217868CE
:10A1A00000F059FF7B680122A3F84C207B68D3F8AC
:10A1B000C0321B689847FB680022C3F81422FB6872
:10A1C0000022C3F818227B681B7C002B09D1FB6896
:10A1D000D3F804224FF400730121786801F02AF8C3
:10A1E00007E0FB68D3F8042240230121786801F0DE
:10A1F00021F8002318461037BD4680BD80B582B0D7
:10A2000000AF78600B46FB708121786800F049FF51
:10A210007B6800221A870121786800F042FF7B6882
:10A220000022A3F878218221786800F03AFF7B6849
:10A230000022A3F84C207B680022A3F84E207B6804
:10A24000D3F8BC32002B0ED07B68D3F8C0325B68E9
:10A2500098477B68D3F8BC32184601F063F87B68F6
:10A260000022C3F8BC22002318460837BD4680BD33
:10A2700080B586B000AF786039607B68D3F8BC32B7
:10A280003B6100237B7300237B810023FB753B69CB
:10A29000002B01D10323AFE03B681B7803F0600380
:10A2A000002B3FD0202B40F09F803B68DB88002BA9
:10A2B0002ED03B681B785BB2002B16DA7B68D3F894
:10A2C000C0329B683A68507839693A68D2889847B2
:10A2D0003B68DB88072B28BF0723FB813B69FA8992
:10A2E00019467868FFF78BFE85E03B685A783B6932
:10A2F00083F800223B68DB88DAB23B6983F80122ED
:10A3000039693B68DB881A467868FFF7A4FE72E07B
:10A310007B68D3F8C0329B683A685078002239686D
:10A32000984768E03B685B780B2B52D801A252F843
:10A3300023F000BF65A30008E1A30008D3A3000831
:10A34000D3A30008D3A30008D3A30008D3A3000815
:10A35000D3A30008D3A30008D3A300088FA3000849
:10A36000B9A300087B6893F89C32DBB2032B07D1BA
:10A3700007F10A03022219467868FFF740FE32E02F
:10A3800039687868FFF7CAFD0323FB752BE07B680B
:10A3900093F89C32DBB2032B07D107F10D030122A6
:10A3A00019467868FFF72BFE1DE039687868FFF7DB
:10A3B000B5FD0323FB7516E07B6893F89C32DBB296
:10A3C000032B0FD039687868FFF7A8FD0323FB75CE
:10A3D00008E039687868FFF7A1FD0323FB7502E008
:10A3E00000BF08E000BF06E039687868FFF796FD17
:10A3F0000323FB7500BFFB7D18461837BD4680BDA3
:10A4000080B584B000AF78600B46FB707B68D3F8F2
:10A41000C432FB607B68D3F8BC32002B01D103232C
:10A420004FE07B68D3F8BC32BB60FA78796813469A
:10A430009B0013449B000B4418331B68002B29D04E
:10A44000FA78796813469B0013449B000B44183339
:10A450001A68F978F8680B469B000B44DB0003444C
:10A4600020331B68B2FBF3F101FB03F3D31A002B7B
:10A4700010D1FA78796813469B0013449B000B4473
:10A48000183300221A60F97800230022786800F05F
:10A49000B0FE15E0BB680022C3F814227B68D3F835
:10A4A000C0321B69002B0BD07B68D3F8C0321B690C
:10A4B000BA68D2F80802BA6802F50471FA789847C7
:10A4C000002318461037BD4680BD80B584B000AF6C
:10A4D00078600B46FB707B68D3F8BC32FB607B680E
:10A4E000D3F8BC32002B01D1032315E0FB781946C9
:10A4F000786800F0C0FE0246FB68C3F80C227B6857
:10A50000D3F8C032DB68FA68D2F80402FA6802F5C0
:10A51000037211469847002318461037BD4680BD88
:10A5200080B584B000AF78607B68D3F8BC32FB6044
:10A53000FB68002B01D103231AE07B68D3F8C032FB
:10A54000002B14D0FB6893F80032FF2B0FD07B68F0
:10A55000D3F8C0329B68FA6892F80002F968FA688A
:10A5600092F801229847FB68FF2283F8002200231B
:10A5700018461037BD4680BD80B483B000AF786008
:10A580007B6843221A80034B18460C37BD465DF8A2
:10A59000047B7047B400002080B483B000AF7860C3
:10A5A0007B6843221A80034B18460C37BD465DF882
:10A5B000047B70477000002080B483B000AF7860E7
:10A5C0007B6843221A80034B18460C37BD465DF862
:10A5D000047B7047F800002080B483B000AF78603F
:10A5E0007B680A221A80034B18460C37BD465DF87B
:10A5F000047B70472C00002080B483B000AF7860EB
:10A6000039603B68002B01D1032304E07B683A6882
:10A61000C3F8C022002318460C37BD465DF8047B02
:10A62000704780B487B000AFF860B9607A60FB68AB
:10A63000D3F8BC327B617B69002B01D1032308E096
:10A640007B69BA68C3F808227B697A68C3F810226C
:10A65000002318461C37BD465DF8047B704780B464
:10A6600085B000AF786039607B68D3F8BC32FB609E
:10A67000FB68002B01D1032304E0FB683A68C3F8B0
:10A680000422002318461437BD465DF8047B70474A
:10A6900080B584B000AF78607B68D3F8BC32BB6013
:10A6A0000123FB737B68D3F8BC32002B01D1032359
:10A6B0001AE0BB68D3F81432002B14D1BB68012216
:10A6C000C3F81422BB68D3F810227B68DA62BB6837
:10A6D000D3F80822BB68D3F810328121786800F0E3
:10A6E00088FD0023FB73FB7B18461037BD4680BDF9
:10A6F00080B584B000AF78607B68D3F8BC32FB6073
:10A700007B68D3F8BC32002B01D103232AE07B689D
:10A710001B7C002B09D1FB68D3F804224FF4007393
:10A720000121786800F086FD07E0FB68D3F8042279
:10A7300040230121786800F07DFDFB68D3F80422F6
:10A74000FB68D3F80C321946104602F0AFFAFB68EA
:10A75000D3F80402FB68D3F80C321A46002107F044
:10A7600019FE002318461037BD4680BD80B500AFE6
:10A7700003F01CF9002212491248FEF76BFB034656
:10A78000002B01D001F09EF80F490E48FEF7C6FBE2
:10A790000346002B01D001F095F80C490948FFF75A
:10A7A0002BFF0346002B01D001F08CF80548FEF783
:10A7B000DCFB0346002B01D001F084F800BF80BD14
:10A7C0003C0100207C02002038000020AC01002069
:10A7D00080B483B000AF03463960FB713B6812223E
:10A7E0001A80034B18460C37BD465DF8047B704752
:10A7F0005C01002080B483B000AF03463960FB7178
:10A800003B6804221A80034B18460C37BD465DF89E
:10A81000047B70477001002080B582B000AF034612
:10A820003960FB71FB79002B05D13A68074908486C
:10A83000FFF785FB04E03A6804490548FFF77FFB12
:10A84000024B18460837BD4680BD00BF4C050020AE
:10A850008835010880B582B000AF03463960FB71CE
:10A860003A6804490448FFF76AFB024B1846083768
:10A87000BD4680BD4C050020A035010880B582B0E2
:10A8800000AF03463960FB713B6836221A8000F046
:10A8900043F8024B18460837BD4680BD74010020BE
:10A8A00080B582B000AF03463960FB71FB79002BA5
:10A8B00005D13A6807490848FFF741FB04E03A68C8
:10A8C00004490548FFF73BFB024B18460837BD46D5
:10A8D00080BD00BF4C050020B435010880B582B0B2
:10A8E00000AF03463960FB71FB79002B05D13A6854
:10A8F00007490848FFF723FB04E03A680449054884
:10A90000FFF71DFB024B18460837BD4680BD00BF50
:10A910004C050020C035010880B584B000AF1C4B49
:10A92000FB601C4B1B68BB601B4B1B687B601B4B9D
:10A930001B683B600822F968B86800F031F8FB68D2
:10A940001033FB60FB682D221A70FB680133002274
:10A950001A70FB680233FB600822F968786800F01F
:10A960001FF8FB681033FB60FB682D221A70FB6830
:10A97000013300221A70FB680233FB600822F96879
:10A98000386800F00DF800BF1037BD4680BD00BF2D
:10A99000760100209075FF1F9475FF1F9875FF1FAB
:10A9A00080B487B000AFF860B9601346FB71002334
:10A9B000FB750023FB7527E0FB681B0F092B0BD8E9
:10A9C000FB681B0FDAB2FB7D5B001946BB680B44CA
:10A9D0003032D2B21A700AE0FB681B0FDAB2FB7D8C
:10A9E0005B001946BB680B443732D2B21A70FB6861
:10A9F0001B01FB60FB7D5B000133BA68134400223E
:10AA00001A70FB7D0133FB75FA7DFB799A42D3D333
:10AA100000BF00BF1C37BD465DF8047B70470000D7
:10AA200080B500AF002205490548FFF7FAFD05494A
:10AA30000348FFF714FE0023184680BDA033002012
:10AA40007C020020A02F002080B400AF0023184615
:10AA5000BD465DF8047B704780B483B000AF034609
:10AA60003960FB711346BB80FB79232B4AD801A2C6
:10AA700052F823F005AB000805AB000805AB000851
:10AA800005AB000805AB000805AB000805AB0008E6
:10AA900005AB000805AB000805AB000805AB0008D6
:10AAA00005AB000805AB000805AB000805AB0008C6
:10AAB00005AB000805AB000805AB000805AB0008B6
:10AAC00005AB000805AB000805AB000805AB0008A6
:10AAD00005AB000805AB000805AB000805AB000896
:10AAE00005AB000805AB000805AB000805AB000886
:10AAF00005AB000805AB000805AB000805AB000876
:10AB000005AB000800BF002318460C37BD465DF8B2
:10AB1000047B704780B582B000AF78603960796897
:10AB20000548FFF79CFD0448FFF7E2FD00231846A7
:10AB30000837BD4680BD00BF7C02002080B584B0D0
:10AB400000AF78600B467B800023FB737B881A463E
:10AB50007968324807F0D5FC314B1B78DBB2002B0B
:10AB600014D02F4B00221A707B881A462B492D488F
:10AB7000FFF757FD2B48FFF78BFD0346002B02D153
:10AB80007B88DBB245E0264B01221A70264B1B78EE
:10AB9000DBB25A1C254B83FB0213D910D317C91AF9
:10ABA0000B469B000B449B00D11A0B46BB73204BFA
:10ABB0001B78DBB2BA7B9A4201D1012329E07B8862
:10ABC000B3F5007F28BF4FF400737B80164B1B78D2
:10ABD000DBB21A461346DB0113449B00154A1344AB
:10ABE0007A880E49184607F08CFC0F4B1B78DBB2B5
:10ABF00018467A880F490346DB0103449B000B4447
:10AC000003F500731A60084ABB7B13700023FB73C3
:10AC1000FB7B18461037BD4680BD00BFA037002023
:10AC2000AA0100207C0200209C2F00206766666637
:10AC30009D2F00204C07002080B586B000AFF86043
:10AC4000B9601346FB710023FB75244B1B78DAB205
:10AC5000234B1B78DBB29A4236D0204B1B78DBB2F9
:10AC60001A461346DB0113449B001E4A99181B4BDE
:10AC70001B78DBB218461B4A0346DB0103449B00EA
:10AC8000134403F500731B681A461748FFF7C9FC05
:10AC90001548FFF7FDFC0346002B13D10F4B1B7823
:10ACA000DBB25A1C114B83FB0213D910D317C91AFC
:10ACB0000B469B000B449B00D11ACAB2074B1A707B
:10ACC000002306E0012304E0094B01221A7097F9E2
:10ACD000173018461837BD4680BD00BF9D2F002095
:10ACE0009C2F00204C0700207C02002067666666CF
:10ACF000AA01002080B598B000AF786007F10C037E
:10AD000054220021184607F045FB7B681B68154A52
:10AD1000934223D14FF40053FB604FF00063BB64B8
:10AD200007F10C031846FAF7CBF80346002B01D0C5
:10AD300000F0C8FD0C4B9B6D0B4A43F40003936578
:10AD4000094B9B6D03F40003BB60BB68002200212C
:10AD50001420FBF756FB1420FBF76DFB00BF603798
:10AD6000BD4680BD005C00400010024080B582B04E
:10AD700000AF78607B681B68074A934208D1074B95
:10AD80009B6D064A23F4000393651420FBF761FBD7
:10AD900000BF0837BD4680BD005C00400010024087
:10ADA00080B582B000AF78607B68D3F8D8227B682A
:10ADB00003F5267319461046FEF722F900BF08373F
:10ADC000BD4680BD80B582B000AF78600B46FB7099
:10ADD0007B68D3F8D802FA78796813469B0013444D
:10ADE000DB000B4403F5B2731A68FB781946FEF7D3
:10ADF0005CF900BF0837BD4680BD80B582B000AFAA
:10AE000078600B46FB707B68D3F8D802FA787968D3
:10AE100013469B001344DB000B4424331A68FB7871
:10AE20001946FEF7A5F900BF0837BD4680BD80B5BD
:10AE300082B000AF78607B68D3F8D8321846FEF74E
:10AE4000B9FA00BF0837BD4680BD80B584B000AFF9
:10AE500078600123FB737B685B79022B01D000F0E3
:10AE600031FD7B68D3F8D832FA7B11461846FEF7DD
:10AE700063FA7B68D3F8D8321846FEF70FFA00BFA2
:10AE80001037BD4680BD000080B582B000AF78604D
:10AE90007B68D3F8D8321846FEF75EFA7B685B7A97
:10AEA000002B05D0044B1B69034A43F006031361D2
:10AEB00000BF0837BD4680BD00ED00E080B582B020
:10AEC00000AF78607B685B7A002B07D0084B1B696A
:10AED000074A23F00603136100F02EFA7B68D3F8CB
:10AEE000D8321846FEF74EFA00BF0837BD4680BD7F
:10AEF00000ED00E080B582B000AF78602B4A7B683F
:10AF0000C2F8D8327B68294AC3F8C422274B284AA2
:10AF10001A60264B08221A71244B02225A71234BC5
:10AF20000222DA71214B00221A72204B00225A723F
:10AF30001E4B00229A721D4B0022DA721B48F5F755
:10AF400009FE0346002B01D000F0BCFC7B68D3F85F
:10AF5000C402182300220021F7F7D5FA7B68D3F842
:10AF6000C402582300228021F7F7CDFA7B68D3F87A
:10AF7000C402C02300228121F7F7C5FA7B68D3F809
:10AF8000C4024FF4887300220121F7F7BCFA7B68F2
:10AF9000D3F8C4024FF4807300228221F7F7B3FA8A
:10AFA000002318460837BD4680BD00BFA0470020DB
:10AFB000005C004080B584B000AF78600023FB7374
:10AFC0000023BB737B68D3F8C4321846F5F790FEB4
:10AFD0000346FB73FB7B184600F0B4F90346BB73D2
:10AFE000BB7B18461037BD4680BD80B584B000AF2E
:10AFF00078600023FB730023BB737B68D3F8C432F3
:10B000001846F5F798FE0346FB73FB7B184600F0E5
:10B0100099F90346BB73BB7B18461037BD4680BD0C
:10B0200080B584B000AF78600023FB730023BB734E
:10B030007B68D3F8C4321846F5F79FFE0346FB73CE
:10B04000FB7B184600F07EF90346BB73BB7B1846BA
:10B050001037BD4680BD80B584B000AF786008462B
:10B0600011461A460346FB700B46BB7013463B80E5
:10B070000023FB730023BB737B68D3F8C402BB7847
:10B080003A88F978F5F7E6FF0346FB73FB7B184631
:10B0900000F058F90346BB73BB7B18461037BD461A
:10B0A00080BD80B584B000AF78600B46FB70002394
:10B0B000FB730023BB737B68D3F8C432FA78114664
:10B0C0001846F6F726F80346FB73FB7B184600F09C
:10B0D00039F90346BB73BB7B18461037BD4680BDAC
:10B0E00080B584B000AF78600B46FB700023FB7323
:10B0F0000023BB737B68D3F8C432FA781146184634
:10B10000F6F7CFF80346FB73FB7B184600F01AF9FD
:10B110000346BB73BB7B18461037BD4680BD80B568
:10B1200084B000AF78600B46FB700023FB730023F4
:10B13000BB737B68D3F8C432FA7811461846F6F729
:10B1400002F90346FB73FB7B184600F0FBF803464D
:10B15000BB73BB7B18461037BD4680BD80B485B03D
:10B1600000AF78600B46FB707B68D3F8C432FB609D
:10B1700097F90330002B0BDAFB7803F07F02F968B4
:10B1800013469B001344DB000B4412331B780BE087
:10B19000FB7803F07F02F96813469B001344DB0041
:10B1A0000B4403F5A9731B7818461437BD465DF8A8
:10B1B000047B704780B584B000AF78600B46FB70AD
:10B1C0000023FB730023BB737B68D3F8C432FA7887
:10B1D00011461846F5F71AFF0346FB73FB7B18462A
:10B1E00000F0B0F80346BB73BB7B18461037BD4672
:10B1F00080BD80B586B000AFF8607A603B600B46DA
:10B20000FB720023FB750023BB75FB68D3F8C402F7
:10B21000F97A3B687A68F6F70DF80346FB75FB7D13
:10B22000184600F08FF80346BB75BB7D18461837EB
:10B23000BD4680BD80B586B000AFF8607A603B60E7
:10B240000B46FB720023FB750023BB75FB68D3F82C
:10B25000C402F97A3B687A68F5F7A3FF0346FB75E9
:10B26000FB7D184600F06EF80346BB75BB7D1846A3
:10B270001837BD4680BD80B582B000AF78600B4600
:10B28000FB707B68D3F8C432FA7811461846F5F79C
:10B29000B9FF034618460837BD4680BD80B582B069
:10B2A00000AF78600B46FB70FB78002B02D0012BBF
:10B2B00013D023E07B685B7A002B07D000F03CF8CA
:10B2C000104B1B690F4A23F0060313617B68D3F808
:10B2D000D8321846FEF756F810E07B68D3F8D8321B
:10B2E0001846FEF739F87B685B7A002B05D0054BD2
:10B2F0001B69044A43F00603136100BF00BF08370F
:10B30000BD4680BD00ED00E080B483B000AF786042
:10B31000034B18460C37BD465DF8047B704700BFF1
:10B320007C4A002080B483B000AF786000BF0C3747
:10B33000BD465DF8047B704780B500AF00F08AF928
:10B3400000BF80BD80B485B000AF0346FB71002311
:10B35000FB73FB79032B17D801A252F823F000BF2F
:10B3600071B3000877B300087DB3000883B3000809
:10B370000023FB730BE00323FB7308E00123FB7343
:10B3800005E00323FB7302E00323FB7300BFFB7B99
:10B3900018461437BD465DF8047B704780B400AF93
:10B3A000BFF34F8F00BF064BDB6803F4E062044934
:10B3B000044B1343CB60BFF34F8F00BF00BFFDE7CB
:10B3C00000ED00E00400FA0580B594B000AFF8F796
:10B3D000CBFF3B4634220021184606F0DBFF00235A
:10B3E0007B603B461846FAF7FFF9BB6903F08063C0
:10B3F000002B04D1BB6903F00063002B29D100BFEF
:10B40000864B1B6903F48033002BF9D1FAF712F84D
:10B41000FAF74CF8814B1B6A804A23F08063136271
:10B420007E4B1B6A7D4A43F0006313627B4B5B6972
:10B430007A4A43F40033536100BF784B1B6903F42D
:10B440008033002BF9D1FAF773F8FAF755F8FAF7C9
:10B4500013F84FF000631B68FB64714B1B68BB64FF
:10B46000704B7B64704B3B64FB6CB3F1FF3F18D0B7
:10B47000BB6CB3F1FF3F14D0FB6CB3F1005F10D392
:10B48000FA6C7B6C9A420CD8BB6CB3F1006F08D39A
:10B49000BA6C3B6C9A4204D8BB6C03F00103002BDE
:10B4A00001D1012300E00023FB63FB6B002B0AD0DA
:10B4B0005E4B1B68002B03D15C4B01221A6005E038
:10B4C00000F0BEF902E0594B00221A60584B1B688D
:10B4D000BB63584B1B687B63554B00221A60554B6E
:10B4E00000221A60BB6B544A934205D17B6B534ACE
:10B4F000934201D100F0A4F9514B1B68514A934289
:10B5000008D04A4B1B68012B04D04D4B4D4A1A60A2
:10B51000FFF744FF4A4B00221A60F8F725FF3B462D
:10B5200034220021184606F035FF00237B603B469D
:10B530001846FAF759F9BB6903F08063002B04D170
:10B54000BB6903F00063002B29D100BF334B1B699B
:10B5500003F48033002BF9D1F9F76CFFF9F7A6FF5C
:10B560002E4B1B6A2D4A23F0806313622B4B1B6A00
:10B570002A4A43F000631362284B5B69274A43F46D
:10B580000033536100BF254B1B6903F48033002B4C
:10B59000F9D1F9F7CDFFF9F7AFFFF9F76DFF00F03B
:10B5A00059F800F0A1F900F003FA00F0B3FA00F046
:10B5B00033FBFFF7DBF800212348FCF78BFD042168
:10B5C0002148FCF787FD08211F48FCF783FD002276
:10B5D000FF21002000F088F81C4802F003FB03F074
:10B5E000B3FB0346002B03D003F034FB03F0ACFBAA
:10B5F00004F00AF8164B00221A7001F079F903469C
:10B60000002B06D000220021FF2000F06DF800F092
:10B6100059F901F037FA00BFFDE700BF00200240F2
:10B62000040000080000022000F00708F05F00207E
:10B63000F45F0020F85F002067452301EFCDAB8960
:10B64000EC5F00200100ADDE644D00209C4C00202A
:10B65000595E002080B594B000AF07F1180338227E
:10B660000021184606F096FE3B1D00221A605A6023
:10B670009A60DA601A614FF40070FAF70FFD012347
:10B68000BB614FF48033FB6102237B630323BB6305
:10B690000923FB636C233B6402237B640623BB64A6
:10B6A0000223FB6407F118031846F8F713FF03465B
:10B6B000002B01D000F006F90F237B600323BB6051
:10B6C0000023FB6000233B6100237B613B1D0421C1
:10B6D0001846F9F711FA0346002B01D000F0F2F8F2
:10B6E00000BF5037BD4680BDB0B584B000AF034643
:10B6F000FB710B46BB7113467B71414B1B68DB6AC8
:10B70000FB60BB791846F4F7BDFE3BA3D3E90023E9
:10B71000F5F74CF802460B464FF000003949F4F7B4
:10B7200063FD02460B4614461D46F868F4F79AFE80
:10B7300002460B4620462946F4F70EFF02460B460A
:10B740002F490C6810461946F5F718F9034663634C
:10B75000FB791846F4F796FE27A3D3E90023F5F703
:10B7600025F802460B464FF000002649F4F73CFD51
:10B7700002460B4614461D46F868F4F773FE02466F
:10B780000B4620462946F4F7E7FE02460B461C49C5
:10B790000C6810461946F5F7F1F80346A3637B7968
:10B7A0001846F4F76FFE14A3D3E90023F4F7FEFF65
:10B7B00002460B464FF000001249F4F715FD024611
:10B7C0000B4614461D46F868F4F74CFE02460B463D
:10B7D00020462946F4F7C0FE02460B4608490C688D
:10B7E00010461946F5F7CAF80346E36300BF103761
:10B7F000BD46B0BDAFF300800000000000E06F4028
:10B80000644D00200000F03F80B584B000AFF860C8
:10B81000B9607A6001F022FA034683F00103DBB2DB
:10B82000002B01D07B6806E07B689BB21946B868A4
:10B83000FFF784F97B6818461037BD4680BD0000CD
:10B8400080B582B000AF00BF1A4B1B6903F4803390
:10B85000002BF9D1F9F7EEFDF9F728FE154B1B6A1D
:10B86000144A43F080631362124B5B69114A43F43C
:10B870000033536100BF0F4B1B6903F48033002B6F
:10B88000F9D1F9F755FEF9F737FEF9F7F5FD0A4B4F
:10B8900001221A60094B1B687B60094B1B683B60E7
:10B8A0003B6883F3088800BF7B68984700BF083770
:10B8B000BD4680BD00200240000001400400FF1F83
:10B8C0000000FF1F80B500AF00220021FF20FFF71E
:10B8D0000BFF40F6B830F8F7B7FDFFF7B1FF72B6CF
:10B8E00000BF00BFFDE7000080B588B000AF07F1E2
:10B8F0000C0300221A605A609A60DA601A612A4BBF
:10B90000DB6C294A43F02003D364274BDB6C03F044
:10B910002003BB60BB68244BDB6C234A43F001036C
:10B92000D364214BDB6C03F001037B607B681E4B0F
:10B93000DB6C1D4A43F00203D3641B4BDB6C03F04A
:10B9400002033B603B6801224FF444714FF090408A
:10B95000FAF774FB4FF44473FB6001233B6100234F
:10B960007B610023BB6107F10C0319464FF0904047
:10B97000FAF7E2F94FF40043FB604FF488133B61A0
:10B9800000237B6107F10C0319460848FAF7D4F944
:10B99000002200212820FAF734FD2820FAF74BFD79
:10B9A00000BF2037BD4680BD0010024000040048A3
:10B9B00080B500AF1F4B204A1A601E4B00225A6010
:10B9C0001C4B00229A601B4B0022DA60194B0122AB
:10B9D0001A74184B00225A74164B00229A74154B95
:10B9E00001225A61134B10229A61124B7D22DA61B7
:10B9F000104B12221A620F4B01225A620D4B032286
:10BA00009A620C4B0E22DA620A4B03221A63094B2C
:10BA100001225A63074B01229A63064B0022DA6324
:10BA20000448FAF731FD0346002B01D0FFF74AFF27
:10BA300000BF80BD9C4C00200064004080B59EB0DB
:10BA400000AF786007F1640300221A605A609A60C0
:10BA5000DA601A6107F1100354220021184606F03B
:10BA600099FC7B681B68284A934248D14FF4805365
:10BA70003B614FF00073BB6407F110031846F9F700
:10BA80001FFA0346002B01D0FFF71CFF1F4B9B6DD5
:10BA90001E4A43F0007393651C4B9B6D03F00073CB
:10BAA000FB60FB68194BDB6C184A43F00203D3645C
:10BAB000164BDB6C03F00203BB60BB684FF44073B2
:10BAC0007B660223BB660023FB6600233B670923DA
:10BAD0007B6707F1640319460D48FAF72DF9002238
:10BAE00000211520FAF78DFC1520FAF7A4FC00229E
:10BAF00000211620FAF785FC1620FAF79CFC00BFFF
:10BB00007837BD4680BD00BF006400400010024091
:10BB10000004004880B500AF1B4B1C4A1A601A4B4A
:10BB20004FF482725A60184B00229A60164B4FF401
:10BB3000E062DA60144B02221A61134B01225A614F
:10BB4000114B4FF400729A610F4B3022DA610E4BA9
:10BB500000221A620C4B00225A620B4B00229A629E
:10BB6000094B0722DA62084B00221A63064B0022B7
:10BB70005A630548FBF722FB0346002B01D0FFF771
:10BB8000A1FE00BF80BD00BF004D0020003C004072
:10BB900080B58AB000AF786007F1140300221A6004
:10BBA0005A609A60DA601A617B681B68174A934290
:10BBB00027D1174B9B6D164A43F400439365144BF2
:10BBC0009B6D03F400433B613B69114BDB6C104AF6
:10BBD00043F00203D3640E4BDB6C03F00203FB6003
:10BBE000FB6838237B610223BB610023FB610023D8
:10BBF0003B6206237B6207F1140319460548FAF7F6
:10BC00009BF800BF2837BD4680BD00BF003C004008
:10BC1000001002400004004880B58AB000AF07F170
:10BC20001C0300221A605A609A603B4600221A6088
:10BC30005A609A60DA601A615A619A612C4B4FF02F
:10BC400080421A602A4B00225A60294B00229A60D7
:10BC5000274B284ADA60264B00221A61244B002227
:10BC60009A612348FCF7DEF90346002B01D0FFF769
:10BC700029FE0023FB6100237B6207F11C031946A8
:10BC80001B48FDF751F80346002B01D0FFF71AFEC1
:10BC900060233B6000237B600023BB6000233B618B
:10BCA0003B46002219461248FCF726FB0346002BB0
:10BCB00001D0FFF707FE3B46042219460C48FCF76B
:10BCC0001BFB0346002B01D0FFF7FCFD3B4608227F
:10BCD00019460748FCF710FB0346002B01D0FFF77D
:10BCE000F1FD034800F026F800BF2837BD4680BDAF
:10BCF000644D002005CA1F0080B485B000AF786095
:10BD00007B681B68B3F1804F0BD1094B9B6D084AD0
:10BD100043F001039365064B9B6D03F00103FB6049
:10BD2000FB6800BF1437BD465DF8047B704700BF59
:10BD30000010024080B588B000AF786007F10C03B6
:10BD400000221A605A609A60DA601A617B681B6888
:10BD5000B3F1804F1CD1104BDB6C0F4A43F0010351
:10BD6000D3640D4BDB6C03F00103BB60BB6807239E
:10BD7000FB6002233B6100237B610023BB61012345
:10BD8000FB6107F10C0319464FF09040F9F7D4FF1F
:10BD900000BF2037BD4680BD0010024080B400AF18
:10BDA00000BFFDE780B400AF00BFFDE780B400AF87
:10BDB00000BFFDE780B400AF00BFFDE780B400AF77
:10BDC00000BFFDE780B400AF00BFBD465DF8047B57
:10BDD000704780B400AF00BFBD465DF8047B70477C
:10BDE00080B400AF00BFBD465DF8047B704780B5EE
:10BDF00000AFF8F70BFB00BF80BD000080B500AFBF
:10BE00000248F4F7DCFF00BF80BD00BFA047002060
:10BE100080B500AF0248FAF757FF00BF80BD00BFF2
:10BE20009C4C002080B500AF0248FAF74DFF00BFE0
:10BE300080BD00BF9C4C002080B500AF4FF4004097
:10BE4000FAF714F900BF80BD80B582B000AF0F4B88
:10BE50001B6E0E4A43F0010313660C4B1B6E03F07E
:10BE600001037B607B68094B9B6D084A43F080535C
:10BE70009365064B9B6D03F080533B603B68FAF77C
:10BE8000B1F900BF0837BD4680BD00BF00100240B9
:10BE900080B586B000AF7860144A154BD31A7B6129
:10BEA0007B693B61134B1B68002B02D1114B124A7B
:10BEB0001A60104B1A687B6813443A699A4207D299
:10BEC00006F0F2FA03460C221A604FF0FF3309E045
:10BED000084B1B68FB60074B1A687B681344054AD4
:10BEE0001360FB6818461837BD4680BD000002206D
:10BEF00000040000B04D00200060002080B586B036
:10BF000000AFF860B9607A6000237B610AE0AFF3AC
:10BF100000800146BB685A1CBA60CAB21A707B69BD
:10BF200001337B617A697B689A42F0DB7B68184653
:10BF30001837BD4680BD80B483B000AF78604FF045
:10BF4000FF3318460C37BD465DF8047B704780B45C
:10BF500083B000AF786039603B684FF400525A609C
:10BF6000002318460C37BD465DF8047B704780B44B
:10BF700083B000AF7860012318460C37BD465DF8EA
:10BF8000047B704780B485B000AFF860B9607A6018
:10BF9000002318461437BD465DF8047B7047000047
:10BFA0000D488546F4F7C4FD0C480D490D4A0023A1
:10BFB00002E0D458C4500433C4188C42F9D30A4A5E
:10BFC0000A4C002301E013600432A242FBD306F0C6
:10BFD00071FAFFF7F9F9FEE70000022000000020E7
:10BFE000580200208CA1020858020020EC5F0020BB
:10BFF000FEE70000F0B482B000AF0146F9710D49D0
:10C00000D1E90001FC79C4F12006A4F1200520FA51
:10C0100004F201FA06F6324321FA05F52A4321FA21
:10C0200004F3134603F0010318460837BD46F0BC7D
:10C03000704700BFC001002080B584B000AF7860B9
:10C040000B46FB700023FB731AE0FB7B1846FFF7DF
:10C05000D1FF0346002B09D0FA7BFB7B5B0079689C
:10C060000B44144931F912201A8006E0FB7B5B0077
:10C070007A6813444FF6FF721A80FB7B0133FB731F
:10C08000FA7BFB789A42E0D3FB78BB7309E0BB7B79
:10C090005B007A6813444FF6FF721A80BB7B013352
:10C0A000BB73BB7B3F2BF2D9FB7818461037BD46DC
:10C0B00080BD00BFB44E002080B483B000AF034603
:10C0C000FB71FB79052B08D0FB79062B05D0FB799A
:10C0D000092B02D0FB790C2B01D1012300E00023B6
:10C0E000DBB218460C37BD465DF8047B704780B460
:10C0F00083B000AF78607B68B3F57A6F02DD6FF0D4
:10C10000010306E07B68002B01DA002301E07B6875
:10C110001BB218460C37BD465DF8047B7047000023
:10C1200090B58BB000AF7860684B1B78402B28BF70
:10C130004023FB77002387F82730BCE097F82730AF
:10C14000BB6197F827307A68134493F80431FB7584
:10C150007A68BB69134403F284431B78BB75FB7D8B
:10C16000002B08D0BB7D1846FFF7A6FF0346002B27
:10C1700001D0012300E000237B757B7D002B2ED1B5
:10C1800097F82730524AD35C002B20D097F82730FD
:10C19000504AD35C0E2B08D897F827304D4AD25C12
:10C1A0000132D1B24B4AD15480E097F82730494A46
:10C1B0000F21D15497F82730454A0021D15497F8E0
:10C1C0002730454A4FF6FE7122F813106EE097F8BB
:10C1D0002730414A4FF6FE7122F8131066E097F8B7
:10C1E00027303C4A0021D1547A68BB6903F5F073CB
:10C1F0005B001344B3F904303B6297F82730344AAC
:10C20000D35C002B15D197F8273034493A6A41F8AE
:10C21000232097F827302E4A0121D15497F8274040
:10C22000386AFFF764FF03461A462B4B23F81420A5
:10C230003CE097F82730294A52F823303B613A6AAC
:10C240003B69D31AFB60FB68254A934205DD3B69D5
:10C2500003F5742303F23F233B62FB68214A9342B8
:10C2600005DA3B69A3F57423A3F23F233B623A6AE4
:10C270003B69D31AFB601C4B1B781A46FB6802FB18
:10C2800003F380331B123A6913443B6197F827305C
:10C2900012493A6941F8232097F827403869FFF797
:10C2A00026FF03461A460C4B23F8142097F8273034
:10C2B000013387F8273097F82720FB7F9A42FFF455
:10C2C0003DAF00BF00BF2C37BD4690BDC801002068
:10C2D000344F0020744F0020B44E0020B44D002095
:10C2E0003F420F00C1BDF0FFCA01002080B5ADF68E
:10C2F000D80D00AF07F6D803A3F6D4031860B04BEF
:10C300001B7887F8D13897F8D12807F61C03114617
:10C310001846FFF791FE07F57573C7F8D43807F68E
:10C32000D803A3F20C5345F6A5221A8007F6D803CA
:10C33000A3F20C5301221A71A24B9B789B10DBB223
:10C3400003F01F03DAB207F6D803A3F20C535A71B5
:10C3500007F6D803A3F20C5397F8D1289A7101235A
:10C3600087F8D33897F8D1385B00C7F8CC3807F690
:10C37000D803A3F20C5300225A80D7F8D42807F62A
:10C38000D803A3F20C5303CB10605160D7F8D43814
:10C390000833C7F8D43807F61C03D7F8CC28194659
:10C3A000D7F8D40806F0ADF8D7F8D428D7F8CC38A9
:10C3B0001344C7F8D438844B1B78002B00F0D48189
:10C3C000002387F8D23832E197F8D2381846FFF7C1
:10C3D00011FE0346002B3DD197F8D22807F6D8036B
:10C3E000A3F60C034FF6FF7123F8121097F8D2282A
:10C3F00007F6D803A3F28C73002123F8121097F8E4
:10C40000D22807F6D803A3F20C73002143F82210B8
:10C4100097F8D22807F6D803A3F20C63002143F85B
:10C42000221097F8D23807F6D802A2F6CC020021E3
:10C43000D15497F8D23807F6D802A2F68C02FF2121
:10C44000D15497F8D23807F6D802A2F64C02002150
:10C45000D154E7E097F8D238C7F8AC3897F8D2381B
:10C4600007F6D802A2F6D4021268134493F80431F6
:10C4700087F8AB3897F8D23807F6D802A2F64C0204
:10C4800097F8AB18D15497F8D23897F8D22807F616
:10C49000D801A1F6D40109689B000B44596807F63E
:10C4A000D803A3F20C7343F8221097F8AB38002B93
:10C4B00000F08C8007F6D803A3F6D4031A68D7F8E7
:10C4C000AC38134403F284431B781846FFF7F4FD9D
:10C4D0000346002B7AD007F6D803A3F6D4031A68D4
:10C4E000D7F8AC3803F5F0735B001344B3F90430AC
:10C4F000C7F8A438D7F8A438B3F57A6F09DCD7F8B1
:10C50000A438002B03DBD7F8A4381BB203E00023C8
:10C5100001E06FF0010397F8D21807F6D802A2F6EF
:10C520000C0222F8113097F8D22807F6D803A3F6A8
:10C53000D4031968D7F8AC3803F5D0735B000B440B
:10C54000998807F6D803A3F28C7323F8121097F892
:10C55000D22807F6D803A3F6D4031968D7F8AC3865
:10C5600090339B000B44596807F6D803A3F20C6381
:10C5700043F8221097F8D23807F6D802A2F6D40270
:10C580001168D7F8AC280A4402F28442117807F601
:10C59000D802A2F68C02D15497F8D23807F6D80206
:10C5A000A2F6D4021168D7F8AC280A4402F2444239
:10C5B000117807F6D802A2F6CC02D15432E000BFBF
:10C5C000C8010020BC4F0020CC01002097F8D228E1
:10C5D00007F6D803A3F60C034FF6FE7123F81210EA
:10C5E00097F8D22807F6D803A3F28C73002123F81A
:10C5F000121097F8D22807F6D803A3F20C63002193
:10C6000043F8221097F8D23807F6D802A2F68C0227
:10C61000FF21D15497F8D23807F6D802A2F6CC02FF
:10C620000021D15497F8D238013387F8D23897F8DF
:10C63000D22897F8D1389A42FFF4C6AE97F8D1388D
:10C640005B00C7F8C83897F8D1385B00C7F8C43822
:10C6500097F8D1389B00C7F8C03897F8D1389B00BD
:10C66000C7F8BC3897F8D138C7F8B83897F8D13838
:10C67000C7F8B43897F8D138C7F8B03897F8D33836
:10C6800063F0010387F8D33807F1CC03D7F8C82843
:10C690001946D7F8D40805F034FFD7F8D428D7F8CE
:10C6A000C8381344C7F8D43807F5A673D7F8C42898
:10C6B0001946D7F8D40805F024FFD7F8D428D7F8BE
:10C6C000C4381344C7F8D43807F5E673D7F8C02840
:10C6D0001946D7F8D40805F014FFD7F8D428D7F8AE
:10C6E000C0381344C7F8D43807F53373D7F8BC28DB
:10C6F0001946D7F8D40805F004FFD7F8D428D7F89E
:10C70000BC381344C7F8D43807F10C03D7F8B8285D
:10C710001946D7F8D40805F0F4FED7F8D428D7F88E
:10C72000B8381344C7F8D43807F14C03D7F8B42805
:10C730001946D7F8D40805F0E4FED7F8D428D7F87E
:10C74000B4381344C7F8D43807F18C03D7F8B028AD
:10C750001946D7F8D40805F0D4FED7F8D428D7F86E
:10C76000B0381344C7F8D4380423A7F8A23807F523
:10C770007573D7F8D428D31A9BB2083BA7F8A03812
:10C7800007F5757397F8D328DA7107F57573B7F85D
:10C79000A218B7F8A0280A4492B25A8007F5757318
:10C7A000D7F8D428D31AC7F89C38D7F89C389AB24F
:10C7B00007F575731146184600F05CFA00BF07F6DE
:10C7C000D807BD4680BD00BF80B5ADF6980D02AF5D
:10C7D00007F50963A3F68C0318603E4B1B7887F8B6
:10C7E0008A3897F88A2807F6080311461846FFF793
:10C7F00023FC0023C7F88C38D7F88C3807F10802DF
:10C80000D018D7F88C38C3F50061334B9B789B1058
:10C8100003F01F0297F88A38009313462F4A05F059
:10C82000ADFC0246D7F88C381344C7F88C38002387
:10C8300087F88B3827E0D7F88C3807F10802D01832
:10C84000D7F88C38C3F5006197F88B38002B01D1ED
:10C85000234A00E0234A97F88B385B0003F509630D
:10C860003B4433F9883C009313461F4A05F086FC8D
:10C870000246D7F88C381344C7F88C3897F88B38B1
:10C88000013387F88B3897F88B2897F88A389A42C3
:10C89000D1D3D7F88C3807F10802D018D7F88C38E4
:10C8A000C3F50063114A194605F068FC0246D7F843
:10C8B0008C381344C7F88C38D7F88C389AB207F103
:10C8C00008031146184600F0D5F900BF07F50967BF
:10C8D000BD4680BDC8010020BC4F0020D0350108F6
:10C8E00004360108083601080C3601081436010820
:10C8F00080B584B000AF0023FB720023FB700023DF
:10C900007B60FB1C19464F4803F052FD03467B60D9
:10C910007B68002B02D1FB78002B05D14A4805F03B
:10C9200025FC4FF0FF3388E0464803F08FFD0346B7
:10C930007B607B68002B05D0444805F017FC6FF046
:10C9400001037AE04FF480720021414805F022FD96
:10C95000402200213F4805F01DFD402200213E48B5
:10C9600005F018FD0023FB6008E03C4AFB684FF629
:10C97000FE7122F81310FB680133FB60FB683F2B4C
:10C98000F3DD374B1B7819462E4804F01EFE034694
:10C990007B607B68002B05D0324805F0E7FB6FF029
:10C9A00002034AE0304B1B781946264804F0E1FEAA
:10C9B00003467B607B68002B05D02C4805F0D6FB36
:10C9C0006FF0020339E001211E4804F057FF0346CF
:10C9D0007B607B68002B05D0254805F0C7FB6FF016
:10C9E00002032AE00221174804F01CFF03467B6083
:10C9F0007B68002B05D01F4805F0B8FB6FF00203E1
:10CA00001BE0104804F04EF903467B607B68002B66
:10CA100005D0194805F0AAFB6FF003030DE0174B92
:10CA200001221A700E4B1B7819460F4B1B781A46C1
:10CA3000134805F033FB97F90B3018461037BD4605
:10CA400080BD00BFBC4F00201C36010830360108F5
:10CA5000B44D0020344F0020744F0020B44E00200D
:10CA6000C801002044360108C901002058360108D9
:10CA70006C3601087C36010894360108705A002093
:10CA8000A836010880B500AF00F02EF800F036F9A6
:10CA900000BFF9E780B584B000AF78600E4B1B781B
:10CAA000402B28BF4023FB730C4B9B789B10DBB2C1
:10CAB00003F01F03BB730A4ABB7B1370FB7B194651
:10CAC0000848FFF7B9FA03467B73054A7B7B53702E
:10CAD00000BF1037BD4680BDC8010020BC4F0020FC
:10CAE000745A0020765A002090B5ADF2DC5D1EAF7E
:10CAF000394B1B78002B66D0384B1B68002B64D059
:10CB0000364B00221A603B1D1946354804F030FBB5
:10CB10000346C7F85C35D7F85C35002B57D13B1D71
:10CB20001846FFF7FDFA3B1D1846FFF7B3FFF7F76E
:10CB30007FFCC7F858052B4B9B68002B07DD294B62
:10CB40009B681A464FF47A73B3FBF2F301E04FF09F
:10CB5000FF33C7F85435244B1B68D7F85825D31A30
:10CB6000D7F854259A4233D81F4AD7F8583513605E
:10CB70001E4B1B78002B0CD01D4C684604F1100393
:10CB80007222194605F0BDFC94E80F0001F072FB1B
:10CB90000BE0174C684604F110037222194605F0A9
:10CBA000B0FC94E80F0001F0E5FC0E4B5B68002B35
:10CBB00004D13B1D1846FFF799FB09E03B1D1846C1
:10CBC000FFF702FE04E000BF02E000BF00E000BF8C
:10CBD00007F26457BD4690BD705A00206C5A002081
:10CBE000BC4F0020CC010020B44F0020595E002033
:10CBF000745A002080B400AF044B1B680133034A11
:10CC0000136000BFBD465DF8047B70476C5A00207E
:10CC100080B582B000AF0346FB80FB88B3F5004FC0
:10CC200001D1FFF7E7FF00BF0837BD4680BD000018
:10CC300080B400AFBFF34F8F00BF064BDB6803F437
:10CC4000E0620449044B1343CB60BFF34F8F00BF36
:10CC500000BFFDE700ED00E00400FA0580B400AF7E
:10CC6000034B1B78DBB21846BD465DF8047B70476A
:10CC70007C5B002080B582B000AF78600B467B8083
:10CC8000094B1B78DBB2002B0AD07B68002B07D046
:10CC90007B88002B04D07B8819467868FDF74EFF0F
:10CCA00000BF0837BD4680BD7C5B002080B582B0E8
:10CCB00000AF786039603B68002B15D00C4B012227
:10CCC0001A703B683F2B01D93F233B603A68796873
:10CCD000084805F016FC074A3B68134400221A7006
:10CCE000054B01221A7000E000BF0837BD4680BD29
:10CCF0007C5B00203C5B0020385B002080B500AFEF
:10CD00000E4B1B78DBB283F00103DBB2002B13D197
:10CD10000A4B00221A703F2209490A4805F06BFBB2
:10CD2000084B002283F83F2000F050F840220021F9
:10CD3000044805F02FFB00E000BF80BD385B0020F9
:10CD40003C5B0020F85A002080B588B000AFF86046
:10CD5000B9607A600023FB612C21F86805F03EFB86
:10CD600078617B69002B01D100232AE07B690022D6
:10CD70001A707B690133BB6115E0FB695A1CFA61CB
:10CD80009B00BA681344BA691A602C21B86905F08F
:10CD900025FB78617B69002B11D07B6900221A701A
:10CDA0007B690133BB61FA697B689A4208DABB6927
:10CDB000002B05D0BB691B78002BDED100E000BF43
:10CDC000FB6918462037BD4680BD0000F0B5CFB0E6
:10CDD00008AF002387F8173107F18C0320220021C8
:10CDE000184605F0D7FA0023C7F8043107F14C03C1
:10CDF0003F22C449184605F0FEFA002387F88B301D
:10CE000007F18C0107F14C0308221846FFF79CFF3D
:10CE1000C7F804010023C7F8103100F084BDBA4AF6
:10CE2000D7F8103152F8332007F14C031146184659
:10CE3000F3F7C4FD0346002B40F07085B24AD7F8E3
:10CE40001031DB0013441B79013B122B00F2598592
:10CE500001A252F823F000BFA5CE0008EFCE0008D3
:10CE600073CF0008D3CF0008D3D0000869D20008E0
:10CE700001D30008BFD30008D9D7000871D3000838
:10CE800003D9000815D5000873D50008E5D50008BA
:10CE900065D6000803D900085FD70008F3D800085A
:10CEA000FBD80008994805F061F9994B994A1A6036
:10CEB000994B9A4A1A609A48FBF7FCFF00224FF4FC
:10CEC00080514FF09040F9F7B9F80023C7F80C31C2
:10CED00005E000BFD7F80C310133C7F80C31D7F8A3
:10CEE0000C3142F20F729342F3DDFFF7A1FED7F847
:10CEF0000431002B04DC8B4805F038F900F00ABD42
:10CF0000D7F88C3088491846F3F758FD0346002BB4
:10CF100008D0D7F88C308549184605F043FA034607
:10CF2000002B06D1824B01221A70824805F01EF9AF
:10CF30001DE0D7F88C3080491846F3F73FFD0346D3
:10CF4000002B08D0D7F88C307C49184605F02AFA17
:10CF50000346002B06D1764B00221A70784805F064
:10CF600005F904E0774805F001F900F0D3BC00F0C2
:10CF7000D1BCD7F80431002B04DC734805F0F6F877
:10CF800000F0C8BCD7F88C307049184605F00AFA92
:10CF90000346002B07D1664B00225A606C4805F00F
:10CFA000E5F800F0B7BCD7F88C306A49184605F0B0
:10CFB000F9F90346002B07D15D4B01225A60664800
:10CFC00005F0D4F800F0A6BC644805F0CFF800F0F6
:10CFD000A1BCD7F80431002B04DC614805F0C6F889
:10CFE00000F098BC5F4B1B78102B36D1D7F88C30F3
:10CFF000184604F0EFFDC7F8B000D7F8B030002BAA
:10D0000003DDD7F8B0303C2B04DD574805F0AEF80F
:10D0100000F080BCD7F8B030DBB21946534804F0BA
:10D02000A8FB0346C7F8AC30D7F8AC30002B04D0CF
:10D030004F4805F09BF800F06DBCD7F8B030DAB27D
:10D040004C4B1A703A4AD7F8B0309360D7F8B0100A
:10D05000494805F023F800F058BC424B1B78402BA0
:10D0600040F05384D7F88C30184604F0B3FDC7F86D
:10D07000B800D7F8B830002B03DDD7F8B8300F2B45
:10D0800004DD3E4805F072F800F044BCD7F8B83033
:10D09000DBB21946354804F06CFB0346C7F8B430E0
:10D0A000D7F8B430002B04D0314805F05FF800F019
:10D0B00031BCD7F8B830DAB22E4B1A701C4AD7F808
:10D0C000B8309360D7F8B8102B4804F0E7FF00F0B1
:10D0D0001CBCD7F80431002B04DC294805F046F8C5
:10D0E00000F018BC002387F80B31D7F88C302549A5
:10D0F0001846F3F763FC0346002B45D1102387F84D
:10D100000B3152E0F85A0020C4480108703701087A
:10D11000F45F002067452301F85F0020EFCDAB8965
:10D120007C02002088370108C8370108CC37010885
:10D13000CC010020D4370108EC370108F037010892
:10D14000F837010810380108503801089C380108E8
:10D15000A0380108BC380108C4380108E0380108CB
:10D160001C390108C801002054390108BC4F0020B7
:10D1700094390108C9010020A8390108C4390108FF
:10D18000043A0108503A0108D7F88C30AC491846E7
:10D19000F3F714FC0346002B03D1402387F80B312F
:10D1A00003E0A84804F0E2FFB4E3A74B1B78002B90
:10D1B00013D0A54B00221A70A44803F009FF0346C0
:10D1C000C7F8C430D7F8C430002B03D0A04804F00F
:10D1D000CDFF9FE39F4804F0C9FF9F4A97F80B31AA
:10D1E00013709D4B1B781946984804F0EEF90346DE
:10D1F000C7F8C030D7F8C030002B03D0974804F0F0
:10D20000B5FF87E397F80B311946954804F046FFC0
:10D210008E4803F047FD0346C7F8BC30D7F8BC3052
:10D22000002B03D08F4804F0A1FF73E38E4804F075
:10D230009DFF854B01221A7097F80B319BB219465E
:10D2400040F2031001F062FE0346002B05D097F870
:10D250000B311946854804F021FF97F80B31194628
:10D26000834804F01BFF55E3D7F80431002B03DC9F
:10D27000804804F07BFF4DE3D7F88C30184604F06B
:10D28000A9FCC7F8CC00744B1B78102B0BD1D7F836
:10D29000CC30002B03DDD7F8CC303C2B0FDD7648AB
:10D2A00004F064FF36E3D7F8CC30002B03DDD7F869
:10D2B000CC300F2B03DD714804F058FF2AE3D7F878
:10D2C000CC30DBB21946614804F053FA0346C7F884
:10D2D000C830D7F8C830002B03D0694804F046FFA7
:10D2E00018E3D7F8CC30DAB2664B1A70664AD7F832
:10D2F000CC309360D7F8CC10644804F0CFFE09E33B
:10D30000D7F80431002B03DC614804F02FFF01E360
:10D31000D7F88C30184604F05DFCC7F8D400D7F875
:10D32000D430002B03DBD7F8D430642B03DD59480D
:10D3300004F01CFFEEE2D7F8D430DAB2564B1A7084
:10D34000554B1B781946414804F034FA0346C7F898
:10D35000D030D7F8D030002B03D0504804F006FF6F
:10D36000D8E24D4B1B7819464D4804F097FED1E2A8
:10D37000D7F80431002B03DC4A4804F0F7FEC9E279
:10D38000D7F88C30184604F025FCC7F8EC00D7F825
:10D39000EC30002B03DBD7F8EC30FF2B03DD4248E9
:10D3A00004F0E4FEB6E2D7F8EC30DAB23F4B1A7084
:10D3B0003E4B1B7819463E4804F070FEAAE2D7F8AF
:10D3C0000431002B03DC3B4804F0D0FEA2E2D7F886
:10D3D0008C3007F148011022184604F091FDC7E98E
:10D3E0003601D7F88C20BB6C9A4203D0BB6C1B78FB
:10D3F000002B03D0304804F0B9FE8BE22F49D7E967
:10D400003623C1E90023D7E9362340F2191001F091
:10D4100015FE0346002B55D0284BD3E900014FF0F1
:10D4200000024FF000030A0000231146234BD3E90A
:10D43000002313461A46224804F030FE54E000BF91
:10D44000543A0108583A0108705A0020BC4F002095
:10D45000903A0108C03A0108C8010020E83A0108E2
:10D46000003B0108203B0108543B0108683B0108D0
:10D47000BC3B0108F03B0108283C0108603C010866
:10D48000983C0108C9010020CC010020B03C0108F3
:10D49000D43C01080C3D0108B84F0020403D010874
:10D4A0005C3D01087C3D0108B83D0108CA0100202F
:10D4B000F03D0108103E0108503E0108C001002067
:10D4C000883E0108C74BD3E900014FF000024FF03E
:10D4D00000030A0000231146C24BD3E90023134680
:10D4E0001A46C14804F0DAFDC04B1B78102B40F0FF
:10D4F0000E82D7E936014FF000024FF00003020C14
:10D5000042EA01420B0C134300F00182B84804F0D8
:10D510002DFEFCE1D7F80431002B03DCB54804F004
:10D5200025FEF7E1D7F88C3000220021184604F0E0
:10D5300047FC0346A7F8F23007F14602B7F8F2308D
:10D540001146184601F0C9FC0346002B06D0B7F877
:10D55000F2301946A84804F0A1FDDBE1B7F8F2105B
:10D56000B7F846301A46B7F84630A44804F096FD9E
:10D57000D0E1D7F80431012B03DCA14804F0F6FD1B
:10D58000C8E1D7F88C3000220021184604F018FCBE
:10D590000346A7F8F630D7F890300022002118464D
:10D5A00004F00EFC0346A7F8F430B7F8F420B7F8FF
:10D5B000F6301146184601F0A9FC0346002B08D0AE
:10D5C000B7F8F430B7F8F62019468E4804F066FD37
:10D5D000A0E1B7F8F430B7F8F62019468A4804F00D
:10D5E0005DFD97E101F036FB034687F8FF3097F8C1
:10D5F000FF30002B03D1854804F0B8FD8AE101F02B
:10D600001DFBC7F8F800D7F8F830002B0BD0804985
:10D61000D7F8F800F3F7D2F90346002B03D17D4881
:10D6200004F0A4FD1DE0D7F8F830002B0BD07A49A8
:10D63000D7F8F800F3F7C2F90346002B03D1774877
:10D6400004F094FD0DE0D7F8F830002B05D0D7F8A2
:10D65000F810734804F022FD5CE1724804F086FD86
:10D6600058E157E1704804F081FD4FF48073A7F84A
:10D67000083120E007F14402B7F808311146184696
:10D6800001F02BFC0346002B0AD1B7F80811B7F8BC
:10D6900044301A46B7F84430644804F0FFFC05E013
:10D6A000B7F808311946624804F0F8FCB7F80831B9
:10D6B0000133A7F80831B7F80831B3F58E7FD9D90F
:10D6C00007F124010E231D2240F2071001F0D9FDBD
:10D6D0000346002B09D197F82430002B05D007F121
:10D6E00024031946534804F0D9FC07F11801042318
:10D6F000092240F2151001F0C4FD0346002B0CD1A5
:10D7000007F58C73A3F580731B78002B05D007F108
:10D7100018031946484804F0C1FC4FF000024FF0CE
:10D720000003C7E9042307F11003194640F219105A
:10D7300001F0DEFC0346002B40F0EB80D7E904014A
:10D740004FF000024FF000030A0000231146D7E912
:10D75000042313461A46394804F0A0FCD9E0D7F850
:10D760000431002B06DC364B1B681946354804F0A3
:10D7700095FCCFE0D7F88C30184604F02BFAC7F8A8
:10D780000001D7F80031002B03DBD7F800313F2B25
:10D7900003DD2D4804F0EAFCBCE0D7F800319BB271
:10D7A00019464FF4817001F0B1FB0346002B04D001
:10D7B000D7F80011254804F071FCD7F8003103F0C8
:10D7C0003F031F4A1360224800F042FED7F80011C1
:10D7D000204804F063FC9DE01F4B1B78002B3DD0DC
:10D7E0001D4B3CE0C0010020C03E0108C8010020E4
:10D7F000E03E0108183F01084C3F0108783F01084E
:10D80000943F0108D43F0108044001082C4001085E
:10D81000744001087C400108E8400108F04001081C
:10D820003C410108A4410108BC410108D84101085C
:10D83000F041010808420108204201083C42010869
:10D840005C5E002060420108A8420108D442010841
:10D85000DC01002014430108745E00203F4BC7F830
:10D86000E8303F4B1B78002B01D03D4B00E03D4B97
:10D87000C7F8E4303C4B1B78002B01D03B4E00E056
:10D880003B4E394B5B68002B01D13A4C00E03A4CDF
:10D890003A4B1B78FB603A4B1B78BB60394B1B78CB
:10D8A0007B60394B1B783B60384B1D68384BD3E9A4
:10D8B00000014FF000024FF000030A000023114660
:10D8C000334BD3E9002313460793069105953A6835
:10D8D00004927A680392BA680292FB6801930094FA
:10D8E0003346D7F8E420D7F8E8102A4804F0D6FBEE
:10D8F00010E0294804F03AFC0CE0284804F036FC1B
:10D9000008E0274804F032FC04E000BF02E000BF5A
:10D9100000E000BF012387F8173109E0D7F8103184
:10D920000133C7F81031D7F81031102B7FF677AAE2
:10D9300097F8173183F00103DBB2002B08D007F111
:10D940004C031946174804F0A9FB174804F00EFCD5
:10D9500000BF07F58E77BD46F0BD00BF4843010804
:10D96000945E002054430108CC0100205C43010870
:10D970006443010870430108BC380108C901002054
:10D98000C8010020B84F0020CA0100205C5E0020C2
:10D99000C001002078430108E8430108F84301086A
:10D9A000004401081C4401083444010880B586B0D5
:10D9B00000AF3B1D00221A605A609A60DA601A615B
:10D9C0004FF480537B601123BB600023FB603B1D41
:10D9D00019464FF09040F8F7AFF900224FF480510C
:10D9E0004FF09040F8F72AFB6420F6F72DFD012256
:10D9F0004FF480514FF09040F8F720FB00BF1837EC
:10DA0000BD4680BD80B483B000AF78607B68082BD2
:10DA100002D87B68DBB224E07B68093B062B1FD869
:10DA200001A252F823F000BF45DA000849DA0008E5
:10DA30004DDA000851DA000855DA000859DA000812
:10DA40005DDA00080C230CE010230AE0142308E040
:10DA5000182306E0202304E0302302E0402300E006
:10DA6000002318460C37BD465DF8047B704700BFA5
:10DA700080B483B000AF0346FB71FB79082B01D85B
:10DA8000FB791EE0FB790C2B01D8092319E0FB7907
:10DA9000102B01D80A2314E0FB79142B01D80B2397
:10DAA0000FE0FB79182B01D80C230AE0FB79202B1F
:10DAB00001D80D2305E0FB79302B01D80E2300E0BF
:10DAC0000F2318460C37BD465DF8047B704780B4C1
:10DAD00083B000AF786039603B68DAB27B681A7057
:10DAE0003B681A0A7B680133D2B21A703B681A0C81
:10DAF0007B680233D2B21A703B681A0E7B6803331C
:10DB0000D2B21A7000BF0C37BD465DF8047B704777
:10DB100080B485B000AFF860C7E900233A78FB68AD
:10DB20001A70D7E900014FF000024FF00003020A1B
:10DB300042EA01620B0AF9680131D3B20B70D7E9EE
:10DB400000014FF000024FF00003020C42EA0142D4
:10DB50000B0CF9680231D3B20B70D7E900014FF01A
:10DB600000024FF00003020E42EA01220B0EF96898
:10DB70000331D3B20B70D7E900014FF000024FF030
:10DB800000030A000023F9680431D3B20B70D7E90F
:10DB900000014FF000024FF000030A0A0023F96869
:10DBA0000531D3B20B70D7E900014FF000024FF0FE
:10DBB00000030A0C0023F9680631D3B20B70D7E9D1
:10DBC00000014FF000024FF000030A0E0023F96835
:10DBD0000731D3B20B7000BF1437BD465DF8047B2C
:10DBE00070470000B0B58EB000AF7860314A7B68F6
:10DBF0001360314B07F120041D460FCD0FC495E88B
:10DC0000030084E803002B4B1B6807F12002114638
:10DC10001846F8F793FD0346002B01D0FDF752FE9E
:10DC2000264B07F108041D460FCD0FC495E80300ED
:10DC300084E803001F4B1B6807F1080211461846D1
:10DC4000F8F77CFD0346002B01D0FDF73BFE1C4B93
:10DC5000002283F8D0221A4B092283F8D122184BD4
:10DC6000002283F8D222134B1B681846F8F7C0FD38
:10DC70000346002B01D0FDF725FE0E4B1B6800224A
:10DC800001211846F8F73AFF0346002B01D0FDF7B3
:10DC900019FE084B1B68072280211846F8F72EFF53
:10DCA0000346002B01D0FDF70DFE00BF3837BD46FF
:10DCB000B0BD00BF545E00206844010880440108E4
:10DCC000805B002080B596B000AFF860B960134665
:10DCD000FB7107F1100348220021184604F05AFB9B
:10DCE000FB683B65FB7987F85430FA7907F110033C
:10DCF000B968184604F005FC1A4B93F8D132013389
:10DD0000DAB2184B83F8D122164B93F8D122164B76
:10DD1000A3FB0213D9080B469B000B445B00D31AEC
:10DD2000DAB2104B83F8D1220E4B93F8D132194658
:10DD30000C4A0B46DB000B44DB001344184607F18A
:10DD400010034822194604F0DCFB064B93F8D2324C
:10DD50000133DAB2034B83F8D22200BF5837BD46F5
:10DD600080BD00BF805B0020CDCCCCCC80B592B014
:10DD700000AF234B93F8D0321946214A0B46DB0003
:10DD80000B44DB001A443B4611464822184604F077
:10DD9000B8FB1C4B1B78002B07D03B6C97F844203A
:10DDA0003946184600F032F806E03B6C97F84420FC
:10DDB0003946184600F082FB114B93F8D0320133FC
:10DDC000DAB20F4B83F8D0220D4B93F8D0220E4BD2
:10DDD000A3FB0213D9080B469B000B445B00D31A2C
:10DDE000DAB2074B83F8D022054B93F8D232013BCD
:10DDF000DAB2034B83F8D22200BF4837BD4680BD5C
:10DE0000805B0020595E0020CDCCCCCC80B5A0B08A
:10DE100000AFF860B9601346FB712F4B1B68002BF5
:10DE200005D0FB79002B02D0FB79402B01D90123CF
:10DE30004DE0294B1B681846F8F74EFE0346002BB1
:10DE400007D1FB791A46B968F868FFF73BFF002352
:10DE50003DE0FB791846FFF70BFEF867F86FFFF718
:10DE6000D1FD034687F87B3007F1380340220021BB
:10DE7000184604F08FFAFA7907F13803B9681846A2
:10DE800004F03FFBFB687B614FF08043BB610023E4
:10DE9000FB61FB6F3B6200237B62104B1B78002B06
:10DEA00002D04FF4801300E00023BB624FF4001354
:10DEB000FB6200233B6300237B63074B1B6807F176
:10DEC000380207F114011846F8F7BAFC0346184661
:10DED0008037BD4680BD00BF545E00205A5E0020E2
:10DEE000B0B5A4B008AF786039601A4B1B78002B2E
:10DEF00006D03968184804F0D1F8164B00221A7081
:10DF00003B6803F00103002B1FD007F130034022D0
:10DF10000021184604F03EFA07F1300307F1080229
:10DF200040217868F8F7D0FC07F1300306936D467E
:10DF300007F118040FCC0FC594E8030085E803002F
:10DF400007F108030FCB00F027F800BF7037BD467C
:10DF5000B0BD00BFF80100209844010880B584B02E
:10DF600000AFF860B9601346FB71FB68074A934243
:10DF700003D3FB68064A934204D9F968054804F0C4
:10DF80008DF800E000BF1037BD4680BD00040906D3
:10DF90003F040906B844010884B080B590B000AFD2
:10DFA00007F1480C8CE80F00BB6CBB637B6D184617
:10DFB000FFF728FD034687F83730A24B1B783B63F9
:10DFC0003B6B002B24D097F837301A46B96B9E482C
:10DFD00004F064F8002387F83F300DE097F83F30F5
:10DFE0003A6F13441B781946984804F057F897F88D
:10DFF0003F30013387F83F3097F83F2097F83730AC
:10E000009A42EBD3924804F0B1F88E4B00221A707A
:10E01000904B5B69BA6B9A4213D0BB6BB3F5207F10
:10E02000C0F0F680BB6BB3F5307F80F0F180BB6B46
:10E03000A3F52072884B1B6803F03F039A4240F01F
:10E04000E7803B462C220021184604F0A3F9002368
:10E0500087F82F3097F82F305A1C87F82F2040333D
:10E060003B44012203F8402C7C4B5B78002B01D011
:10E07000012200E0002297F82F30591C87F82F105A
:10E0800040333B4403F8402C754B1B78002B01D0E8
:10E09000012200E0002297F82F30591C87F82F103A
:10E0A00040333B4403F8402C6E4B1B78002B01D0CF
:10E0B000012200E0002297F82F30591C87F82F101A
:10E0C00040333B4403F8402C634B1B68DAB297F8AB
:10E0D0002F30591C87F82F1002F03F02D2B2403384
:10E0E0003B4403F8402C97F82F30033387F82F3048
:10E0F00097F82F303A461344564A1268114618468C
:10E10000FFF7E5FC97F82F30043387F82F3097F8A6
:10E110002F303A4613444F4A526811461846FFF7CB
:10E12000D6FC97F82F30043387F82F3097F82F302C
:10E130003A461344474A926811461846FFF7C7FC0F
:10E1400097F82F30043387F82F3097F82F303A465E
:10E150001344404AD26811461846FFF7B8FC97F8B6
:10E160002F30043387F82F3097F82F303A46134476
:10E17000384A126911461846FFF7A9FC97F82F3064
:10E18000043387F82F3097F82F303A461344314A3A
:10E19000526911461846FFF79AFC97F82F3004335E
:10E1A00087F82F3097F82F303A461344294A92695E
:10E1B00011461846FFF78BFC97F82F30043387F889
:10E1C0002F3097F82F303A46D118274BD3E9002348
:10E1D0000846FFF79DFC97F82F30083387F82F305B
:10E1E0001C4B9B6939460822184600F067F91F4B03
:10E1F0001B7883F00103DBB2002B1CD01B4B0122E8
:10E200001A70144B9B691946194803F047FF12E036
:10E21000134B1B78002B07D097F837301A46396F0D
:10E22000B86BFFF79BFE06E097F837301A46396F58
:10E23000B86B00F091F94037BD46BDE8804004B0AE
:10E24000704700BFF9010020D444010808450108C7
:10E2500010450108DC0100205C5E0020D801002090
:10E26000595E00205A5E0020C0010020605E002040
:10E270001445010884B080B598B000AF07F1680C70
:10E280008CE80F00664B5B7883F00103DBB2002B58
:10E2900040F0BD8097F86930002B02D097F86930C4
:10E2A00001E0604B1B7887F85F3097F85F30002BF8
:10E2B00000F0AF8097F85F30402B02D9402387F8F9
:10E2C0005F30102387F85B3097F85F2097F85B305A
:10E2D00013445A1E97F85B30B2FBF3F387F85A30B9
:10E2E000514B5B687B64504B9B68BB644E4BDB6857
:10E2F000FB644D4B1B693B65002387F85E307AE079
:10E30000002387F85D3097F85D305A1C87F85D2050
:10E3100097F8682060333B4403F85C2C97F85D3035
:10E320005A1C87F85D2060333B4497F85F2003F860
:10E330005C2C97F85E2097F85B3012FB03F387F8AC
:10E34000593097F8592097F85B301A4497F85F30A6
:10E350009A4206DD97F85F2097F85930D31ADBB25E
:10E3600001E097F85B3087F85830002387F85C307D
:10E3700029E097F8592097F85C3013445B00683324
:10E380003B445B88A7F8563097F85D305A1C87F8F5
:10E390005D20B7F85620D2B260333B4403F85C2CC2
:10E3A000B7F956301B121AB297F85D30591C87F82E
:10E3B0005D10D2B260333B4403F85C2C97F85C30BC
:10E3C000013387F85C3097F85C2097F858309A4210
:10E3D000CFD397F85E309B0060333B4453F81C3C2E
:10E3E00097F85D20391D1846FFF710FD97F85E304D
:10E3F000013387F85E3097F85E2097F85A309A42DA
:10E4000008D297F85E30032B7FF67AAF02E000BFA8
:10E4100000E000BF6037BD46BDE8804004B07047F3
:10E42000D8010020C8010020DC01002080B582B0A6
:10E4300000AF78603960054B93F8D232002B01D0E1
:10E44000FFF794FC00BF0837BD4680BD805B00200D
:10E4500080B485B000AF7860174B1B68FB60FB6829
:10E4600003F1C16303F58033BB607B68BA681A604F
:10E47000BB6803F140027B685A60BB6803F180020D
:10E480007B689A60BB6803F1C0027B68DA60BB6896
:10E4900003F580727B681A61BB6803F580627B6854
:10E4A0005A61BB6803F588627B689A6100BF1437C4
:10E4B000BD465DF8047B70475C5E002080B58EB081
:10E4C00000AFF860B9601346FB71214B1B68002B4D
:10E4D00005D0FB79002B02D0FB79082B01D9012351
:10E4E00031E01B4B1B681846F8F7F6FA0346002B81
:10E4F00007D1FB791A46B968F868FFF7E3FB0023F8
:10E5000021E0FB791A46B968124803F0FAFFFB686C
:10E510007B614FF08043BB610023FB6108233B62BA
:10E5200000237B620023BB620023FB6200233B636A
:10E5300000237B63064B1B6807F11401054A18464C
:10E54000F8F77EF9034618463837BD4680BD00BF50
:10E55000545E0020645E002080B485B000AFF86097
:10E56000B9601346FB7100BF1437BD465DF8047BEC
:10E570007047000084B080B586B000AF07F1200C72
:10E580008CE80F004B4B5B7883F00103DBB2002B70
:10E5900040F0868097F82130402B28BF40233B7500
:10E5A0003B7D002B7ED00323FB743A7DFB7C134420
:10E5B0005A1EFB7CB2FBF3F3BB740023FB756AE0CD
:10E5C0003B1D00221A605A600023BB75BB7D5A1C9C
:10E5D000BA7597F8202018333B4403F8142CBB7D00
:10E5E0005A1CBA7518333B44FA7D03F8142CFA7D93
:10E5F000FB7C12FB03F37B7400237B7529E07A7CA0
:10E600007B7D13443B743A7C3B7D9A4206D23B7C33
:10E610005B0020333B44B3F9023001E04FF0FF339D
:10E62000FB81BB7D5A1CBA75FA89D2B218333B44C0
:10E6300003F8142CB7F90E301B121AB2BB7D591C0B
:10E64000B975D2B218333B4403F8142C7B7D0133E7
:10E650007B757A7DFB7C9A42D1D3174B5B68391D61
:10E6600008221846FFF72AFFBB7C062B10D9FA7D3B
:10E67000BB7C013B9A420BD200233B6003E03B682A
:10E680003B6801333B603B6844F61F629342F6D916
:10E69000FB7D0133FB75FA7DBB7C9A4290D302E08F
:10E6A00000BF00E000BF1837BD46BDE8804004B0A1
:10E6B000704700BFD8010020DC01002080B400AF0B
:10E6C000034B1B881846BD465DF8047B704700BFAE
:10E6D000E075FF1F80B582B000AFFFF7EFFF034684
:10E6E00003F500339B027B607B68A3F580531846DB
:10E6F0000837BD4680BD80B582B000AFFFF7DEFFB2
:10E70000034603F500339B027B607B68A3F500633F
:10E7100018460837BD4680BD80B483B000AF78602E
:10E720007B6803F5006318460C37BD465DF8047B33
:10E73000704780B483B000AF78607B68D3E9002372
:10E74000104619460C37BD465DF8047B7047000043
:10E7500080B58AB000AF786007F1100300221A601C
:10E760005A609A60DA600023FB6000233B6101235A
:10E77000FB61224B1B6A03F48003002B1BD0FFF7C5
:10E780009DFF03469B025B0803F100637B627A688E
:10E790007B6A9A4207D302237B617A687B6AD31A29
:10E7A000DB0ABB610EE001237B617B6803F17843E8
:10E7B000DB0ABB6106E001237B617B6803F17843E0
:10E7C000DB0ABB6107F10C0207F110031146184682
:10E7D000F6F76EFF034687F8233097F82330002BB7
:10E7E00003D1FB68B3F1FF3F01D0012300E0002318
:10E7F000DBB218462837BD4680BD00BF002002406E
:10E8000080B584B000AFF860C7E90023D7E90023E2
:10E81000F9680020F6F7A2FD034618461037BD46FA
:10E8200080BDF0B484B000AF064608463146F9809A
:10E830000146B980F9880804B988014300200A46D6
:10E840000346C7E90223D7E9022314464FF0FF35F8
:10E8500022462B46104619461037BD46F0BC70477D
:10E8600080B483B000AFC7E90001D7E900014FF0E1
:10E8700000024FF00003020C42EA01420B0C93B27B
:10E8800018460C37BD465DF8047B704780B483B0F2
:10E8900000AFC7E900013B8818460C37BD465DF85C
:10E8A000047B704780B58AB000AFFFF713FF786232
:10E8B000FFF721FF3862786AFFF73BFFC7E90601DF
:10E8C0007B6A08331846FFF734FFC7E90401386A4A
:10E8D000FFF72FFFC7E902013B6A08331846FFF72D
:10E8E00028FFC7E90001D7E90423B3F1AA3F08BF15
:10E8F000B2F1AA3F01D17B6A52E0D7E90023B3F11C
:10E90000AA3F08BFB2F1AA3F01D13B6A48E0D7E96C
:10E910000623B3F1AA3F08BFB2F1AA3F01D17B6A37
:10E920003EE0D7E90223B3F1AA3F08BFB2F1AA3F04
:10E9300001D13B6A34E0D7E90623B3F1EE3F08BFCB
:10E94000B2F1EE3F11D1D7E90223B3F1FF3F08BF87
:10E95000B2F1FF3F09D1D7E90023B3F1FF3F08BF70
:10E96000B2F1FF3F01D17B6A1AE0D7E90223B3F18C
:10E97000EE3F08BFB2F1EE3F11D1D7E90623B3F164
:10E98000FF3F08BFB2F1FF3F09D1D7E90423B3F13C
:10E99000FF3F08BFB2F1FF3F01D13B6A00E0002317
:10E9A00018462837BD4680BD80B582B000AF78607C
:10E9B000FFF790FE02467B68934203D1FFF79BFE70
:10E9C000034602E0FFF786FE034618460837BD46B9
:10E9D00080BD80B584B000AF78607B681033FB6089
:10E9E0007868FFF799FEB8600FE0F868FFF7A1FEBE
:10E9F00002460B46B3F1FF3F08BFB2F1FF3F01D122
:10EA0000FB6808E0FB680833FB60FB680833BA6802
:10EA10009A42EAD2002318461037BD4680BD80B521
:10EA200088B000AFF8600B467A607B81F868FFF72A
:10EA300073FEB861BB69FB6123E0FB69083BFB61C6
:10EA4000F869FFF776FEC7E90401D7E90423B3F1BB
:10EA5000FF3F08BFB2F1FF3F12D0D7E90401FFF733
:10EA6000FFFE03461A467B8993420AD1D7E9040187
:10EA7000FFF70CFF03461A467B681A80002306E066
:10EA800000BFFB680833FA699A42D6D801231846BA
:10EA90002037BD4680BD000090B59BB000AF7860C8
:10EAA00039605E4B4CF2FA321A613868FFF750FE5B
:10EAB000034687F85F3097F85F30002B05D0584B3E
:10EAC000584A1A6097F85F30A4E04FF0EE324FF0EA
:10EAD000EE333868FFF794FE034687F85F3097F807
:10EAE0005F30002B05D04E4B4F4A1A6097F85F30CD
:10EAF00090E007F10C0340220021184603F04AFC85
:10EB00007868FFF709FEB865BB6D7B663B6810331C
:10EB10003B6654E07B6E083B7B66786EFFF709FE30
:10EB2000C7E91401D7E91423B3F1FF3F08BFB2F1DD
:10EB3000FF3F43D0D7E91401FFF792FE0346A7F841
:10EB40004E30B7F84E30A3F58073A7F84C30B7F8C5
:10EB50004C303F2B33D8B7F84C3068333B4413F874
:10EB60005C3C002B2BD13B6E03F108043868FFF7A7
:10EB7000D3FD03469C4204D9294B2C4A1A60012339
:10EB800048E0D7E91423386EFFF73AFE034687F8CA
:10EB90005F3097F85F30002B05D0214B244A1A6074
:10EBA00097F85F3036E03B6E08333B66B7F84C3081
:10EBB00068333B44012203F85C2C00E000BF7B6813
:10EBC00008337A6E9A42A5D83B6803F108014FF0EA
:10EBD000AA324FF0AA330846FFF712FE034687F821
:10EBE0005F3097F85F30002B05D00D4B114A1A604B
:10EBF00097F85F300EE07868FFF7AAFD034687F8C4
:10EC00005F3097F85F30002B02D0054B0A4A1A603C
:10EC100097F85F3018466C37BD4690BD0020024023
:10EC2000705E0020AC450108CC450108EC450108A8
:10EC300008460108284601084846010880B400AF8C
:10EC4000034B1B681846BD465DF8047B704700BF48
:10EC50006C5E002080B584B000AF0023FB73304BA6
:10EC6000304A1A60FFF736FD7860FFF744FD3860E0
:10EC70002D4BBB602D4ABB68934201D22B4BBB602E
:10EC80007A68BB689A4204D2254B294A1A6001234C
:10EC900042E0F6F7CFFB0346002B04D0204B254A79
:10ECA0001A60012338E0244B4CF2FA321A6178687A
:10ECB000FFF74EFD0346FB73FB7B002B03D0184B85
:10ECC0001E4A1A601FE03868FFF742FD0346FB73D7
:10ECD000FB7B002B03D0124B194A1A6013E07B68B0
:10ECE00003F108014FF0AA324FF0AA330846FFF7AC
:10ECF00087FD0346FB73FB7B002B03D0084B114AB7
:10ED00001A6000E000BFF6F7B7FBFB7B002B02D1D7
:10ED1000034B00221A60FB7B18461037BD4680BDAE
:10ED20006C5E00206846010888350108E4A30208EB
:10ED3000704601087846010800200240804601081C
:10ED4000884601089046010880B58EB000AFFFF7F5
:10ED5000A9FD78637B6B002B03D1FFF77BFF034694
:10ED6000B7E0FFF7B7FC3863FFF7C5FCF862386B14
:10ED7000FFF7DFFCC7E908013B6B08331846FFF7D4
:10ED8000D8FCC7E90601F86AFFF7D3FCC7E904011C
:10ED9000FB6A08331846FFF7CCFCC7E90201D7E944
:10EDA0000823B3F1AA3F08BFB2F1AA3F07D0D7E9C1
:10EDB0000623B3F1AA3F08BFB2F1AA3F01D1012354
:10EDC00000E00023FB71FB7903F00103FB71D7E93D
:10EDD0000423B3F1AA3F08BFB2F1AA3F07D0D7E995
:10EDE0000223B3F1AA3F08BFB2F1AA3F01D1012328
:10EDF00000E00023BB71BB7903F00103BB71D7E9CD
:10EE00000823B3F1EE3F08BFB2F1EE3F07D1FB7923
:10EE100083F00103DBB2002B01D0012300E00023CB
:10EE20007B717B7903F001037B71D7E90423B3F194
:10EE3000EE3F08BFB2F1EE3F07D1BB7983F001038B
:10EE4000DBB2002B01D0012300E000233B713B79B2
:10EE500003F001033B717B79002B0ED0BB79002BB3
:10EE60000BD0F6F7E7FA396BF86AFFF715FE0346A1
:10EE7000FB70F6F701FBFB782BE03B79002B0ED003
:10EE8000FB79002B0BD0F6F7D5FAF96A386BFFF750
:10EE900003FE0346BB70F6F7EFFABB7819E0FB7987
:10EEA000002B15D0BB79002B12D0F6F7C3FAD7E9A7
:10EEB0000823B3F1EE3F08BFB2F1EE3F03D1F86A89
:10EEC000FFF746FC02E0386BFFF742FCF6F7D4FA96
:10EED000002318463837BD4680BD80B584B000AFEA
:10EEE00003463960FB80FFF7DDFCF860FB68002B10
:10EEF00001D1012306E0FB883A681946F868FFF75C
:10EF00008EFD034618461037BD4680BD80B586B0DD
:10EF100000AF03460A46FB801346BB803E4B0022EF
:10EF20001A60FFF7BFFC38613B69002B1DD1FFF76A
:10EF300091FE0346FB75FB7D002B0BD0374B1B6806
:10EF4000002B02D0354B1B6800E0354B324A136072
:10EF5000FB7D5DE0FFF7A6FC38613B69002B04D127
:10EF60002D4B304A1A60012352E0F6F763FA03464C
:10EF7000002B04D0284B2C4A1A60012348E02B4B6D
:10EF80004CF2FA321A613869FFF723FDF860FB682A
:10EF9000002B23D13869FFF707FDB860B9683869DD
:10EFA000FFF77AFD0346FB75FB7D002B07D01A4B5C
:10EFB0001B68002B26D1184B1D4A1A6022E0BB6843
:10EFC0003B613869FFF705FDF860FB68002B05D150
:10EFD000114B184A1A600123FB7516E0BA88FB88AA
:10EFE00011461846FFF71DFC02460B46F868FFF76E
:10EFF00007FC0346FB75FB7D002B05D0064B0E4A34
:10F000001A6002E000BF00E000BFF6F735FAFB7DB2
:10F0100018461837BD4680BD705E00206C5E00202B
:10F0200098460108A8460108C4460108002002408D
:10F03000D8460108F44601081047010890B587B08A
:10F0400000AF0146C7E900230B46FB813A88FB89E4
:10F0500011461846FFF75AFF0346FB75FB7D002B50
:10F0600001D0FB7D40E0FB8901339CB2D7E9000170
:10F070004FF000024FF00003020C42EA01420B0C79
:10F0800093B219462046FFF741FF0346FB75FB7D0F
:10F09000002B01D0FB7D27E0FB8902339CB2D7E92E
:10F0A00000014FF000024FF000030A00002393B26A
:10F0B00019462046FFF72AFF0346FB75FB7D002B10
:10F0C00001D0FB7D10E0FB8903339CB2D7E900013E
:10F0D0004FF000024FF000030A0C002393B21946D0
:10F0E0002046FFF713FF034618461C37BD4690BD68
:10F0F0002DE9F04F8FB000AF0346B962FB850023C6
:10F10000FB860023BB8600237B8600233B8607F11A
:10F110003602FB8D11461846FFF7DFFE0346002B33
:10F1200001D0012369E0FB8D01339AB207F134036A
:10F1300019461046FFF7D1FE0346002B01D00123EC
:10F140005BE0FB8D02339AB207F132031946104699
:10F15000FFF7C3FE0346002B01D001234DE0FB8DDA
:10F1600003339AB207F1300319461046FFF7B5FE94
:10F170000346002B01D001233FE03B8E9BB20022CF
:10F180003B627A624FF000004FF000013B6A1904C5
:10F1900000207B8E9BB20022BB61FA614FF000021F
:10F1A0004FF00003BE693300002240EA020A41EA40
:10F1B000030BBB8E9BB200223B617A61D7E904123C
:10F1C0000B464FEA13490B464FEA03484AEA080444
:10F1D0004BEA0905FB8E9BB20022BB60FA60D7E9BF
:10F1E00002120B4623433B6013462B437B60BB6AF2
:10F1F000D7E90012C3E90012002318463C37BD4688
:10F20000BDE8F08F80B584B000AF03463960FB8065
:10F2100013467B710023FB732AE0FB7B5B001A46DD
:10F220003B6813441B78BB73FB7B5B0001333A687C
:10F2300013441B787B73BB7B1AB27B7B1BB21B0214
:10F240001BB213431BB27B81FB7B9AB2FB88134436
:10F250009BB27A8911461846FFF758FE03467B7227
:10F260007B7A002B01D07B7A07E0FB7B0133FB73B9
:10F27000FA7B7B799A42D0D3002318461037BD46DB
:10F2800080BD80B586B000AF396011461A4603468E
:10F29000FB800B467B7113463B717B79002B01D1C0
:10F2A00001234AE00023FB753CE00023FB81FB7D4A
:10F2B0009AB2FB8813449BB207F10E02114618461E
:10F2C000FFF70BFE0346002B04D03B6800221A70A8
:10F2D000012332E0FB89BB75FB891B0A9BB27B755E
:10F2E000FB7D5B003B617B79013B3A699A4204D22A
:10F2F0003A683B691344BA7D1A703B695A1C7B79A2
:10F30000013B9A4205D23B6901333A6813447A7D46
:10F310001A70BB7D002B09D07B7D002B06D0FB7DB6
:10F320000133FB75FA7D3B799A42BED37B79013B71
:10F330003A68134400221A70002318461837BD4655
:10F3400080BD000080B582B000AF78607B6800228D
:10F350001A707B6800225A707B6800229A707B6862
:10F360004022DA707B680F221A717B6800225A7182
:10F370007B68A0229A7179684FF0FF324FF0FF331B
:10F38000C1E902237B6800221A747B682D330822AE
:10F390000549184603F02FF87B68002283F83520D2
:10F3A00000BF0837BD4680BD28470108F0B587B0CB
:10F3B00002AF786007F10E0319464FF48070FFF733
:10F3C0008CFD0346002B03D1FB89DAB27B681A70EF
:10F3D00007F10E03194640F20110FFF77EFD0346C8
:10F3E000002B03D1FB89DAB27B685A7007F10E0358
:10F3F00019464FF48170FFF770FD0346002B03D1CF
:10F40000FB89DAB27B689A7007F10E03194640F265
:10F410000310FFF762FD0346002B09D1FB89102B77
:10F4200002D0FB89402B03D1FB89DAB27B68DA700A
:10F4300007F10E0319464FF48270FFF74EFD0346A5
:10F44000002B1CD1FB89002B0BD0FB893C2B08D84F
:10F450007B68DB78102B04D1FB89DAB27B681A71E8
:10F460000DE0FB89002B0AD0FB890F2B07D87B68A6
:10F47000DB78402B03D1FB89DAB27B681A7107F184
:10F480000E03194640F20510FFF727FD0346002B37
:10F4900006D1FB89642B03D8FB89DAB27B685A71E9
:10F4A00007F10E0319464FF48370FFF716FD03466C
:10F4B000002B06D1FB89FF2B03D8FB89DAB27B68CE
:10F4C0009A717B6803F11004F4F7E0FF0646F4F745
:10F4D000E9FF0546F4F7F2FF034601930095334632
:10F4E0001B4A1D21204602F049FE7B68002283F85A
:10F4F0002C207B6803F12D010423092240F2151012
:10F50000FFF7BFFE7B6893F82D30002B0AD17B6894
:10F510002D3308220F49184602F06DFF7B68002248
:10F5200083F835207B680833194640F21910FFF73D
:10F53000DFFD0346002B06D079684FF0FF324FF015
:10F54000FF33C1E9022300BF1437BD46F0BD00BF41
:10F55000304701082847010880B584B000AF7860C3
:10F560007B681B7819464FF48070FFF7CFFC7B68EF
:10F570005B78194640F20110FFF7C8FC7B689B7866
:10F5800019464FF48170FFF7C1FC7B68DB781946A0
:10F5900040F20310FFF7BAFC7B681B7919464FF461
:10F5A0008270FFF7B3FC7B685B79194640F2051067
:10F5B000FFF7ACFC7B689B7919464FF48370FFF72B
:10F5C000A5FC07F1080308220021184602F0E2FE1C
:10F5D0007B6803F12D0107F108030822184602F0A9
:10F5E0000AFF07F108030422194640F21510FFF73D
:10F5F00009FE7B68D3E9022340F21910FFF71EFDD4
:10F6000000BF1037BD4680BDF0B593B004AF3B4698
:10F610001846FFF797FE3B461846FFF7C7FE3B46E6
:10F620001846FFF799FF3B78002B14BF01230023F6
:10F63000DAB2384B1A70384B01221A70BB7803F0DB
:10F640003F03364A13603648FEF702FF7B78002BF3
:10F6500014BF01230023DAB2324B1A702D4B1B78F2
:10F66000002B01D0304900E030492E4B1B78002B95
:10F6700001D02D4A00E02D4A284B1B68F8783C79D0
:10F680007D79BE790396029501940090284802F096
:10F6900005FD234B1C68224B5D68214B9E68204B67
:10F6A000DB681F4A12691E4949691D488069039039
:10F6B00002910192009333462A4621461D4802F0EA
:10F6C000EDFCFA781C4B1A703A791C4B1A707A7957
:10F6D0001B4B1A70BA791B4B1A70D7E902231A49CF
:10F6E000C1E900233B4610331C221946174802F09B
:10F6F00082FE164B00221A773B462D33082219460C
:10F70000134802F078FE124B00221A7200BF3C37F9
:10F71000BD46F0BD595E0020585E00205C5E0020B2
:10F72000DC0100205A5E0020444701084C470108D4
:10F7300058470108C0470108C8010020C90100203E
:10F74000B84F0020CA010020C0010020745E0020D4
:10F75000945E002080B584B000AFF8600B467A60FC
:10F760007B81798901237A68F86800F037F90346CC
:10F7700018461037BD4680BD80B582B000AF7860B6
:10F780000B467B8013467B707A1C7988012378684E
:10F7900000F006F8034618460837BD4680BD000055
:10F7A00090B5ADF5815D83B000AF07F1280444F852
:10F7B0001C0C084607F1280141F8242C07F1280207
:10F7C00042F8283C07F12803024623F81E2C0023A8
:10F7D00007F5815202F107021370002307F58152E9
:10F7E0001360002307F5805202F11C02136000230E
:10F7F00007F5805202F118021360002307F58052CA
:10F8000002F11C021360CFE007F1280353F8283CF3
:10F81000B3F5805F24D907F5805303F11C031B68FF
:10F8200003F5805307F1280252F8282C9A420FD290
:10F8300007F1280353F8282C07F5805303F11C0324
:10F840001B68D31A07F5805202F11802136010E00A
:10F850004FF4805307F5805202F11802136008E05C
:10F8600007F1280353F8283C07F5805202F11802EB
:10F87000136007F5805303F11C031B689AB207F16C
:10F88000280333F81E3C134407F5805202F1160298
:10F89000138007F5805303F116031B881B0A9BB2E4
:10F8A000DBB263F07F03DAB207F1280303F8142C0C
:10F8B00007F5805303F116031B88DAB207F128031A
:10F8C00003F8132C002307F5815213601EE007F59F
:10F8D00081531A6807F5805303F11C031B68134416
:10F8E00007F1280252F8242C1A4407F581531B68AB
:10F8F0000233127807F128010B4403F8142C07F5A2
:10F9000081531B68013307F58152136007F581535A
:10F910001B6807F5805202F1180212689A42D6D885
:10F9200007F5805303F118031B68023307F5805273
:10F9300002F118021360002210214FF09040F6F7F8
:10F940007DFB07F5805303F118031B689AB207F596
:10F95000805303F118031B68642101FB03F307F1D3
:10F96000280114391C48F7F7D4FC03461A4607F55A
:10F97000815303F107031B78134307F5815202F10A
:10F9800007021370012210214FF09040F6F756FB4A
:10F9900007F5805303F11C031B6803F5805307F53B
:10F9A000805202F11C02136007F1280307F5805210
:10F9B00002F11C02126853F8283C9A42FFF424AF6B
:10F9C00007F5815303F107031B78184607F58157A4
:10F9D0000C37BD4690BD00BF004D002090B5ADF581
:10F9E000815D81B000AF07F1200444F8140C084693
:10F9F00007F1200141F81C2C07F1200242F8203CBD
:10FA000007F12003024623F8162C002307F5805245
:10FA100002F11F021370002307F5805202F1180251
:10FA20001360002307F5805202F1140213600023D3
:10FA300007F5805202F118021360B2E007F12003CB
:10FA400053F8203CB3F5805F24D907F5805303F1C8
:10FA500018031B6803F5805307F1200252F8202C8D
:10FA60009A420FD207F1200353F8202C07F5805358
:10FA700003F118031B68D31A07F5805202F1140230
:10FA8000136010E04FF4805307F5805202F1140226
:10FA9000136008E007F1200353F8203C07F580527B
:10FAA00002F11402136007F5805303F118031B6879
:10FAB0009AB207F1200333F8163C134407F580523D
:10FAC00002F11202138007F5805303F112031B8821
:10FAD0001B12DBB203F07F03DAB207F1200303F855
:10FAE000102C07F5805303F112031B88DAB207F1DB
:10FAF000200303F80F2C002210214FF09040F6F75E
:10FB00009DFA07F1200110394FF48053022230484A
:10FB1000F7F7FFFB03461A4607F5805303F11F036F
:10FB20001B78134307F5805202F11F02137007F18F
:10FB3000200353F81C2C07F5805303F118031B68AE
:10FB4000D11807F5805303F114031B689AB207F527
:10FB5000805303F114031B68642000FB03F31C486B
:10FB6000F7F74DFD03461A4607F5805303F11F03CF
:10FB70001B78134307F5805202F11F021370012214
:10FB800010214FF09040F6F759FA07F5805303F132
:10FB900018031B6803F5805307F5805202F1180221
:10FBA000136007F1200307F5805202F11802126872
:10FBB00053F8203C9A42FFF441AF07F5805303F11C
:10FBC0001F031B78184607F581570437BD4690BDC3
:10FBD000004D002080B485B000AF78600B467B807C
:10FBE0000023FB6021E07A68FB6813441B781A0647
:10FBF000FB68013379680B441B781B041A43FB68CC
:10FC0000023379680B441B781B021343FA680332F2
:10FC100079680A4412781343BB607A68FB6813441E
:10FC2000BA681A60FB680433FB607B88FA689A4202
:10FC3000D9D300BF00BF1437BD465DF8047B7047C1
:10FC400080B582B000AF786039603868F4F7FCFBAB
:10FC5000002318460837BD4680BD80B584B000AF8C
:10FC60007860084611461A460346FB700B46BB7087
:10FC700013463B800023FB730023BB7378687B68CB
:10FC800003F5A062FB783988FFF7A8FE03461A4601
:10FC9000FB7B1343FB737B680A211846FFF7D0FFF9
:10FCA00003461A46FB7B1343FB73BB7BC72B04D96C
:10FCB000FB7B43F00103FB731AE0FB78032B09D9AC
:10FCC0007B6893F802357E2B04D9FB7B43F042031B
:10FCD000FB730DE0BB7B0133BB73BB787A681344C5
:10FCE00093F800253B7E1340DBB23A7F9A42C5D1A0
:10FCF000FB7B18461037BD4680BD80B584B000AF91
:10FD000078600023FB730023BB817B6807F10B0243
:10FD100006211846FFF71EFD03461A46FB7B1343D8
:10FD2000FB73FB7A5BB2002B10DA7B6807F10A02E7
:10FD300007211846FFF70EFD03461A46FB7B1343C7
:10FD4000FB73BB7A03F00103002B11D17B68012107
:10FD50001846FFF775FFBB890133BB81FB7A03F0BF
:10FD60000103002B06D1BB89B3F5FA7FCDD302E0A6
:10FD700000BF00E000BFFB7B18461037BD4680BDCA
:10FD800080B5EAB002AF07F5D073A3F5CE73186063
:10FD90000A4607F5D073A3F29D131A70002387F863
:10FDA0009B3107F5D073A3F5C873D94A92E80300D5
:10FDB00083E8030007F5D073A3F5CC73D54A92E826
:10FDC000030083E8030007F5D073A3F5CE731B6827
:10FDD00003F5A06007F5D073A3F5CE731B6810334D
:10FDE0004FF4F472194602F08CFB07F5D073A3F2BE
:10FDF0009D131B78102B40F0228107F5D073A3F5DB
:10FE0000CE731B6803F5A26207F5D073A3F5C87320
:10FE100003CB1060516007F5D073A3F5CE731B6858
:10FE200003F5A0634FF4F4711846FFF7D3FE07F50E
:10FE3000D073A3F5CE731B6803F23C5107F198030E
:10FE40004FF48072184602F05CFB07F5D073A3F5FF
:10FE5000CE731B6803F5C86107F1180380221846AA
:10FE600002F04FFB002387F89E31ACE0002387F8B7
:10FE70009F319CE097F99F2197F99E31DB00134455
:10FE80005A0007F5D073A3F5847353F8222097F92D
:10FE90009F1197F99E31DB000B445B00591C07F55D
:10FEA000D073A3F5847353F821301A4497F99F1146
:10FEB00097F99E31DB000B440433590007F5D073EA
:10FEC000A3F5847353F821301A4497F99F1197F9D9
:10FED0009E31DB000B445B0003F1090107F5D07391
:10FEE000A3F5847353F82130134497F99F1197F9C0
:10FEF0009E2192000A44990807F5D073A3F58473F4
:10FF000043F8221097F99F2197F99E31DB001344A3
:10FF10005A0007F5D073A3F5C47333F912301946AC
:10FF200097F99F2197F99E31DB0013445B005A1C1F
:10FF300007F5D073A3F5C47333F912300B4497F966
:10FF40009F1197F99E21D2000A440432510007F50F
:10FF5000D072A2F5C47232F91120134497F99F119F
:10FF600097F99E21D2000A44520002F1090107F5D7
:10FF7000D072A2F5C47232F911201344002B00DABA
:10FF800003339B10194697F99F2197F99E319B00E7
:10FF90001A4409B207F5D073A3F5C47323F81210FD
:10FFA00097F99F31DBB20133DBB287F89F3197F9C4
:10FFB0009F31032B7FF75EAF97F99E31DBB20133A0
:10FFC000DBB287F89E3197F99E31032B7FF74EAF56
:10FFD00007F11803203360220021184602F0DAF9F5
:10FFE00007F198034033C0220021184602F0D2F9ED
:10FFF00007F5D073A3F5CE731B6803F23C5307F1EA
:020000040801F1
:1000000098014FF48072184602F07BFA07F5D0731E
:10001000A3F5CE731B6803F5C86307F118018022AE
:10002000184602F06EFA07F5D073A3F5CE731B687D
:1000300003F5A0634FF4F4711846FFF7CBFD0023DE
:10004000A7F89C311BE0B7F89C3103F10802B7F820
:100050009C3107F5D071A1F5CE7109680A4492F878
:10006000001507F5D072A2F5CE72126813440A4645
:1000700083F80025B7F89C310133A7F89C31B7F815
:100080009C31B3F5F27FDED307F5D073A3F5CE73C1
:100090001B6803F5DC6207F5D073A3F5CC7303CBC3
:1000A0001060516007F5D073A3F5CE73186807F59B
:1000B000D073A3F5CE731B6803F5A0624FF4F473FD
:1000C00042F61861FFF76CFB03461A4697F89B311E
:1000D000134387F89B3107F5D073A3F5CE70032344
:1000E0000193FF2300934FF4305301220421006851
:1000F000FFF7B3FD03461A4697F89B31134387F881
:100100009B3197F89B31184607F5D077BD4680BDE7
:10011000384801084048010880B5CAB002AF07F569
:100120009073A3F58E7318600A4607F59073A3F2D7
:100130001D131A70002387F81D319A4A07F58A7338
:1001400092E8030083E80300974A07F5867392E874
:10015000030083E80300954BC7F8083107F5907357
:10016000A3F58E731B6803F5A06007F59073A3F5E4
:100170008E731B6803F5FC734FF44272194602F04C
:10018000C0F907F59073A3F21D131B78102B40F0F4
:10019000D28007F59073A3F58E731B6803F5A163F6
:1001A0001A4607F58A7303CB1060516007F5907308
:1001B000A3F58E731B6803F5A4631A4607F58673CF
:1001C00003CB1060516007F59073A3F58E731B6825
:1001D00003F5A0634FF442711846FFF7FBFC07F5E7
:1001E0009073A3F58E731B6803F2345107F1080373
:1001F0004FF48072184602F084F9002387F81E310C
:100200005DE0002387F81F314EE097F91F2197F931
:100210001E31DB0013445A0007F59073A3F58C736D
:1002200053F8222097F91F1197F91E31DB000B4478
:100230005B00591C07F59073A3F58C7353F82130BC
:100240001A4497F91F1197F91E31DB000B44043350
:10025000590007F59073A3F58C7353F821301A44B5
:1002600097F91F1197F91E31DB000B445B0003F176
:10027000090107F59073A3F58C7353F821301344EB
:1002800097F91F1197F91E2192000A44990807F562
:100290009073A3F58C7343F8221097F91F31DBB2EA
:1002A0000133DBB287F81F3197F91F31032BACDD27
:1002B00097F91E31DBB20133DBB287F81E3197F9B3
:1002C0001E31032B9DDD07F108034033C0220021BE
:1002D000184602F05FF807F59073A3F58E731B685C
:1002E00003F2345307F108014FF48072184602F00C
:1002F00008F907F59073A3F58E731B6803F5A063E7
:100300004FF442711846FFF765FC07F59073A3F5AB
:100310008E731B6803F23463D7F808211A6007F55F
:100320009073A3F58E731B6803F5AF63042200215D
:10033000184602F02FF807F59073A3F58E7318682E
:1003400007F59073A3F58E731B6803F5A0624FF455
:10035000427342F6F841FFF723FA03461A4697F82C
:100360001D31134387F81D3107F59073A3F58E7087
:1003700003230193FF2300934FF430530122042100
:100380000068FFF76AFC03461A4697F81D311343CD
:1003900087F81D3197F81D31184607F59077BD464F
:1003A00080BD00BF4848010850480108A0FC01007A
:1003B00080B584B000AF786039600023FB73002300
:1003C000BB7300237B737B68002247F6FF711846DE
:1003D000FFF7D2F903461A46FB7B1343FB737B6896
:1003E00007F10E0200211846FFF7B4F903461A463A
:1003F000FB7B1343FB737B6807F10D020121184659
:10040000FFF7A8F903461A46FB7B1343FB737B688F
:10041000022247F6FF711846FFF7AEF903461A4667
:10042000FB7B1343FB73BB7BF02B06D17B7B0C2B3D
:1004300003D13B6801221A7002E03B6800221A7067
:10044000FB7B18461037BD4680BD000080B588B0E4
:1004500002AF78600023FB754FF001133B6101236D
:10046000FB600023BB607B68804ADA607B68804A5F
:100470009A607B68002283F8AC2A7B68002247F6EA
:10048000FF711846FFF778F903461A46FB7D1343C0
:10049000FB757B68042209211846FFF76DF90346B6
:1004A0001A46FB7D1343FB757B6840220F211846DB
:1004B000FFF762F903461A46FB7D1343FB757B6821
:1004C00003220A211846FFF757F903461A46FB7D17
:1004D0001343FB757B6807F1160247F6FF71184658
:1004E000FFF738F903461A46FB7D1343FB757B681B
:1004F00001220C211846FFF73FF903461A46FB7DFF
:100500001343FB757B68002240F201111846FFF788
:1005100033F903461A46FB7D1343FB757B680022C3
:100520004FF481711846FFF727F903461A46FB7D01
:100530001343FB757B6801224FF485711846FFF762
:100540001BF903461A46FB7D1343FB757B680122AA
:1005500044F202011846FFF70FF903461A46FB7DE5
:100560001343FB757B68002244F202011846FFF733
:1005700003F903461A46FB7D1343FB757B68032290
:100580004FF485711846FFF7F7F803461A46FB7DCE
:100590001343FB757B68012240F203111846FFF7F5
:1005A000EBF803461A46FB7D1343FB757B6800227C
:1005B0000C211846FFF7E0F803461A46FB7D13436B
:1005C000FB757B6843220F211846FFF7D5F80346D9
:1005D0001A46FB7D1343FB757B6801211846FFF724
:1005E0002FFB03461A46FB7D1343FB757B684022B5
:1005F0000F211846FFF7C0F803461A46FB7D134348
:10060000FB757B6801220A211846FFF7B5F80346FF
:100610001A46FB7D1343FB757B6864211846FFF780
:100620000FFB03461A46FB7D1343FB757B680022D4
:1006300047F6FF711846FFF79FF803461A46FB7D01
:100640001343FB7501230193FF230093062300222C
:1006500001217868FFF701FB03461A46FB7D13432F
:10066000FB75FB7D002B40F0098303E0189D020819
:100670004C9902087B6801220E211846FFF77CF88E
:1006800003461A46FB7D1343FB757B68022247F63F
:10069000FF711846FFF770F803461A46FB7D1343B7
:1006A000FB757B68012247F6FF711846FFF764F877
:1006B00003461A46FB7D1343FB757B680122062126
:1006C0001846FFF759F803461A46FB7D1343FB759E
:1006D00004230193FF230093212300220121786842
:1006E000FFF7BBFA03461A46FB7D1343FB757B6895
:1006F000002247F6FF711846FFF73EF803461A46F8
:10070000FB7D1343FB757B6807F1160247F6FF710B
:100710001846FFF71FF803461A46FB7D1343FB7587
:100720007B6801220C211846FFF726F803461A467B
:10073000FB7D1343FB757B68002247F6FF7118466B
:10074000FFF71AF803461A46FB7D1343FB757B68D7
:10075000002240F201111846FFF70EF803461A4630
:10076000FB7D1343FB757B6800224FF481711846B3
:10077000FFF702F803461A46FB7D1343FB757B68BF
:1007800001224FF485711846FEF7F6FF03461A461C
:10079000FB7D1343FB757B68012244F2020118467E
:1007A000FEF7EAFF03461A46FB7D1343FB757B68A1
:1007B000002244F202011846FEF7DEFF03461A4605
:1007C000FB7D1343FB757B6803224FF4857118464C
:1007D000FEF7D2FF03461A46FB7D1343FB757B6889
:1007E000012240F203111846FEF7C6FF03461A46DF
:1007F000FB7D1343FB757B68002244F20F01184612
:10080000FEF7BAFF03461A46FB7D1343FB757B6870
:10081000432240F21A211846FEF7AEFF03461A465D
:10082000FB7D1343FB757B68032240F21A211846B7
:10083000FEF7A2FF03461A46FB7D1343FB757B6858
:10084000012240F21A211846FEF796FF03461A4687
:10085000FB7D1343FB757B68002240F21A2118468A
:10086000FEF78AFF03461A46FB7D1343FB757B6840
:10087000002240F219211846FEF77EFF03461A4671
:10088000FB7D1343FB757B68002240F21B21184659
:10089000FEF772FF03461A46FB7D1343FB757B6828
:1008A000002247F6FF711846FEF766FF03461A4618
:1008B000FB7D1343FB757B6807F1160247F6FF715A
:1008C0001846FEF747FF03461A46FB7D1343FB75A8
:1008D0007B68012247F6FF711846FEF74DFF03467D
:1008E0001A46FB7D1343FB757B68092247F6FF71AF
:1008F0001846FEF741FF03461A46FB7D1343FB757E
:1009000078684FF40043DE4A0021FEF749FF0346B2
:100910001A46FB7D1343FB757B680A2247F6FF717D
:100920001846FEF729FF03461A46FB7D1343FB7565
:1009300078684FF40043D34A0021FEF731FF0346A5
:100940001A46FB7D1343FB757B680B2247F6FF714C
:100950001846FEF711FF03461A46FB7D1343FB754D
:1009600078684FF4A043C84A0021FEF719FF0346F8
:100970001A46FB7D1343FB757B68012247F6FF7126
:100980001846FEF7F9FE03461A46FB7D1343FB7536
:100990007B68012247F6FF711846FEF7EDFE03461D
:1009A0001A46FB7D1343FB757B680322062118461C
:1009B000FEF7E2FE03461A46FB7D1343FB757B6898
:1009C00005211846FFF73CF903461A46FB7D134301
:1009D000FB757B68002247F6FF711846FEF7CCFED8
:1009E00003461A46FB7D1343FB757B6807F116022D
:1009F00047F6FF711846FEF7ADFE03461A46FB7D2B
:100A00001343FB757B6801220C211846FEF7B4FEE8
:100A100003461A46FB7D1343FB757B68002247F6AD
:100A2000FF711846FEF7A8FE03461A46FB7D1343E6
:100A3000FB757B6800224FF48A711846FEF79CFE16
:100A400003461A46FB7D1343FB757B68002240F288
:100A500015111846FEF790FE03461A46FB7D134318
:100A6000FB757B6842224FF48B711846FEF784FEBB
:100A700003461A46FB7D1343FB757B68002240F258
:100A800017111846FEF778FE03461A46FB7D1343FE
:100A9000FB757B6800220B211846FEF76DFE0346AE
:100AA0001A46FB7D1343FB757B6807F1160247F678
:100AB000FF711846FEF74EFE03461A46FB7D1343B0
:100AC000FB757B6800220C211846FEF755FE034695
:100AD0001A46FB7D1343FB757B6801220B211846E8
:100AE000FEF74AFE03461A46FB7D1343FB75786802
:100AF000FFF703F903461A46FB7D1343FB75FB7DA5
:100B0000002B40F0C9807B68022247F6FF7118462F
:100B1000FEF732FE03461A46FB7D1343FB757868E9
:100B20007B6803F5A062042342F6FC71FEF756FFD2
:100B300003461A46FB7D1343FB757B6803F5A063F0
:100B400004211846FFF746F87B6803F5A0631B688D
:100B5000BB60BB684D4A934204D0FB7D43F0050364
:100B6000FB759AE078682823494A42F6D871FEF767
:100B700017FE03461A46FB7D1343FB7502230193C0
:100B8000FF2300934FF43053002204217868FFF7CD
:100B900064F803461A46FB7D1343FB7578687B684F
:100BA00003F5A0624FF4F67342F60441FEF716FF18
:100BB00003461A46FB7D1343FB757B6803F1100067
:100BC0007B6803F5A0634FF4F472194601F099FCB9
:100BD00010217868FFF7D4F803461A46FB7D1343CB
:100BE000FB757B6803F5FC732A4A184611464FF4DF
:100BF00042731A4601F085FC10217868FFF78CFAE1
:100C000003461A46FB7D1343FB7578687B689A6838
:100C10004FF4737342F63441FEF7C2FD03461A46A1
:100C2000FB7D1343FB7503230193FF2300934FF4D4
:100C30003053012204217868FFF70FF803461A4663
:100C4000FB7D1343FB7507F1100104234DF6803241
:100C5000786800F0F5FE03461A46FB7D1343FB75EA
:100C600007F10C0104234DF66412786800F0E8FEE9
:100C700003461A46FB7D1343FB750EE000BF0CE0F4
:100C80004C4901084CC901084C4902089E6C0B0CE8
:100C900020A00208189D020800BFFB7D18461837E7
:100CA000BD4680BDB0B59CB002AF7860002387F828
:100CB000673000233B6500237B654FF44073FB6482
:100CC00007F15B031946786800F05AFC03461A46A0
:100CD00097F86730134387F867307B6800225A60C3
:100CE0007B68FF229A70B84B07F13C040FCB84E875
:100CF0000F00B64B07F10C041D460FCD0FC40FCDEE
:100D00000FC495E80F0084E80F00FB6B0833FB630A
:100D1000FB6B1033FB63FB6B2033FB63FB6B4033DC
:100D2000FB63FB6B8033FB63FB6B03F58073FB633F
:100D3000FB6B03F50073FB63FB6B03F58063FB63E5
:100D4000FB6B03F50063FB6300233B6673E03B6EC4
:100D50009B0068333B4453F85C3C002B67D03B6EF0
:100D60005B099B0068333B4453F82C2C3B6E03F02B
:100D70001F0322FA03F303F00103002B57D007F1FE
:100D80000C023B6E9B001344FB65FB6D1B7803F06C
:100D90000F03DBB2002B3AD0FB6D1B78C3F30303C8
:100DA000DBB20C2B33D8FB6D5B8845F2CF4293420C
:100DB00010D9FB6D5B8845F68F0293420AD897F8ED
:100DC0005B30C3F30B0399B2FA6D138861F30F1311
:100DD000138009E097F85B30C3F30B0399B2FA6D07
:100DE000138861F30F1313807B685B68FA6D1278C8
:100DF000C2F30302D2B21146FA6D1288C2F30B128B
:100E000092B201FB02F21A447B685A6009E07B68E7
:100E10005B68FA6D1288C2F30B1292B21A447B68B7
:100E20005A607B685B681A1D7B685A6000E000BFEF
:100E30003B6E01333B663B6E0B2B88D97B685B684E
:100E400003F118027B685A6007F10C0130234DF65C
:100E50008012786800F0F4FD03461A4697F8673070
:100E6000134387F867307B685B683B653B6E0133F3
:100E70007B6507F1500108234DF66812786800F091
:100E8000DFFD03461A4697F86730134387F867304B
:100E900007F13C0110234DF67012786800F0D0FD88
:100EA00003461A4697F86730134387F867307B6824
:100EB000002247F6FF711846FEF75EFC03461A460D
:100EC00097F86730134387F867307B68052209215C
:100ED0001846FEF751FC03461A4697F8673013434D
:100EE00087F867307B68022247F6FF711846FEF7E5
:100EF00043FC03461A4697F86730134387F8673078
:100F0000786807F14C02042342F6FC71FEF748FCB6
:100F100003461A4697F86730134387F86730032370
:100F20000193FF2300934FF430530122042178688A
:100F3000FEF793FE03461A4697F86730134387F887
:100F400067307B6803F5A0610C2345F24042786866
:100F500000F0ECFC03461A4697F86730134387F815
:100F600067307B6803F5A1631B889BB2A7F85830F4
:100F7000B7F858301A467B685B689A4202D0FF2364
:100F800087F867307B6803F5A06108234EF2C4023E
:100F9000786800F0CBFC03461A4697F86730134395
:100FA00087F867307B6893F80635002B05D097F8F3
:100FB000673043F0030387F8673097F867301846C7
:100FC0006837BD46B0BD00BF5848010868480108F1
:100FD00080B586B000AF78600023FB740023FB75FA
:100FE0000023BB820023FB60786807F10C02042316
:100FF00042F6FC71FEF7F2FC03461A46FB7D1343F2
:10100000FB75FB6840F2FF4293424DD07B6893F83A
:10101000AC3A002B48D17B68002247F6FF71184696
:10102000FEF7AAFB03461A46FB7D1343FB757B685C
:10103000162215211846FEF79FFB03461A46FB7D34
:101040001343FB757B68012214211846FEF794FBBD
:1010500003461A46FB7D1343FB7521E07B6807F1CD
:10106000130206211846FEF775FB03461A46FB7D60
:101070001343FB757B680A211846FEF7E1FD034622
:101080001A46FB7D1343FB75BB8A0133BB82BB8AC7
:10109000B3F5FA7F04D9FA7CFB7D1343FB7503E0BB
:1010A000FB7C5BB2002BD9DA7B6807F113020621C7
:1010B0001846FEF74FFB03461A46FB7D1343FB75AC
:1010C000FB7C5BB2002B15DA7B6807F1130207216A
:1010D0001846FEF73FFB03461A46FB7D1343FB759C
:1010E000FB7C842B06D0FB7C852B03D0FA7CFB7D1C
:1010F0001343FB757B68002247F6FF711846FEF725
:101100003BFB03461A46FB7D1343FB757B680022BD
:1011100014211846FEF730FB03461A46FB7D1343A5
:10112000FB757B68002215211846FEF725FB034658
:101130001A46FB7D1343FB757B6804220921184680
:10114000FEF71AFB03461A46FB7D1343FB757B68CB
:10115000022247F6FF711846FEF70EFB03461A46B9
:10116000FB7D1343FB75FB7D18461837BD4680BDDC
:1011700080B588B000AF786039600023FB7778686D
:101180007B6803F5A0627B685B680021FEF726FCA4
:1011900003461A46FB7F1343FB777B6893F80025D1
:1011A0007B689A707B6803F5A0627B685B689BB282
:1011B00019461046FEF70EFD1023BB610EE1BB6918
:1011C00003F5A0637A681344BB60BB681B78C3F364
:1011D0000303DBB2012B15D9BB681B78C3F30303F0
:1011E000DBB20C2B0ED8BB681B78C3F30303DBB256
:1011F0001A46BB681B88C3F30B139BB202FB03F3B5
:101200003B6105E0BB681B88C3F30B139BB23B61DA
:10121000BB685B884EF28402934200F0BB804EF2C2
:101220008402934200F3D2804EF24402934200F0D3
:10123000A3804EF24402934200F3C8804DF64472FC
:10124000934200F08B804DF64472934200F3BE80CF
:101250004DF6C462934273D04DF6C462934200F3DC
:10126000B5804DF6C43293425CD04DF6C432934201
:1012700000F3AC804DF68432934245D04DF6843273
:10128000934200F3A3804DF65802934200F0908001
:101290004DF65802934200F3998045F2D0529342A2
:1012A00024D045F2D052934200F3908045F2B442EC
:1012B000934204D045F2D04293420AD086E0BB6903
:1012C0000C337A68134493F800355AB23B681A70AD
:1012D0007DE03B68181DBB69043303F5A0637A68A1
:1012E00013443A69194601F00CF970E03B6803F5C4
:1012F000A270BB69043303F5A0637A6813443A69AA
:10130000194601F0FEF862E03B6803F58270BB69A4
:10131000043303F5A0637A6813443A69194601F06F
:10132000F0F854E03B6803F51170BB69043303F532
:10133000A0637A6813443A69194601F0E2F846E07E
:101340003B6803F55170BB69043303F5A0637A6809
:1013500013443A69194601F0D4F838E03B6803F5C4
:101360007170BB69043303F5A0637A6813443A696A
:10137000194601F0C6F82AE03B6803F24440BB6915
:10138000043303F5A0637A6813443A69194601F0FF
:10139000B8F81CE03B6803F28440BB69043303F5F2
:1013A000A0637A6813443A69194601F0AAF80EE07E
:1013B0003B6803F2C440BB69043303F5A0637A6859
:1013C00013443A69194601F09CF800E000BFBA697D
:1013D0003B691344BB61BB690433BB617B685B68D9
:1013E000BA699A42FFF4EBAE0023BB610DE03A68A4
:1013F000BB699B0013445B68DA0A3968BB699B00D0
:101400000B445A60BB690133BB61BB693F2BEED90A
:101410000023BB6144E03A68BB6903F5F0735B00ED
:101420001344B3F90430002B00DA03339B1019B2D4
:101430003A68BB6903F5F0735B0013440A469A806F
:101440003A68BB69134403F244431B785B08D9B282
:101450003A68BB69134403F244430A461A703A6877
:10146000BB6903F5D0735B0013449B88DB0999B219
:101470003A68BB6903F5D0735B0013440A469A804F
:101480003A68BB6990339B0013445B68DA0A396899
:10149000BB6990339B000B445A60BB690133BB614D
:1014A000BB693F2BB7D90023BB611BE03A68BB691E
:1014B000134403F582731B78002B10D100237B614A
:1014C0000AE0BA697B6913443A681344FF2283F83F
:1014D00084247B6901337B617B69002BF1D0BB697C
:1014E0000133BB61BB693F2BE0D90023BB6114E032
:1014F0003A68BB6903F599739B0013449B681F4AC4
:10150000A2FB0323DA0B3968BB6903F599739B00CF
:101510000B449A60BB690133BB61BB691F2BE7D9E0
:101520007B6893F808351B02FB817B6893F80935CB
:101530001A46FB891343FB817B685B68043B7A682E
:10154000134493F800351B02BB817B685B68033B47
:101550007A68134493F800351A46BB891343BB815C
:10156000FA89BB899A4203D0FB7F43F00203FB77E1
:10157000FB7F18462037BD4680BD00BF018000803C
:1015800080B584B000AF786039600023FB737B685E
:1015900003F5A061082345F25042786800F0C6F9CF
:1015A00003461A46FB7B1343FB737B6893F80025C5
:1015B0007B6893F8013512FB03F3DAB23B681A70CB
:1015C000FB7B18461037BD4680BD80B584B000AFA8
:1015D00078600B46FB700023FB73FB78102B02D066
:1015E000402B55D0A9E07B6803F5A06110234AF693
:1015F0003852786800F09AF903461A46FB7B134389
:10160000FB737B68402283F804257B68402283F8C3
:1016100006257B68042283F809257B6803F5A06111
:1016200010234AF63852786800F00AFA03461A4640
:10163000FB7B1343FB737B6803F5A061082345F232
:101640005042786800F072F903461A46FB7B134358
:10165000FB737B68042283F800257B68042283F8EF
:1016600001257B68082283F804257B68082283F81B
:1016700005257B6803F5A061082345F25042786890
:1016800000F0DEF903461A46FB7B1343FB7357E079
:101690007B6803F5A06110234AF63852786800F0A1
:1016A00045F903461A46FB7B1343FB737B68102204
:1016B00083F804257B68102283F806257B680122C5
:1016C00083F809257B6803F5A06110234AF6385298
:1016D000786800F0B5F903461A46FB7B1343FB73A9
:1016E0007B6803F5A061082345F25042786800F05A
:1016F0001DF903461A46FB7B1343FB737B680822E4
:1017000083F800257B68082283F801257B68042282
:1017100083F804257B68042283F805257B6803F59C
:10172000A061082345F25042786800F089F9034629
:101730001A46FB7B1343FB7302E07F23FB7300BF5E
:10174000FB7819467868FEF71BFB03461A46FB7BBD
:101750001343FB73FB7819467868FEF7DDFC0346FC
:101760001A46FB7B1343FB73FB7B18461037BD46C1
:1017700080BD80B588B004AF78600B46FB70002355
:10178000FB737B6803F5A06101230293012301939E
:10179000FB1C0093042345F25842786800F0EEF9F0
:1017A00003461A46FB7B1343FB73FB7B184610373B
:1017B000BD4680BD80B588B004AF78600B46FB7035
:1017C0000023FB73FB78632B04D9FB7B43F07F037F
:1017D000FB7320E0FA7813461B029B1A104A82FB27
:1017E00003125211DB17D31ADBB2BB737B6803F50C
:1017F000A0610D2302930123019307F10E030093CF
:1018000010234AF6D862786800F0B8F903461A4601
:10181000FB7B1343FB73FB7B18461037BD4680BD33
:101820001F85EB5180B588B004AF78600B46FB7024
:101830000023FB73FB78012B02D0FB78022B14D121
:101840007B6803F5A0610023029301230193FB1C35
:10185000009304234AF66462786800F08FF9034627
:101860001A46FB7B1343FB7303E0FB7B43F07F03D0
:10187000FB73FB7B18461037BD4680BD80B584B036
:1018800000AF78600B46FB700023FB730023BB6046
:101890007B6803F5A06108234AF63052786800F0AF
:1018A00045F803461A46FB7B1343FB73FB78012B79
:1018B00002D0032B0BD015E07B68012283F80125B1
:1018C0007B68032283F803250023BB600DE07B685F
:1018D000032283F801257B68022283F80325012374
:1018E000BB6002E07F23FB7300BF7B6803F5A06150
:1018F00008234AF63052786800F0A2F803461A46E8
:10190000FB7B1343FB7307F1080104234DF66412BC
:10191000786800F095F803461A46FB7B1343FB7387
:10192000FB7B18461037BD4680BD000080B58CB0EB
:1019300002AFF860B9607A607B80002387F82530B9
:101940007B880C333B623D4A07F1140307CA83E8E6
:1019500007007B88B3F5B46F03D9FF2387F82530E0
:1019600065E07B681B0ADBB23B757B68DBB27B758D
:101970007B881B11DBB2BB757B88DBB21B01DBB242
:10198000FB75F86807F114020C2342F6F471FDF7B9
:1019900007FF03461A4697F82530134387F825308A
:1019A00003230193FF2300934FF4305301220421BA
:1019B000F868FEF752F903461A4697F825301343A4
:1019C00087F82530F868FB6803F5A0623B6A42F6A9
:1019D0000441FEF703F803461A4697F825301343EF
:1019E00087F82530FB6803F5A0627B880C339BB237
:1019F00019461046FEF7EEF80023FB8411E0B7F914
:101A000026301A1DB7F92630B9680B44F9680A4424
:101A100092F800251A70B7F926309BB201339BB2B9
:101A2000FB84B7F90230B7F926209A42E7DB97F832
:101A3000253018462837BD4680BD00BF98480108AC
:101A400080B58CB002AFF860B9607A607B8000230B
:101A500087F827300023FB6100233B7500237B754B
:101A60000023BB750F23FB7505233B7601237B7693
:101A70007B8808331B12DBB2BB767B88DBB2083372
:101A8000DBB2FB767B88C3F53F5334337B847B88A2
:101A9000B3F5B46F03D9FF2387F8273068E07B687C
:101AA0001B0ADBB23B777B68DBB27B777B881B1141
:101AB000DBB2BB777B88DBB21B01DBB2FB777B88B9
:101AC0001946B868FEF786F87B88013B9BB2BB8459
:101AD00012E0B7F92430BA681A44B7F92430043355
:101AE0001178FA6813440A4683F80025B7F92430C0
:101AF0009BB2013B9BB2BB84B7F92430002BE8DAE0
:101B0000FB6803F5A063FA691A607B88043303F568
:101B1000A063FA6813441A4607F1140303CB10605C
:101B20005160F868FB6803F5A0627B880C33798C00
:101B3000FDF736FE03461A4697F82730134387F819
:101B4000273003230193FF2300934FF430530122E6
:101B50000421F868FEF781F803461A4697F8273003
:101B6000134387F827307B881946B868FEF732F8A8
:101B700097F8273018462837BD4680BD80B586B017
:101B800000AFF860B9607A607B800023FB757B88CA
:101B90007A68B968F868FFF7C9FE03461A46FB7D04
:101BA0001343FB753B8DBA681344BA8C396A1846E7
:101BB00000F0A7FC7B887A68B968F868FFF740FFF7
:101BC00003461A46FB7D1343FB75FB7D1846183709
:101BD000BD4680BD0A22002100F07AB8242B2DE9F1
:101BE000F0478646904601D8012B06D100F05CFCF8
:101BF000162303600020BDE8F08734480D462A46CE
:101C000015F8014B065D16F00806F8D12D2C10D101
